:0900000C32322E312E302E31313A
:1000000A4863694B8F846A458A969A7954797F57EF
:1000000A9782865B636462656468666B6C67AEA29E
:1000000A945FB4A7B1966E8C8F71B19E8D907685F0
:1000000A838084888383878B86838F91928E938E55
:1000000A8E929691938F9B9D9E9A9F9A9A9EA29D5D
:1000000A9AA4A3AAA5AAA5A5A9ADA8A5AEAEB5B05E
:1000000AB5B0B0B4B8B3B0D3B5D7A8DECDD0B6D0FA
:1000000AD4B9F9D7BC05F9EBB6ECDBDEC4EEF2C71E
:0200000AECEC1C
:020000040800F2
:4080000028F00020CDC70308DFC70308F1F60308E3C70308E5C70308E7C703080000000000000000000000000000000021830008EBC7030800000000E583000859840008E3
:40804000F1C70308F1C70308F1C70308F1C70308F1C70308F1C70308F1C70308F1C70308F1C70308F1C70308F1C70308F1C70308F1C70308F1C70308F1C70308F1C70308D0
:40808000F1C70308F1C703087D5E0308DB630308EF640308F1C70308F1C70308F1C7030837C7030843C703084FC70308C7C60308E9C60308F7C6030803C70308198F030883
:4080C000298F0308398F0308438F0308F1C703084D980308196F0308236F03082D6F0308F1C70308F1C70308F1C703085BC7030867C7030873C703082BC70308F1C70308CF
:40810000F1C70308F1C703080DC70308F1C70308F1C70308F1C7030819C7030823C70308F1C70308F1C70308F1C70308F1C70308F1C70308F1C70308F1C703089564030858
:4081400063650308D9650308F1C70308F1C70308F1C70308F1C70308F1C703084B6F03084D8F03085D8F0308F1C70308F1C70308F1C70308F1C70308F1C7030800000000A2
:40818000F1C70308F1C70308556F03085F6F0308F1C70308F1C7030857980308F1C703080000000000000000F1C7030800F002F800F073F80AA090E8000C82448344AAF1F0
:4081C0000107DA4501D100F068F8AFF2090EBAE80F0013F0010F18BFFB1A43F001031847A0020400C00204000A444FF0000C10F8013B13F0070408BF10F8014B1D1108BFD1
:4082000010F8015B641E05D010F8016B641E01F8016BF9D113F0080F1EBF10F8014BAD1C0C1B09D16D1E58BF01F801CBFAD505E014F8016B01F8016B6D1EF9D59142D6D37C
:40824000704700000023002400250026103A28BF78C1FBD8520728BF30C148BF0B607047632937F0E680732937F0EB80002070471FB53BF0E0FD9DE8030037F06FF836F0E8
:40828000F4FE37F0BEF90400002000213AF004FF401C60601FBD10B510BD37F08DF91146FFF7E6FF12F035FE37F0BEF903B4FFF7F2FF03BC37F0EEF980F309887047EFF3F8
:4082C00009807047684680F3098804480078C00714BF0220032080F314887047C8730408DFF818C0EFF305831B0618BF6047EFF31483DB0708BF604700DF70471F22040878
:40830000DFF818C0EFF305831B0618BF6047EFF31483DB0708BF604700DF704725240408EFF30980816911F8021C01B142E010B590E80F10E047BDE81040EFF3098C254B22
:4083400093E80600914232D041B91EF0100F16D12149086820F00100086010E00CB41EF0100F06BF2CED108A0323012381F826302CE9F00FC1F82CC03AF0EAFB0CBC1A60CE
:40838000D2F82CC0BCE8F00F92F8263013F0020F1ABFBCEC108A6FF0120E6FF0020E8CF3098813F0010F08BF704792F82500CCF80000704710B5094A1268914209D8084C02
:4083C00054F8214090E80F10A047EFF3098C8CE80F0010BD0808002034EF00E0E0F60308E0F6030810B53AF067FABDE81040194B93E80600914208BF70470CB4EFF3098CE4
:408400001EF0100F06BF2CED108A0223002381F826302CE9F00FC1F82CC03AF099FB0CBC1A60D2F82CC0BCE8F00F92F8263013F0020F1ABFBCEC108A6FF0120E6FF0020E71
:408440008CF3098813F0010F1CBF92F82530CCF8003070470808002010B53AF049FCC4E710B539F0DBFE3AF043FCBEE70B49D1F800C04A685CF8043B1068184442F8040B51
:408480008C4528BFA1F1DC0C8A4228BFA1F1DC02C1F800C04A6020F00040704720EA00200146FB48B0F8AA0000EE100AB8EE400A81ED080AF64890ED800A81ED010A90ED84
:4084C000810A81ED020A90ED820A81ED030A90F8AF0000EE100AB8EE400A81ED050AEC4890F8AE000877EA4890ED7D0A81ED000A90F8B00000EE100AB8EE400A81ED060A02
:40850000B7EE000A81ED040A012070474FF6FF76DFF880C300DF074639460120DFF878C300DF0421DD4880F8D0110021DC4880F8441000BF002231460120DFF868C300DF99
:408540000446012C17D100BFD44890F8D10140F00101D24880F8D111B0F8DC014FF6FF71884207DACD48B0F8DC01401C81B2CB48A0F8DC11DEE7022CDCD1DFF82CC300DFD6
:40858000054605F001000028D4D0C548FFF788FFD0E7C34880ED0C0ADFEDC40AC0ED0D0ADFEDC20AC0ED0F0ADFEDC00AC0ED0E0A80ED0A0A704710B52DED0C8BB0EE409AA2
:4085C000B0EE608AF0EE419A9FEDB80AF0EE408A2422B349243101F1240036F0DCFD9FEDB40AC9EE000AAE48C0ED090AB5EEC08AF1EE10FA04D1B0EE480AFFF7CAFF10E18C
:40860000B5EEC08AF1EE10FA07DDA54890ED130AB5EEC00AF1EE10FA0CD9B5EEC08AF1EE10FA0FD29E4890ED130AB5EEC00AF1EE10FA07DBB0EE480AFFF7ABFF31F0C9F9DC
:4086400097490867964A92ED080ABCEEC00A10EE101A106F31F0C3F950BBB5EEC08AF1EE10FA0ADD9FED930A8D4880ED0A0A9FED8F0A914880ED000A11E09FED900A88489F
:4086800080ED0A0AD0ED050AB7EE001A81EE200AF0EE000A80EE201A874880ED001A804890ED0A0A80ED0C0A012085490870B8E09FED800AB4EEC08AF1EE10FA07DB9FEDFB
:4086C000810A774880ED0A0AF0EE488A80E09FED7B0AB4EEC08AF1EE10FA07D89FED7A0A6F4880ED0A0AF0EE488A71E0724890ED000A30EE290A80ED000A694890ED050A4B
:40870000DFED720A20EE200A6B48D0ED000A20EE200A10EE101A08463BF01CFB41EC1D0BB0EE4D0AF0EE6D0A38F0AEFDB0EE40BAF0EE60BA5A4890ED060A10EE101A0846A8
:408740003BF008FB41EC1C0B53EC1B2B3BF00CF841EC1A0B3AF0C2FC08EE900AF5EEC08AF1EE10FA05DD4E4890ED060AF0EE408A06E04B4890ED060AB1EE400AF0EE408A9F
:4087800038EE880AF0EE408AB5EEC08AF1EE10FA09DDF5EEC08AF1EE10FA04D89FED4C0AF0EE408A0DE0B5EEC08AF1EE10FA08D2F5EEC08AF1EE10FA03DB9FED460AF0EED6
:4087C000408A374890ED000A20EE280A80ED0A0A3B48007870B13248C0ED0C8A90ED0A0AD0ED090A30EE600A80ED0D0A00203449087016E09FED2D0A2949243101F12400F7
:4088000016F033FA26493431A1F1300015F08EFEF0EE408A224890ED0C0A30EE280A80ED0C0A1F4890ED0A0AB5EEC00AF1EE10FA0BDD90ED0C0AB5EEC00AF1EE10FA04D271
:408840009FED1A0A80ED0C0A54E0154890ED0A0AB5EEC00AF1EE10FA0BD290ED0C0AB5EEC00AF1EE10FA04DD9FED100A80ED0C0A40E00B4890ED0C0ADFED0E0AB4EEE00A07
:40888000F1EE10FA28DD9FED0B0A80ED0C0A31E018210020C92F04088923040860420020CC160020E9230408312304080000000000007A440000C842940300200000C8C23B
:4088C0009003002066662640666626C0DB0FC9400AD7233C0AD723BCF74890ED0C0A5FED090AB4EEE00AF1EE10FA03D21FED0D0A80ED0C0AF04890ED0C0ABDEC0C8B10BDF5
:4089000001B500BF01226946EC480068B03012F0BBFD20B99DF80000E94981F8B00000BFE848D0F8CC110120DFF89CC300DF08BD10B52DED020B00BF04226946DF48006853
:4089400000F5FA7012F0A0FD20B99DED000ADC4880ED7D0A00BFDB48D0F8CC110120DFF868C300DF1CBD01B500BF01226946D3480068AE3012F088FD20B99DF80000D0495C
:4089800081F8AE0000BFCF48D0F8CC110120DFF838C300DF08BD01B500BF01226946C7480068AF3012F070FD20B99DF80000C44981F8AF0000BFC348D0F8CC110120DFF868
:4089C00008C300DF08BD10B52DED020B00BF04226946BA48006800F5027012F055FD20B99DED000AB64880ED820A00BFB548D0F8CC110120DFF8D0C200DF1CBD10B52DED7D
:408A0000020B00BF04226946AC48006800F5017012F03AFD20B99DED000AA94880ED810A00BFA848D0F8CC110120DFF89CC200DF1CBD10B52DED020B00BF042269469F487B
:408A4000006800F5007012F01FFD20B99DED000A9B4880ED800A00BF9A48D0F8CC110120DFF864C200DF1CBD01B500BF0222694692480068AA3012F007FD20B9BDF80000B0
:408A80008F49A1F8AA0000BF8E48D0F8CC110120DFF834C200DF302004F05CFD08BD10B58AB00446022C1FD1B2EE040A8DED090A9FED860A8DED020A1FED840A8DED030ACD
:408AC0009FED820A8DED040A9FED810A8DED060A01208DF820009FED7F0A8DED010AB1EE080A8DED070AA8E0042C1FD1B3EE080A8DED090A1FED910A8DED020A1FED950AD9
:408B00008DED030A1FED950A8DED040A1FED970A8DED060A01208DF820009FED6F0A8DED010AB1EE040A8DED070A86E0052C01D01A2C1FD1B2EE060A8DED090A9FED670AE4
:408B40008DED020A1FEDA70A8DED030A9FED630A8DED040A1FEDA90A8DED060A01208DF820009FED5F0A8DED010AB2EE020A8DED070A62E00E2C1FD1B2EE040A8DED090A43
:408B80009FED520A8DED020A1FEDB80A8DED030A9FED520A8DED040A9FED4D0A8DED060A01208DF820009FED4E0A8DED010AB2EE040A8DED070A40E0152C1FD1B2EE040AAE
:408BC0008DED090A9FED470A8DED020A1FEDC90A8DED030A9FED430A8DED040A9FED3C0A8DED060A01208DF820009FED3A0A8DED010AB1EE080A8DED070A1EE01FEDD50A22
:408C00008DED090A1FEDD70A8DED020A1FEDD90A8DED030A1FEDDB0A8DED040A1FEDDD0A8DED060A00208DF820001FEDE00A8DED010A1FEDE20A8DED070A9DED090ABDEEBD
:408C4000C00A10EE101A08B2FFF70EFFDDED020AB0EE600AFFF7EDFEDDED030AB0EE600AFFF7CCFEDDED040AB0EE600AFFF7ABFE9DED060ABCEEC00A10EE101AC8B2FFF7C2
:408C80008AFE9DF82000FFF76EFEDDED010AB0EE600AFFF74DFE9DED070ABCEEC00A10EE101AC8B2FFF72CFE302004F053FC552004F050FC0AB010BDCC160020F003002042
:408CC000182100206042002089230408000048420000A042F3FDD43CA69B443C0000484396438B3C0000F042204890ED0A0ABDEEC00A10EE100A00B270471C4890ED090A34
:408D0000BDEEC00A10EE100A00B2704780220270164A92ED010ADFED160A20EE200ABCEEC00A10EE102A91B241700A0A82700F4A92ED020ADFED0E0A20EE200ABCEEC00A01
:408D400010EE102A91B2C1700A0A0271074A92ED030ADFED070A20EE200ABCEEC00A10EE102A91B241710A0A82717047CC1600200000C84270B5054601249048DFF840C21D
:408D800000DF204670BD8F49097801708E49416001218160002181764176704700B5A1B06846FFF7F0FF01208DF8180006219DF81920501CC0B28DF819000DF14B00815490
:408DC00000208DF819006846019930F0D3FA002021B000BD00B5A1B06846FFF7D4FF02208DF8180005219DF81920501CC0B28DF819000DF14B00815400208DF8190068469C
:408E0000019930F0B7FA9DF81800401E0DF11B01085C21B000BD2DE9F74F814615464FF000081FFA89F7E8191FFA80FBBBF5005F02DD4FF0080854E02D2D02DD4FF040088C
:408E40004FE04FF47A615D48DFF880C100DF012802D14FF0100844E0842035F0A1FF044654B3FFF79BFFFFF7B5FF82462046FFF78AFFE81C20760221627E501C607604F11D
:408E80004B008154390A627E501C607604F14B008154627E501C607604F14B008754627E014650182A46019936F030F9002060762046616830F05EFA94F8800001280BD145
:408EC000FFF788FF06460AF0020010B106F0020020B14FF0800801E04FF02008204635F09AFF3648DFF8E8C000DFB8F1000F05D03848007840EA0800364908704046BDE83B
:408F0000FE8F2DE9F043A1B080460F4614460026BDB260191FFA80F9B9F5005F01DD082642E02D2C01DD40263EE06846FFF72BFFE01CC0B28DF8180003219DF81920501CC8
:408F4000C0B28DF819000DF14B008154290A9DF81920501CC0B28DF819000DF14B0081549DF81920501CC0B28DF819000DF14B0085549DF81920014650185522214636F03B
:408F80003CF900208DF819006846019930F0F2F99DF88000012806D122460DF11E01404636F0B4F800E0202626B10A480078304308490870304621B0BDE8F083BC460020F5
:408FC0005D2704083E07002000380040512804086D270408ED03002000487047E4E80020401ECAB210F8011F8A4202D00029F9D10020704720F07CBFFFFFFFFFFFFFFFFF37
:40900000FE4890ED0A0A704710B52DED048BB0EE408A0446F94890ED720ADFEDF90A80EE201AB0EE419AF74890F8AE0058B1FFF7E7FFF0EE409A9FEDF41AF0EE480AFFF786
:40904000BAFAB0EE408AEF4890F89C00012803D1B1EE480AB0EE408A9FEDEC0AB4EEC08AF1EE10FA04D29FEDE90AB0EE408A0AE09FEDE70AB4EEC08AF1EE10FA03DD9FED67
:40908000E40AB0EE408A0E2C14D008DCA4F10200052866D2DFE800F0111410124B00A4F1120009285DD2DFE800F0430C5C065C5C0D5C0A0000BF00BF00BF00BF00BF00BFFF
:4090C00000BF00BFB5EEC08AF1EE10FA0ED2B1EE480AB0EE408A0021CE4800782EF0E6F80121CD4800782EF0E1F819E0B5EEC08AF1EE10FA0ADD0121C64800782EF0D6F848
:409100000021C54800782EF0D1F809E00021C14800782EF0CBF80021BF4800782EF0C6F8B0EE480ABD48007832F09EFC1AE000BFF0EE000A89EE200A9FEDB51AC8EE010A33
:4091400060EE890AB1EE001AC0EE811A70EE218ADFEDB30AB0EE680AB24800782EF020F900E000BF00BFBDEC048B10BDAE480078704710B50446AD480078A04205D0AB4813
:4091800004700C2027F086FF0DE0A948006830F048FCB0F5FA7F06D930F01BFCA44908600C2027F077FF10BD10B50446954991F830000FF0B9FE90B12046FFF7DAFF214681
:4091C0009C4800782EF072F821469B4800782EF06DF82146994800782EF068F81CE02EF08EFE50B12146934800782EF05FF82146914800782EF05AF80EE021468D48007868
:409200002EF054F821468C4800782EF04FF821468A4800782EF04AF810BD10B52EF06FFEC8B127F0E1F9DFED860AB4EEE00AF1EE10FA10D24FF47A718248006830F0CFFB17
:40924000E0B101217D4800782EF030F830F0C1FB7D49086012E02EF052FE78B140F6B8317948006830F0BBFB40B10021734800782EF01CF830F0ADFB7249086010BD6A4925
:409280000870704770B52DED048B04460D466F48007848B10120207001216D4880F8291030F097FB6A490862207830B1012845D0022857D003287ED168E0654890F82900BC
:4092C00001280ED16248016A284630F0B9FBFA2807D2012020705E4890ED090A84ED010A2BE05B4890F8350001280ED15848C16A284630F0A5FBFA2807D2022020705448FC
:4093000090ED0C0A84ED010A17E0514890F8410001280ED14E48816B284630F091FBFA2807D2032020704A4890ED0F0A84ED010A03E09FED480A84ED010A3FE0444890F85F
:40934000290030B14248016A284630F079FBFA2802D90020207004E03D4890ED090A84ED010A2BE03A4890F8350030B13848C16A284630F065FBFA2802D90020207004E075
:40938000334890ED0C0A84ED010A17E0304890F8410030B12E48816B284630F051FBFA2803D90020207005E005E0294890ED0F0A84ED010A02E00020207000BF00BF94ED42
:4093C000020A84ED030A2078B0B194ED050AB5EEC00AF1EE10FA6ED094ED010A10EE101A08463AF0B7FC41EC190BB0EE490AF0EE690A37F089F82FE086E00000EC08002023
:4094000000007A44182100206F12833A0000C8C20000C84231070020320700208F070020030058415707002038000020400000203C000020700700208807002090070020B1
:409440003D0A0F4030000020340000202D0000204008002000000000B0EE408AF0EE608A9FEDFA0B53EC102B51EC180B3AF040F93DD894ED010AB5EEC00AF1EE10FA04D133
:409480001FED0C0A84ED020A35E094ED010AD4ED050A30EE600AD4ED020AB4EEE00AF1EE10FA09DD94ED020AD4ED050A30EE200A84ED020A1FE01AE094ED010AD4ED050A75
:4094C00030EE200AD4ED020AB4EEE00AF1EE10FA08D294ED020AD4ED050A30EE600A84ED020A08E094ED010A84ED020A03E094ED010A84ED020A94ED020A84ED040A01209C
:40950000D44981F8480013E01FED2E0A84ED020A1FED300A84ED010A1FED320A84ED030A1FED340A84ED040A0020CA4981F8480094ED040AC74880ED110ABDEC048B70BDC9
:4095400070B52DED088B044603F061FFB0EE408A94ED090AD4ED0B0A30EE200AF0EE000A80EE201AF0EE418A94ED080AD4ED0A0A30EE200AF0EE000A80EE201AB0EE419A70
:4095800094ED020AB4EEE80AF1EE10FA33DD94F84400022825D1B2EE040A03F000F8E0B994ED120A38EE400AF0EE040AB4EEE00AF1EE10FA11D20FF0DAFC10B141F288309D
:4095C00001E04FF47A7005462946E06C30F007FA30B101215020015502E000215020015508E0022084F8440084ED128A30F0F1F9E06400BF5EE094ED020AB4EEC90AF1EEA1
:4096000010FA33D294F84400012825D1B2EE040A02F081FFE0B994ED120A38EE400AF8EE040AB4EEE00AF1EE10FA11DD0FF09FFC10B141F2883001E04FF47A700546294601
:40964000E06C30F0CCF930B101215020015502E000215020015508E0012084F8440084ED128A30F0B6F9E06400BF23E0002084F8440094ED120A30EE480A10EE101A084619
:409680003AF068FB41EC1B0BB0EE4B0AF0EE6B0A36F03AFFB0EE40AAF0EE60AA9FED6E0B53EC102B51EC1A0B3AF05CF902D2002150200155BDEC088B70BD70B52DED0C8B5B
:4096C00004460D4694ED0A0AF2EE040AB4EEE00AF1EE10FA0CD294ED0A0AFAEE040AB4EEE00AF1EE10FA03DD1FEDA60A84ED0A0A94ED0A0A5FEDBE0AC0EE208A95ED020A47
:40970000D5ED080AB4EEE00AF1EE10FA18D895ED0C0AD5ED020A20EE200A1FEDC31AC0EE010A94ED780A20EE800A1FEDCB1AC0EE010A95ED0D0A30EEC00A84ED620A25E008
:4097400095ED020AD5ED090AB4EEE00AF1EE10FA18DB95ED0C0AD5ED020A60EE200A1FEDD41A80EE810AD4ED780A60EE200A1FEDDC1A80EE810AD5ED0D0A30EE200A84ED05
:40978000620A03E01FEDCD0A84ED620A95ED020AB5EEC00AF1EE10FA02D11FEDE78A18E094ED620A10EE101A08463AF0D3FA41EC1B0BB0EE4B0AF0EE6B0A36F0A5FEB0EE14
:4097C00040AAF0EE60AA51EC1A0B39F087FC08EE100A94ED620A10EE101A08463AF0BAFA41EC1D0BB0EE4D0AF0EE6D0A36F08CFEB0EE40BAF0EE60BA18EE900A3AF0AAFAEB
:4098000041EC1D0BB0EE4D0AF0EE6D0A36F07CFEB0EE40CAF0EE60CA53EC1B2B51EC1C0B3AF0AEF941EC1A0B39F058FC09EE100A89EE080AB0EE409A1E210948B0EE490A1D
:409840001DF09FFEBDEC0C8B70BD0000000000000000594040080020000000000000F83F2C0800202DE9F0412DED028B04460D46F84890F8BD010A287DD14FF43270015975
:40988000001D0151001FD4F8C4120151F248007832F045F8C4F8C4024FF432700059D4F8C412081A00EE100AB8EEC00ADFEDEB0A80EE201A84EDB41A94EDB40AB2EE041A74
:4098C000C0EE010A9FEDE60A20EE800A84EDC40A95ED020AD5ED080AB4EEE00AF1EE10FA23D895ED0E0AD5ED020A20EE200A9FEDDD1AC0EE010A94ED780A20EE800A9FED87
:40990000DA1AC0EE010A95ED0F0A30EEC00A84EDDA0A94EDDA0AB5EEC00AF1EE10FA37DD9FEDD20A84EDDA0A32E095ED020AD5ED090AB4EEE00AF1EE10FA25DB95ED0E0A92
:40994000D5ED020A20EE200A9FEDC61AC0EE010A94ED780A20EE800A9FEDC31AC0EE010A95ED0F0A30EE800A84EDDA0A94EDDA0AB5EEC00A00E087E0F1EE10FA08D29FEDFF
:40998000BB0A84EDDA0A03E09FEDB80A84EDDA0AB04890F83000912809D0AE4890F83000922804D0AB4890F83000712803D132274FF0480802E032274FF04108D4EDC40A37
:4099C000B0EE600A394604F53E701DF0DAFDD4EDDA0AB0EE600A414604F554701DF0D1FD94EDD40AD4EDBE0A30EE600AF2EE040A20EE208A9FED9C0AB4EEC08AF1EE10FA6C
:409A000004DD9FED990AB0EE408A0AE09FED980AB4EEC08AF1EE10FA03D29FED950AB0EE408A012104F53970B0EE480A1DF0A9FD94EDD40A84EDDD0A94EDBE0A84EDC70AB0
:409A400004261AE0711E04F55D7000EB810090ED000A04F55D7000EB860080ED000A04F5477000EB810090ED000A04F5477000EB860080ED000A701EC6B2002EE2DC94ED1E
:409A8000B90A7C4880ED150ABDEC028BBDE8F081704991F84A10062904D06E4991F84A10122901D1012000E00020704710B52DED020B00BF042269466F48006800F55870CD
:409AC00011F0E2FC20B99DED000A624880EDD80A00BF1CBD10B52DED020B00BF042269466548006800F5577011F0CEFC20B99DED000A584880EDD70A00BF1CBD10B52DED9B
:409B0000020B00BF042269465B48006800F5567011F0BAFC20B99DED000A4E4880EDD60A00BF1CBD10B52DED020B00BF042269465148006800F5557011F0A6FC20B99DEDDE
:409B4000000A444880EDD50A00BF1CBD414991F84A10032901D1012000E00020704710B52DED020B00BF042269464348006800F55C7011F089FC20B99DED000A354880ED17
:409B8000DC0A00BF1CBD10B52DED020B00BF042269463948006800F55B7011F075FC20B99DED000A2B4880EDDB0A00BF1CBD10B52DED020B00BF042269462F48006800F56E
:409BC0005A7011F061FC20B99DED000A214880EDDA0A00BF1CBD10B52DED020B00BF042269462548006800F5597011F04DFC20B99DED000A174880EDD90A00BF1CBD15490F
:409C000091F84A10042922D0124991F84A1002291DD0104991F84A10052918D00D4991F84A100E2913D00B4991F84A1015290ED0084991F84A10132909D0064991F84A1059
:409C4000182904D0034991F84A101A2916D1012015E0000018210020540700208DED244800606A470000C84200007A440000000000007AC440080020F0030020002070473D
:409C800010B52DED028B84B00446FFF75FFF10B1B2EE048A01E0B7EE008AFE4890ED280A20EE080A84ED000AB0F8A80000EE100AB8EE400A84ED020A1FED140A84ED010A6C
:409CC000F44890F89C0084F82C00F24890F842106C3000EB810090ED000A84ED030AED4890F84210743000EB810090ED000A84ED040AE84890F842107C3000EB810090ED77
:409D0000000A84ED050AE34890F84210843000EB810090ED000A84ED060ADE4890ED700A84ED070A90ED710A84ED080A90ED720A84ED090A90ED730A84ED0A0A2DF08CFAB3
:409D4000002876D0FFF7A4FE78B30121D24800782DF0ACFA0021D14800782DF0A7FA0021CF4800782DF0A2FAB2EE040AFFF7DAFE9FEDCC0AFFF7C2FEB7EE000AFFF7AAFE81
:409D80001FED460AFFF792FE9FEDC70AFFF723FF9FEDC60AFFF70BFF9FEDC50AFFF7F3FE1FED4F0AFFF7DBFE95E0FFE7FFF727FFF0B3C048009094ED020AF0EE400A9FED87
:409DC000BE0A01231A46BD49BD48007831F0AEFA0021B14800782DF069FA0121AF4800782DF064FA0121AE4800782DF05FFA9FEDB50AFFF797FE9FEDAD0AFFF77FFE9FED8F
:409E0000AC0AFFF767FE1FED680AFFF74FFE9FEDAE0AFFF7E0FE9FEDA50AFFF7C8FE9FEDA40AFFF7B0FE1FED700AFFF798FE52E000E041E0FFF78AFE70B39E48009094ED86
:409E4000020AF0EE400A9FED9C0A01231A469B499B48007831F06AFA00218F4800782DF025FA01218D4800782DF020FA01218C4800782DF01BFA9FED930AFFF753FE9FED46
:409E80008B0AFFF73BFE9FED8A0AFFF723FE1FED8A0AFFF70BFE1EE000217F4800782DF005FA01217D4800782DF000FA01217C4800782DF0FBF90EE07E48009094ED020AD8
:409EC000F0EE400A9FED7C0A012300227F497C48007831F02BFA94F82C00B0B90020009001900290034603227949039055202DF0B4FA0020009001900290034603227549A2
:409F0000039056202DF0A9FA15E00020009001900290034603226F49039055202DF09DFA0020009001900290034603226849039056202DF092FA012004B0BDEC028B10BD32
:409F40002DED028B5421644835F081F94FF46771624835F07CF95821614835F078F95E48604908605E4848305F4908605B485F49086000F5F0705E490860A0F5DC705D49E0
:409F8000086000F5B0705C49086000F59E705B4908604C305A490860514854305949086059485A4908604C481430594908601FEDD30A143880ED030A1FEDD60A484880ED34
:409FC000130A9FED540A80ED140AFFF7BFFD40B1DFF844C100DF06460A2202212FF003FE0AE02DF039F938B1DFF82CC100DF0646012202212FF0F7FDDFF81CC100DF06466D
:40A0000002212FF01FFEDFF810C100DF064631460120DFF808C100DF0321414880F8541000BF00224FF6FF710320DFF8F8C000DF044604F001000028F3D104F002000028DE
:40A04000EFD0DFF8E4C000DF054605F0010030B121481430FFF714FE1D2027F01BF805F002000028DDD03148007818F093FA1B4880ED780AD0ED780AB0EE600A142100F574
:40A08000E4701DF07EFA2DF0CFF808B1284851E05FE00000182100206C0700208D0700208C0700206F12833A00401C45000048420000FA4330DC0020A037A04B001800400B
:40A0C0008F070020000048450080544500000140A1070020A207002098080020EC080020400800200000002004000020080000200C000020100000201400002018000020C2
:40A10000200000201C000020540C002024000020280000200000C8C2C92F04088923040860420020E9230408312304080F07002060070020007818F0EAFBFE4880ED0A0A2E
:40A14000D0ED0A0AB0EE600A1E2110301DF019FA87E02DF081F8002823D0FFF799FC08B3F548007818F0D3FBF24880ED8E0AF348007818F00FFAEF4880EDA40AD0EDA40ABE
:40A18000B0EE600A142100F51E701DF0FAF9E948D0ED8E0AB0EE600A142100F508701DF0F0F95EE0E648007818F0B1FBE14880ED0A0AD0ED0A0AB0EE600A1E2110301DF012
:40A1C000E0F9DC4890ED0A0AD0ED040A30EE600A20EE000AB0EE408A1E212030B0EE480A1DF0CFF9D748007818F091FBD14880ED200AD0ED200AB0EE600A1E2168301DF0FC
:40A20000C0F9CC4890ED200AD0ED1A0A30EE600A20EE000AB0EE408A1E217830B0EE480A1DF0AFF9C848007818F071FBC14880ED360AD0ED360AB0EE600A1E21C0301DF042
:40A24000A0F9C248007818F062FBBA4880ED4C0AD0ED4C0AB0EE600A1E2100F58C701DF090F9BB49B348FFF7FDFAB949B148FFF724FAB748FFF764F92FF0ABFB06463146E3
:40A28000B348FEF7FFFFB248007818B1B14890F84800A0BB2CF0C8FF90B19FEDAF0AAC4880ED020A0020A34908700021AB4800782CF0FCFF0021AA4800782CF0F7FF50E087
:40A2C0002CF0CAFF00284CD09FEDA30AA04880ED020A0020974908700021A14800782CF0E5FF00219D4800782CF0E0FF00219D4800782CF0DBFF0020FEF7C1FF31E0FFE7E8
:40A30000944890F8480001282BD18A48007840BB2CF08AFF68B10120864908700121904800782CF0C3FF01218C4800782CF0BEFF17E02CF091FFA0B101207E4908700121D4
:40A34000874800782CF0B2FF0121844800782CF0ADFF0121834800782CF0A8FF0120FEF78EFFFEF75AFFFEF701FF0646FEF71CFF7D4991F84A007649D1ED020AB0EE600A07
:40A38000FEF742FE4DE601B50DF0B6FA70B900BF01226946754800689C3011F075F820B99DF80000704981F89C0000BF7048016D0120DFF8C0C100DF142003F0CBF808BD91
:40A3C00010B52DED020B00249DED000AF2EE040AB4EEE00AF1EE10FA05DDB2EE040A8DED000A02240BE09DED000AB5EEC00AF1EE10FA04D29FED580A8DED000A032400BF19
:40A400000422694659480068A03011F03DF820B99DED000A544880ED280A00BF5448016D0120DFF850C100DF192003F093F820461CBD01B500BF022269464C480068A830CD
:40A4400011F022F820B9BDF800004749A1F8A80000BF4748016D0120DFF818C100DF08BD10B5FFF773FB58B144F62060FFF7E1FFB6EE000AFFF7A4FF0020FFF784FF1BE094
:40A48000FFF706FB50B12820FFF7D3FF9FED320AFFF796FF0020FFF776FF0DE0FFF7AFFB50B144F62060FFF7C4FF9FED2B0AFFF787FF0020FFF767FF2B4991F84A00FEF7C0
:40A4C000EEFA012010BD70B52DED028BB0EE408A04460D460026012C04D0022C03D0032C6DD101E000BF00BF1A4890ED140AB4EEC80AF1EE10FA05DD90ED140AB0EE408A82
:40A5000003260CE0134890ED130AB4EEC80AF1EE10FA04D290ED130AB0EE408A022610210C48DFF854C000DF012846D004EB4401084823E0EC080020580700205D07002088
:40A540006007002063070020A1070020A207002098080020400800200000000071070020720700207307002018210020F0030020604200208923040851280408143000EBAC
:40A58000810080ED018A2FF024FA04EB4402F84941F82200012104EB4402F54800EB8200017204EB4401F24800EB81004572F0481438DFF8C0C300DF00E0062601E0062639
:40A5C00000BF00BF3046BDEC028B70BDE848143890ED110A7047E84890F85000012800D170470020FCE7E248143890ED150A70470020DF49143991F84810012904D1DF4917
:40A600000978012900D10120704701B500BF01226946DB4800684A3010F036FF20B99DF80000D84981F84A0000BFFFF719FFD648016D0120DFF854C300DF272002F08AFFEA
:40A6400008BDCE4890ED780A7047CC4890ED8E0A7047CA4890ED040A7047C84890ED1A0A7047C64890ED080A7047C44890ED300A7047C24890ED460A704700B5FFF766FA46
:40A6800030B1C348007808B1012000BD0020FCE70020FAE700207047BD480078022804D1BC48007D012800D170470020FCE710B5FFF7EEF930B1B84800782DF0F9F908B150
:40A6C000012010BD0020FCE7AE4890F84A00182801D1012070470020FCE700B50121FFF7F3FF00B900E00021084600BD70B52DED068B0024FFF77CFF80B32CF0C9FD68B39B
:40A70000FFF7EBFF50B3FFF77AFA38B39D4890EDD50A10EE101A084639F01CFB41EC180BFEF76EFC10EE105A284639F013FB41EC1A0BB0EE4A0AF0EE6A0A35F0E5FEB0EEF2
:40A74000409AF0EE609A53EC182B51EC190B39F009F901D2012000E0002004462046BDEC068B70BD0020844991ED020A854991F84220743101EB8201D1ED000AB4EEE00A76
:40A78000F1EE10FA10DB7C4991ED020A7D4991F84220843101EB8201D1ED000AB4EEE00AF1EE10FA00D8012070470020724991ED020A744991F842206C3101EB8201D1EDDD
:40A7C000000AB4EEE00AF1EE10FA10D86A4991ED020A6C4991F842207C3101EB8201D1ED000AB4EEE00AF1EE10FA00DB0120704700B50023FFF7D9FF10B9FFF7B3FF00B141
:40A800000123184600BD70B52DED068B0024FFF7EFFE88B32CF03CFD70B3FFF7E9FF58B3FFF75BFF40B3FFF7EAF928B3554890EDD60A10EE101A084639F08CFA41EC180B00
:40A84000FEF7DEFB10EE105A284639F083FA41EC1A0BB0EE4A0AF0EE6A0A35F055FEB0EE409AF0EE609A53EC182B51EC190B38F03FFF02D2012001E001E000200446204660
:40A88000BDEC068B70BD70B52DED068B0024FFF7AFFE70BB2CF0FCFC58B3FFF71EFF40B3FFF7ADF928B3374890EDD70A10EE101A084639F04FFA41EC180BFEF7A1FB10EE2F
:40A8C000105A284639F046FA41EC1A0BB0EE4A0AF0EE6A0A35F018FEB0EE409AF0EE609A53EC182B51EC190B39F03CF802D2012001E001E0002004462046BDEC068B70BDC8
:40A9000070B52DED068B0024FFF779F970B3FFF76FFE58B32CF0BCFC40B3FFF7DEFE28B3184890EDD50A10EE101A084639F012FA41EC180BFFF799FE10EE105A284639F073
:40A9400009FA41EC1A0BB0EE4A0AF0EE6A0A35F0DBFDB0EE409AF0EE609A53EC182B51EC190B38F0FFFF19D2012018E018E00000540800206D27040898080020EC080020FC
:40A98000F00300201821002060420020892304082C000020E82B002094070020002004462046BDEC068B70BD70B52DED068B0024FFF725F988B3FFF71BFE70B3FFF7F5FEE2
:40A9C00058B32CF065FC40B3FFF787FE28B3F74890EDD60A10EE101A084639F0BBF941EC180BFFF742FE10EE105A284639F0B2F941EC1A0BB0EE4A0AF0EE6A0A35F084FD2B
:40AA0000B0EE409AF0EE609A53EC182B51EC190B38F06EFE02D2012001E001E0002004462046BDEC068B70BD70B52DED068B0024FFF7E5F880B3FFF7DBFD68BB2CF028FC36
:40AA400050B3FFF74AFE38B3D84890EDD70A10EE101A084639F07EF941EC180BFFF705FE10EE105A284639F075F941EC1A0BB0EE4A0AF0EE6A0A35F047FDB0EE409AF0EE0B
:40AA8000609A53EC182B51EC190B38F06BFF01D2012000E0002004462046BDEC068B70BD70B52DED068B0024FFF7A9F880B3FFF79FFD68B32CF0ECFB50B3FFF70EFE38B3BE
:40AAC000BA4890EDD50A10EE101A084639F042F941EC180BFFF7CDFD10EE105A284639F039F941EC1A0BB0EE4A0AF0EE6A0A35F00BFDB0EE409AF0EE609A53EC182B51EC0B
:40AB0000190B38F02FFF01D2012000E0002004462046BDEC068B70BD70B52DED068B0024FFF76DF888B3FFF763FD70B3FFF71AFE58B32CF0ADFB40B3FFF7CFFD28B39B483D
:40AB400090EDD60A10EE101A084639F003F941EC180BFFF78EFD10EE105A284639F0FAF841EC1A0BB0EE4A0AF0EE6A0A35F0CCFCB0EE409AF0EE609A53EC182B51EC190B65
:40AB800038F0B6FD02D2012001E001E0002004462046BDEC068B70BD70B52DED068B0024FFF72DF880B3FFF723FD68BB2CF070FB50B3FFF792FD38B37C4890EDD70A10EE37
:40ABC000101A084639F0C6F841EC180BFFF751FD10EE105A284639F0BDF841EC1A0BB0EE4A0AF0EE6A0A35F08FFCB0EE409AF0EE609A53EC182B51EC190B38F0B3FE01D289
:40AC0000012000E0002004462046BDEC068B70BD70B52DED088B0024FEF7F1FFB8B32CF037FBA0B3FFF759FD88B3FFF71EFDF0EE400AFFF71EFD30EE800AB0EE408A5B4871
:40AC400090EDD80A10EE101A084639F083F841EC190BFFF7FEFC30EE480A10EE105A284639F078F841EC1B0BB0EE4B0AF0EE6B0A35F04AFCB0EE40AAF0EE60AA53EC192B44
:40AC800051EC1A0B38F06EFE02D2012001E002E00020044600BF2046BDEC088B70BD444890ED030A704710B50124404890F84A000E281BD03D4890F84A00022816D03B48D2
:40ACC00090F84A00152811D0384890F84A001A280CD0364890F84A00032802D12CF0BCFA20B9324890F84A00182800D100240CB1012010BD0020FCE710B50024FFF778FC79
:40AD0000B0B12CF0C5FA98B1FFF7CDFF80B1FFF7E4FC68B1FFF7C3FF2448D0EDD90AB4EEE00AF1EE10FA01DD012000E000200446204610BD10B50024FFF75AFCB0B12CF045
:40AD4000A7FA98B1FFF7AFFF80B1FFF7A8FF1748D0EDDA0AB4EEE00AF1EE10FA04D2FFF7BCFC08B1012000E000200446204610BD10B50024FFF73CFCB0B92CF089FA98B1BF
:40AD8000FFF791FF80B1FFF78AFF0848D0EDDB0AB4EEE00AF1EE10FA04DDFFF79EFC08B1012000E000200446204610BD18210020880C00209B4890ED030A704710B5002414
:40ADC000FFF716FCB0B12CF063FA98B1FFF76BFF80B1FFF782FC68B1FFF7ECFF9248D0EDD90AB4EEE00AF1EE10FA01DD012000E000200446204610BD10B50024FFF7F8FBEC
:40AE0000B0B12CF045FA98B1FFF74DFF80B1FFF764FC68B1FFF7CEFF8348D0EDDA0AB4EEE00AF1EE10FA01D2012000E000200446204610BD10B50024FFF7DAFBB0B92CF0DD
:40AE400027FA98B1FFF72FFF80B1FFF746FC68B1FFF7B0FF7448D0EDDB0AB4EEE00AF1EE10FA01DD012000E000200446204610BD70B52DED068B00242CF00AFA88B3FFF789
:40AE800012FF70B3FFF729FC58B3674890EDDC0A10EE101A084638F05DFF41EC180BFFF7FEFEF0EE400AFFF785FF30EEC00A10EE105A284638F04EFF41EC1A0BB0EE4A0AD1
:40AEC000F0EE6A0A35F020FBB0EE409AF0EE609A53EC182B51EC190B38F044FD02D2012001E001E0002004462046BDEC068B70BD10B52DED028B9FED4D0AB0EE408A2CF063
:40AF000093F928B14A4890ED030AB0EE408A11E02CF0A2F970B1FFF7C2FEB0EE408AB3EE040AB4EEC08AF1EE10FA03D89FED3F0AB0EE408AB0EE480ABDEC028B10BD3D482D
:40AF400090EDA40A704710B52DED068BFEF7A0FD20B1FFF7A4FEB0EE408A0CE0324890F84A00032803D1344890ED038A03E0FFF770FBB0EE408A18EE100A38F0EBFE41EC55
:40AF80001A0BB0EE4A0AF0EE6A0A35F0BDFAB0EE409AF0EE609A9FED290B53EC102B51EC190B38F0A5FB03D89FED200AB0EE408AB0EE480ABDEC068B10BD00B50022FFF7DC
:40AFC00017FB90B1FEF764FD78B1FFF7B8FFF0EE400AFFF736FB9FED1B1A20EE010AF4EEC00AF1EE10FA00DD0122104600BD00B50022FFF7FDFA90B1FEF74AFD78B1FFF7A1
:40B000009EFFF0EE400AFFF71CFB9FED0F1A20EE010AF4EEC00AF1EE10FA00D20122104600BD0000E00C00201821002000000000380D0020EC080020900D00200000000038
:40B04000000034406666663FCDCCCC3D10B501F008FF292002F07EFA2A2002F07BFA0EF051F870B1DFF8E4C300DF044604212EF0E9FDDFF8D8C300DF044602212EF0E2FD35
:40B080000DE0DFF8C8C300DF044604212EF0F7FDDFF8B8C300DF044602212EF0F0FD10BD10B5EB48C16B01202EF006FEE848C16B0120DFF8A0C300DF10BD10B52DED0C8B2B
:40B0C000B0EE408AE44890ED630AB0EE409AB4EEC98AF1EE10FA02DD01F0ADFE38B9B4EEC98AF1EE10FA2CD201F0A5FE48BBDA4890ED6A0A10EE101A084638F02BFE41EC96
:40B100001B0B38EE490A10EE101A084638F022FE41EC1D0BB0EE4D0AF0EE6D0A35F0F4F9B0EE40CAF0EE60CA53EC1B2B51EC1C0B38F01AFB41EC1A0B37F0D0FF08EE900A53
:40B140003BE0B4EEC98AF1EE10FA02DD01F073FE38B1B4EEC98AF1EE10FA2CD201F06BFE48B3BD4890ED6B0A10EE101A084638F0F1FD41EC1B0B38EE490A10EE101A0846B6
:40B1800038F0E8FD41EC1D0BB0EE4D0AF0EE6D0A35F0BAF9B0EE40CAF0EE60CA53EC1B2B51EC1C0B38F0E0FA41EC1A0B37F096FF08EE900A01E0DFEDA98A9FEDA90AF4EED1
:40B1C000C08AF1EE10FA03DD9FEDA50AF0EE408A9FEDA40AF4EEC08AF1EE10FA03D29FEDA10AF0EE408AB0EE680ABDEC0C8B10BD10B52DED028B2EF0ECFB9B49086000205C
:40B2000001F076F9B0EE408AFFF757FF964880ED030A01F03FFBBDEC028B10BD2821924834F015F801218A4880F82012DFF81CC200DF0646012204212EF0D5FCDFF80CC2C6
:40B2400000DF0646192202212EF0CDFCDFF8FCC100DF064631460120DFF8F8C100DF03217B4880F8201200BF00224FF6FF710720DFF8F8C100DF85B2012DF5D0022DF3D1BE
:40B28000DFF8ECC100DF044604F0040008B101F0DDFB04F0020018B1FFF7AAFFFFF700FF04F001000028DFD0FFF7D0FEDCE710B504466748D0F81C122046DFF898C100DF98
:40B2C00010BD10B52DED088B634890ED630AD0ED610A30EE600ADFED630A80EE801A11EE104A204638F036FD41EC1B0BB0EE4B0AF0EE6B0A35F008F9B0EE40AAF0EE60AA40
:40B3000051EC1A0B37F0DEFE41EC190B37F0E6FE08EE900A504890ED620AD0ED630A30EE600ADFED4F0A80EE801A11EE104A204638F010FD41EC1A0BB0EE4A0AF0EE6A0AD2
:40B3400035F0E2F8B0EE409AF0EE609A51EC190B37F0C4FE08EE100A002001F06AFA3E4890F83000912809D03B4890F83000922804D0394890F8300071280CD1364890F861
:40B38000B201032807D19FED3B0AB0EE408AB1EE480AF0EE408AB0EE680A01F0C2FAB0EE480A01F0D2FABDEC088B10BD70B505460C4601F0F9F9284600F022FE204600F019
:40B3C00037FEFFF77EFF64201BF0C1FA0120FFF76EFF70BD2448D0ED030AB0EE600A7047214890F82400042801D0012070470020FCE70220704710B52DED088BB0EE408A15
:40B4000018EE100A38F0A6FC41EC190BFFF7E2FF10EE104A204638F09DFC41EC1B0BB0EE4B0AF0EE6B0A35F06FF8B0EE40AAF0EE60AA53EC192B51EC1A0B38F059F903D2B2
:40B440000120BDEC088B10BD0020FAE7C92F0408604200208923040818210020000000000000C8420000C8C2C81C0020E923040831230408D051863910B501F0F2FC2920ED
:40B4800002F068F82A2002F065F80DF074FE70B1DFF828C400DF044604212EF0D3FBDFF81CC400DF044602212EF0CCFB0DE0DFF80CC400DF044604212EF0E1FBDFF8FCC3BA
:40B4C00000DF044602212EF0DAFB10BD10B5FC48C16B01202EF0F0FBF948C16B0120DFF8E4C300DF10BDF0EE400AF748D0ED631AB0EE611AD0ED611AF4EEC11AF1EE10FA91
:40B500001FD2F4EEC10AF1EE10FA08D2D0ED671A90ED6A2AB0EE610A02EE200A31E0F4EEC10AF1EE10FA09DBE748D0ED691A90ED6B2AB0EE610A02EE200A22E09FEDE30A8E
:40B540001FE0F4EEC10AF1EE10FA09D2DE48D0ED691A90ED6B2AB0EE610A02EE200A10E0F4EEC10AF1EE10FA09DBD748D0ED671A90ED6A2AB0EE610A02EE200A01E09FED58
:40B58000D30A7047D048B0F9A0037047CE48B0F9A2037047CE49097D31B1012906D0022906D0032906D106E0002006E0012004E0022002E000BF032000BF00BF704710B56D
:40B5C0002DED028BFFF7E6FF10B9FFF7DFFF01E0FFF7D8FF08EE100A2EF0FBF9BD490860002000F085FFF0EE408AFFF77CFFB94880ED030A90ED030AF8EEC80A30EE600AFC
:40B6000080ED030A01F046F9BDEC028B10BD2C21B04833F01CFE0121A94880F83412DFF89CC200DF0646012204212EF0DCFADFF88CC200DF0646192202212EF0D4FADFF8FD
:40B640007CC200DF064631460120DFF878C200DF03219B4880F8341200BF00224FF6FF710720DFF874C200DF85B2012DF5D0022DF3D1DFF868C200DF044604F0040008B173
:40B6800001F0E4F904F0020018B1FFF798FFFFF71DFF04F001000028DFD0FFF7EDFEDCE710B504468648D0F830122046DFF814C200DF10BD8448B0F8900370478248B0F818
:40B6C0008E0370478048B0F88C03704710B52DED048BFFF7EFFF0146FFF7F4FF081A00EE100AB8EEC00A7848D0ED630A90ED611A70EEC10A80EE201AB0EE418AFFF7DEFF41
:40B700000146FFF7D7FF081A00EE100AB8EEC00A6D48D0ED620A90ED631A70EEC10A80EE201AF0EE418AFFF7C5FF00EE100AB8EE400A6548D0ED630A08EE600AB0EE409AA9
:40B74000FFF7B8FF00EE100AB8EE400A5E48D0ED630A08EEE00AF0EE409A002001F069F8B0EE480A01F0DDF8B0EE680A01F0EDF8B0EE490A01F0FDF8B0EE690A01F00DF9CF
:40B78000BDEC048B10BD70B505460C4601F00CF8284600F035FC204600F04AFCFFF796FF0120FFF77DFF70BD4A48D0ED030AB0EE600A7047474890F82400042801D00120E3
:40B7C00070470020FCE70220704773B50D46002400BF022269464248006800F563700FF053FE20B9BDF800003749A1F88C0300BF5C2001F0AFFE20467CBD73B50D4600242E
:40B8000000BF022269463648006800F28E300FF03BFE20B9BDF800002B49A1F88E0300BF5D2001F097FE20467CBD31B5002400BF022269462A48006800F564700FF024FEBB
:40B8400020B9BDF800002049A1F8900300BF5E2001F080FE204638BD31B5002400BF022269461F48006800F292300FF00DFE20B9BDF800001449A1F8920300BF622001F02A
:40B8800069FE204638BD1048B0F89203704731B5002400BF022269461148006800F565700FF0F2FD20B9BDF800000749A1F8940300BF682001F04EFE204638BDC92F040874
:40B8C00060420020892304081821002000000000302C0020202A0020E923040831230408F00300205648B0F89403704731B5002400BF012269465348006800F567700FF007
:40B90000C3FD20B9BDF800004D4981F89C0300BF692001F01FFE204638BD494890F89C03704731B5002400BF012269464548006800F29E300FF0A8FD20B9BDF800004049E0
:40B9400081F89E0300BF632001F004FE204638BD3B4890F89E03704731B5002400BF022269463848006800F568700FF08DFD20B9BDF900003249A1F8A00300BF6D2001F05D
:40B98000E9FD204638BD31B5002400BF022269462C48006800F2A2300FF076FD20B9BDF900002749A1F8A20300BF6C2001F0D2FD204638BD10B52DED0C8BB0EE408AFFF721
:40B9C00079FE044637F080FE41EC1A0BFFF772FE00EE100AB8EE401AFFF7E6FE31EE400A10EE104A204638F0B5F941EC1D0BB0EE4D0AF0EE6D0A34F087FDB0EE40CAF0EE7D
:40BA000060CA9FED110B53EC102B51EC1C0B37F0ABFE41EC1B0B53EC1A2B37F04DFC41EC190B37F05BFB08EE900AF4EEC88AF1EE10FA03D20120BDEC0C8B10BD0020FAE7C0
:40BA400018210020F0030020000000000000594010B52DED028BB0EE408AB44880ED008A2DF0B7FFB2490860BDEC028B10BD10B52DED088BB0EE408A9FEDAE0AF0EE408AFB
:40BA8000B3EE040AB0EE40BA18EE100A38F062F941EC1A0BB0EE4A0AF0EE6A0A34F034FDB0EE409AF0EE609A9FEDA30B53EC102B51EC190B37F056FF0ED2B3EE040A38EE1B
:40BAC000400ADFED9F0A80EE201AB3EE040A21EE000AF0EE408A03E09FED960AF0EE408AB0EE680ABDEC088B10BD10B52DED048B04469FED900AB0EE408A9FED8E0AF0EE57
:40BB0000408A904890F83000922804D08D4890F83000932874D18B4890F8FF01022804D0884890F8FF01032806D1814800682DF078FFB0F57A7F03D300208349087001E05F
:40BB400081480470814800682DF06BFFC82857D37C4890F830001D2849D17B48007828B1724890ED000AB0EE408A15E0784800782BF062FD00EE100AB8EE400ADFED750A34
:40BB800070EE600A9FED741A80EE810AF2EE0E0A20EE200AB0EE408A704890ED000A78EE400A6F4890ED000A9FED6E1A01EE200A80ED000A062025F06DFA44B114F09DFA0F
:40BBC000B0EE409AFFF753FFF0EE408A03E001F097FCF0EE408A644890ED000A30EE280A624880ED000A052025F054FA2CE05648007830B14D4890ED000AB0EE408A16E025
:40BC000036E0534800782BF017FD00EE100AB8EE400AF3EE040A30EE600ADFED4F0A80EE201AB2EE0E0A21EE000AB0EE408A4B4890ED000A78EE400A90ED000A9FED491AF7
:40BC400001EE200A80ED000A2DF0C3FE3F4908603C4890F8FF01022804D03A4890F8FF01032802D1042025F015FA072025F012FABDEC048B10BD394890ED000A704701B54A
:40BC800000BF012269463A48006800F2FF100FF0FBFB20B99DF800002A4981F8FF0100BF08BD224890ED000A70472D4890ED000A70472E4890ED000A70472B4890ED000A2C
:40BCC0007047F0B50546059C0E78022E02D0042E28D113E08F78487867F31F2000EE100AB8EE400ADFED230A30EE600ADFED220A80EE201A1C4E86ED001A14E08F7848782B
:40BD000067F31F2000EE100AB8EE400ADFED190A30EE600ADFED180A80EE201A0F4E86ED001A00E000BF00BFF0BD000000040020180400200000000000000000000034409C
:40BD40000000A04218210020140400201C0400205507002000004842000080450C040020040400209A99993E1004002008040020F00300200000FB4600007A44002383804B
:40BD8000C38002810160704701460022C8888B88984201D10A890EE0C8888B88984206DA8888CB88C01A0B89181A82B203E0C8888B88C01A82B2501E80B270470146C88816
:40BDC0008A88904201D1012070470020FCE782880A448280828803899A4203DB82880389D21A82807047C2880A44C280C28803899A4203DBC2880389D21AC28070470A4658
:40BE0000C3889B1A19B2002903DA03890B44C38000E0C180704788B0016807914168069181680591C1680491016903914169029181690191C169009108B0704700000000A4
:40BE40000000000000000000000000000000000000000000000000000000000000000000000000000000000000000000526176656E20496E647573747269657320496E6342
:40BE80000000000000000000000000004175672D31382D32303138000000000032322E312E302E3131000000000000005374656572696E6720436F6E74726F6C20556E6998
:40BEC0007400000000000000000000003037373031373135323100000000000000000000000000000000000000000000FFFFFFFFFFFFFFFFFFFFFFFFFFFFFFFFFFFFFFFFE3
:40BF0000FFFFFFFFFFFFFFFFFFFFFFFFFFFFFFFFFFFFFFFFFFFFFFFFFFFFFFFFFFFFFFFFFFFFFFFFFFFFFFFFFFFFFFFFFFFFFFFFFFFFFFFFFFFFFFFFFFFFFFFFFFFFFFFF41
:40BF4000FFFFFFFFFFFFFFFFFFFFFFFFFFFFFFFFFFFFFFFFFFFFFFFFFFFFFFFFFFFFFFFFFFFFFFFFFFFFFFFFFFFFFFFFFFFFFFFFFFFFFFFFFFFFFFFFFFFFFFFFFFFFFFFF01
:40BF8000FFFFFFFFFFFFFFFFFFFFFFFFFFFFFFFFFFFFFFFFFFFFFFFFFFFFFFFFFFFFFFFFFFFFFFFFFFFFFFFFFFFFFFFFFFFFFFFFFFFFFFFFFFFFFFFFFFFFFFFFFFFFFFFFC1
:40BFC000FFFFFFFFFFFFFFFFFFFFFFFFFFFFFFFFFFFFFFFFFFFFFFFFFFFFFFFFFFFFFFFFFFFFFFFFFFFFFFFFFFFFFFFF00C00008FFFF030800800008FBBF000808B425B2BF
:40C0000001B500BF01226946FE48006800F5D9700FF03AFA20B99DF80000FB4981F8B20100BF02201AF0C1FA0120FFF740F908BD01B500BF01226946F248006800F2B31063
:40C040000FF022FA20B99DF80000EF4981F8B30100BF02201AF0A9FA0120FFF728F908BD70B52DED068BB0EE408AF0EE608A04460425E54890F8B201E4490978884206D11D
:40C08000E14890F8B301E249097888427ED0DE4890F8B2010C287CD2DFE800F05D213E06595A5B5C073C3D5E00BF9FEDDA0ADA4880ED000A9FEDD70AD84880ED000A9FED5B
:40C0C000D50AD74880ED000A9FEDD20AD54880ED000A0120D4490870D449087059E0B6EE000ACD4880ED000A9FEDD10ACB4880ED000A9FEDC80ACA4880ED000A9FEDC50ADE
:40C10000C84880ED000A0120C74908700020C74908703EE000BF00BF9FEDC60ABE4880ED000A9FEDC50ABD4880ED000A9FEDB90ABB4880ED000A9FEDB70ABA4880ED000A4C
:40C140000120B94908700020B849087021E000BF00BF00BF00BF00BF9FEDAE0AAE4880ED000A9FEDAC0AAD4880ED000A9FEDA90AAB4880ED000A9FEDA70AAA4880ED000A21
:40C180000120A94908700020A84900E002E0087000BF00BFA448007808B900254CE0A3480078012804D1FEF768FA50B3002543E03CB99A4890ED000AB4EEC08AF1EE10FA7F
:40C1C00009DC012C09D1974890ED000AB4EEC08AF1EE10FA01DD01252EE03CB98E4890ED000AB4EEC08AF1EE10FA09D3012C09D18B4890ED000AB4EEC08AF1EE10FA01D2FA
:40C20000002519E018EE900A37F0A4FD41EC1A0BB0EE4A0AF0EE6A0A34F076F9B0EE409AF0EE609A9FED850B53EC102B51EC190B37F098FB00D203252846BDEC068B70BD7F
:40C2400031B52DED020B044600BF042269466D48006800F5C2700FF017F920B99DED000A694880ED610A00BF0CF04CFF10B1FFF728F808E00CF07FFF10B1FFF727FA02E091
:40C2800001201AF08BFA212024F004FF01203EBD31B52DED020B2DED088B044694B300209FED680A19F040F810EE105A284637F051FD41EC1B0BB0EE4B0AF0EE6B0A34F0A8
:40C2C00023F9B0EE40AAF0EE60AA51EC1A0B36F005FF08EE100A4C4890EDE20A30EE480AF0EE408A90EDE20A30EE080AB0EE409A9DED080AB4EEC90AF1EE10FA03DD8DED9C
:40C30000089A09E009E09DED080AB4EEE80AF1EE10FA01D2CDED088A0FE000BF042208A93848006800F562700FF0AEF820B99DED080A354880EDE20A00BF00BF042208A9D8
:40C340003048006800F5C6700FF09EF820B99DED080A2D4880ED630A00BF0CF0D3FE10B1FEF7AFFF08E00CF006FF10B1FFF7AEF902E002201AF012FA212024F08BFE012009
:40C38000BDEC088B3EBD31B52DED020B044600BF042269461B48006800F5C4700FF074F820B99DED000A184880ED620A00BF0CF0A9FE10B1FEF785FF08E00CF0DCFE10B13B
:40C3C000FFF784F902E003201AF0E8F9212024F061FE01203EBD014600200B2955D2DFE801F054494A06474854543B4546009FED161AC0EE010A9FED151A70EE810AFCEEA3
:40C40000E00A25E0F0030020182100205800002059000020000000005C0000206000002064000020680000206C0000206D00002066664640CDCCCC3C33339F400000000057
:40C4400000406F4035FA0E3D0000AF4300401C4510EE902A90B21AE05FED040A70EE200AFCEEE00A10EE902A90B210E000BF00BF00BF00BF00BFDFEDFC0A60EE200AFCEE3D
:40C48000E00A10EE902A90B201E0002000BF00BF7047014600200B2926D2DFE801F0251A1B0618192525101617005FED190A80EE201AFDEEC10A10EE902A10B216E0FCEED8
:40C4C000C00A10EE902A10B210E000BF00BF00BF00BF00BFDFEDE40A60EE200AFDEEE00A10EE902A10B201E0002000BF00BF70475FED380AB0EE600A28B9DC49D1ED560ADC
:40C50000B0EE600A06E0012804D1D849D1ED990AB0EE600A704770B52DED0A8BB0EE408A9FEDD30AC8EE000A10EE905AD14890ED610AF0EE408A90ED630AB0EE409A002056
:40C54000FFF7D6FFF0EE409A284637F003FC41EC1A0B38EEE90A78EEC90A80EE201A11EE106A304637F0F6FB41EC1C0BB0EE4C0AF0EE6C0A33F0C8FFB0EE40BAF0EE60BA3B
:40C5800053EC1A2B51EC1B0B37F0B2F801D2012000E0002004462046BDEC0A8B70BD70B52DED0A8BB0EE408A9FEDB10AC8EE000A10EE905AAF4890ED620AF0EE408A90ED84
:40C5C000630AB0EE409A0020FFF792FFF0EE409A284637F0BFFB41EC1A0B38EEE90A78EEC90A80EE201A11EE106A304637F0B2FB41EC1C0BB0EE4C0AF0EE6C0A33F084FF57
:40C60000B0EE40BAF0EE60BA53EC1A2B51EC1B0B37F06EF801D2012000E0002004462046BDEC0A8B70BD70B52DED0C8BF0EE408A9FED8F0AC8EE800A10EE904A8D4890EDDA
:40C64000620AF0EE409A90ED610AB0EE40AA90ED630AB0EE408A0020FFF74AFFB0EE409A204637F077FB41EC1B0B39EE480A7AEE480A80EE201A11EE106A304637F06AFB55
:40C6800041EC1D0BB0EE4D0AF0EE6D0A33F03CFFB0EE40CAF0EE60CA53EC1B2B51EC1C0B37F026F824D2204637F054FB41EC1B0B39EE480A79EEC80A80EE201A11EE106AA7
:40C6C000304637F047FB41EC1D0BB0EE4D0AF0EE6D0A33F019FFB0EE40CAF0EE60CA53EC1B2B51EC1C0B37F003F801D2012000E0002005462846BDEC0C8B70BD5B4890F881
:40C700005000042801D0012070470020FCE710B50124FFF7F3FF28B95449C86A64212DF05EF900B10024204610BD504890F82800042801D0012070470020FCE710B5012444
:40C74000FFF7F3FF28B94949486864212DF047F900B10024204610BD10B5FFF7EFFF10B1FFF7D5FF08B9022411E0424890ED6A0AB5EEC00AF1EE10FA08D090ED6B0AB5EE7A
:40C78000C00AF1EE10FA01D0012400E00024204610BD18B9354991ED080A04E0012802D1324991ED120A704710B50021324800782FF048F90021314800782FF043F92D48F4
:40C7C00090F8B201032802D0082820D10FE000209FED2B0AFFF734FD00201FEDF20AFFF757FD00209FED270AFFF7CDFD1FE000209FED250AFFF724FD00201FEDFA0AFFF7C3
:40C8000047FD00209FED210AFFF7BDFD0FE00020B6EE000AFFF714FD0020B0EE040AFFF737FD0020B1EE020AFFF7ADFD00BF00BF10BD01B50F4890F8410001280FD000BF20
:40C84000012269461248006800F2B5100EF01CFE20B99DF80000074981F8B50100BF212024F018FC08BD000000007A44E80D00200000C84218210020540700205307002050
:40C8800090ED24C990ED244900803BC500803B45F003002010B52DED028B044694ED030AD4ED040A30EE600A84ED060A94ED030A84ED040A2DF08DF82060D4E90001401A2E
:40C8C000A06094ED020AB8EE400A5FED190A80EE201AB0EE418A20686060B5EEC08AF1EE10FA1BDD94ED060AC0EE080AC4ED050A0CF03DFB48B1D4ED050AB0EE600AC82126
:40C9000004F11C001AF03DFE08E0D4ED050AB0EE600A042104F11C001AF033FEBDEC028B10BD10B52DED020B00BF04226946FA48006800F5D4700EF0A7FD20B99DED000AFB
:40C94000F64880ED6A0A00BF1CBD10B52DED020B00BF04226946F048006800F5D6700EF093FD20B99DED000AEC4880ED6B0A00BF1CBD10B52DED020B00BF04226946E6484E
:40C98000006800F5CE700EF07FFD20B99DED000AE24880ED670A00BF1CBD10B52DED020B00BF04226946DC48006800F5D2700EF06BFD20B99DED000AD84880ED690A00BF80
:40C9C0001CBD19B9D64A82F8280004E0012902D1D34A82F85000704710B52DED088BB0EE408A9FEDD00AF0EE408AB3EE040AB0EE40BA18EE100A37F0ADF941EC1A0BB0EE3F
:40CA00004A0AF0EE6A0A33F07FFDB0EE409AF0EE609A9FEDC50B53EC102B51EC190B36F0A1FF0AD21FED6E0AC8EE000A9FEDC00A20EE800AF0EE408A03E09FEDBA0AF0EE9D
:40CA4000408AB0EE680ABDEC088B10BD10B52DED028BB34890F86D02012816D0AF4890F84B00AF4981F86C02084690F86C1254301AF076FDAA4890F86C1200F5B0701AF051
:40CA80006FFD0120A64981F86D02A44890F8B2010B287DD2DFE800F0FE06162AFDFCFBFA2B3BB400A34800782AF0C6FD00EE100AB8EE400ADFEDA00A20EE200A984880ED33
:40CAC000040A03E19B4800782AF0B6FD00EE100AB8EE400ADFED980A20EE200ADFED970A80EE201A8E4880ED041AEFE000BF914800782EF014FF00EE100AB8EEC00A8848B0
:40CB0000D0ED000A30EE200A80ED040ADEE00AF0F3FE10B90AF0A5FD18B3FDF757FDB0EE408AFFF759FF864880ED000A854800682CF077FF00EE100AB8EE400A5FEDB60A84
:40CB400080EE201A804880ED001A7D4890ED000A7D48D0ED000A20EE200A7C4880ED000A20E0744800782EF0DAFE00EE100AB8EEC00A7748D0ED000A30EE600A5FEDC60AA7
:40CB800080EE201A714880ED001A6A48007800E094E02EF0C4FE00EE100AB8EEC00A6C4880ED000A2CF015FF664908605C4890ED040A6648D0ED000A30EE200AF6EE000A6B
:40CBC000B4EEE00AF1EE10FA19DD554890ED040A5E48D0ED000A30EE200AF1EE020AB4EEE00AF1EE10FA0AD24D4890ED040A5748D0ED000A30EE200A494880ED040A65E092
:40CC0000FFF75BF8B2EE041AC0EE010AB0EE040A30EE800A424880ED040A464800782EF07EFE00EE100AB8EEC00A4948D0ED000A30EE600A5FEDF40A80EE201A404880EDFC
:40CC4000001A3C4800782EF06AFE00EE100AB8EEC00A3F4880ED000A3A4800682CF0E1FE00EE100AB8EE400ADFED3A0A80EE201A354880ED001A324890ED000A3248D0EDD1
:40CC8000000A20EE200AF1EE040A04E018E00FE008E006E013E020EE200A2F4880ED000A14E000BF9FED1F0A1D4880ED040A0DE09FED1C0A1A4880ED040A07E000BF00BF6A
:40CCC0009FED180A164880ED040A00BF00BF144890F86C12D0ED040AB0EE600A54301AF0EBFB0F48001DFFF7D5FD0D4890ED081AF0EE410A90ED041AB0EE410A0020FFF793
:40CD0000AFF904460021FFF75CFE044890F8B3010B2866D222E00000F003002018210020E80D0020000000000000000000003440713DAA3F540700203333533A0CAC233F87
:40CD400070000020800000207C000020780000207400002000007A4454000020DFE800F0420616312A2B3B3532333400FE4800782AF062FC00EE100AB8EE400A5FED120A4F
:40CD800020EE200AF94880ED0E0A31E0F64800782AF052FC00EE100AB8EE400A5FED1A0A20EE200A5FED1B0A80EE201AEF4880ED0E1A1DE000BF1FED250AEC4880ED0E0A11
:40CDC00016E000BF00BF00BF00BF1FED2A0AE74880ED0E0A0CE01FED2D0AE44880ED0E0A06E000BF1FED310AE04880ED0E0A00BF00BFDE4890F86C12D0ED0E0AB0EE600A4D
:40CE000000F5B0701AF058FBD8482C30FFF742FDD64890ED121AF0EE410A90ED0E1AB0EE410A0120FFF71CF904460121FFF7C9FDBDEC028B10BDCE4890ED610AD0ED630AD2
:40CE400030EE600AB5EEC00AF1EE10FA01DD012070470020FCE7B0EE040AC44880ED040A704730B589B02AF00AFA40B10021084619F081FC0121002019F07DFC2AE0BC483D
:40CE800090F8B201032804D0B94890F8B201082808D10021032019F06EFC0121032019F06AFC17E0B24890F8B20109280AD10021032019F060FC0121032019F05CFCFFF70B
:40CEC000CAFF07E00021032019F055FC0121002019F051FCA64890F8B25190F8B3410B2D7ED2DFE805F08C06182A8E8F608D2B2C2D000020009001900290034603229D498A
:40CF00000390084600782AF0A8FA0321994800782AF051FE88E000200090019002900346032294490390084600782AF096FA0021904800782AF03FFE76E000BF00BF00BF12
:40CF400000200090019002900346022289490390084600782AF081FA0221864800782AF02AFE2AF061F968B183485FED920A9FED830A04230022824900907E4800782EF0AD
:40CF8000D5F90FE02AF068F960B17B485FED9B0A9FED7A0A0423002219070090754800782EF0C4F940E000200090019002900346022270490390084600782AF04EFA062160
:40CFC0006C4800782AF0F7FD002000900190022314220121029004A82EF0C0FA04A800E00DE05FEDB00A9FED670A032300224FF0804100905F4800782EF098F914E000BF4E
:40D0000000BF00BF00200090019002900346032258490390084600782AF01FFA0121554800782AF0C8FD00BF00BF0B2C7ED2DFE804F08B06182A8D8E608C2B2C2D000020B0
:40D040000090019002900346032247490390084600782AF002FA0321434800782AF0ABFD9AE00020009001900290034603223E490390084600782AF0F0F900213A480078EE
:40D080002AF099FD88E000BF00BF00BF00200090019002900346022233490390084600782AF0DBF90221304800782AF084FD2AF0BBF868B130485FEDE50A9FED300A0423E4
:40D0C00001222F490090284800782EF02FF90FE02AF0C2F860B128485FEDEE0A9FED270A04230122910700901F4800782EF01EF952E00020009001900290034602221A4937
:40D100000390084600782AF0A8F90621164800782AF051FD002000900190034614220121029004A82EF01AFA04A800E00CE0DFED160A9FED120A02230122910700900A4856
:40D1400000782EF0F3F827E000BF00BF00BF00200090019002900346032203490390084600782AF07AF911E053070020E80D0020182100205407002030DC0020809FD54AB9
:40D1800000040140A037A04C000000000121DE4800782AF010FD00BF00BF09B030BD10B5DA4988684FF496712CF019FC10BDD84890ED000A704710B52DED048B19F08EFADF
:40D1C00010EE104A204636F0C5FD41EC190BB0EE490AF0EE690A33F097F9B0EE408AF0EE608A9FEDCC0B53EC102B51EC180B36F07FFA03D20120BDEC048B10BD0020FAE73B
:40D20000C64991F84110012901D1012007E0C34991F8B51109B1012100E000210846704710B52DED068BB0EE408ABD48007838B91FED2B0ABB4880ED000A0120B849087029
:40D24000FFF7DEFF002879D0FFF7B5FF18B90AF053FB002872D0FFF7AAFF10EE104A204636F078FD41EC1A0BB0EE4A0AF0EE6A0A33F04AF9B0EE409AF0EE609A9FEDAA0BB8
:40D2800053EC102B51EC190B36F032FA56D2FFF786FF002852D123F0ABF9DFEDA50AB4EEE00AF1EE10FA49DBFFF756FA012845D19A4890F83000912840D0984890F8300008
:40D2C00092283BD0954890F83000712836D0934890F8B2010B282AD2DFE800F029121306141529290708160000BF00BF8D4890ED000ADFED900A08EE200A80ED000A1CE072
:40D3000000BF00BF00BF00BF8448D0ED630A9FED891A48EE410AB0EE600A0120FEF7B8FF1FED670A7F4880ED000A06E006E01FED6A0A7C4880ED000A00BF00BFBDEC068B7C
:40D3400010BD784890F8280008B9012070470020FCE7744890F82800012800D170470020FCE7704890F82800032801D1012070470020FCE76B4890F8500008B90120704750
:40D380000020FCE7674890F85000012800D170470020FCE7634890F85000032801D1012070470020FCE700B50021FFF7CAFF08B13D2103E0FFF7CDFF00B13C21084600BD6A
:40D3C00000B50021FFF7CDFF08B1082117E0FFF7B8FF08B1072112E0FFF7BBFF08B106210DE0FFF7D7FF08B10B2108E0FFF7A9FF08B10A2103E0FFF7ACFF00B109210846F7
:40D4000000BD10B519F08BFA0446204610BD10B52DED028B0BF076FE20B1FDF7DBFFB0EE408A16E019F056F93C48D0ED640A30EE600ADFED410A20EE200AD0ED650A90ED00
:40D44000641A70EEC10A80EE201A9FED3C0A31EE008AB0EE480ABDEC028B10BD01B59DF80000202801DD2020009000BF01226946334800684B300EF007F820B99DF8000054
:40D48000264981F84B0000BF0020264981F86D0208BD10B54FF41C71224831F0D8FE10BD28490870704727480078704710B52DED028BB0EE408A2448007830B9144800211F
:40D4C0000160416001202049087023F08DF8F0EE408AF0EE680AB0EE480A18F0F4FF1B4880ED000A28210A48184A92ED000A1AF048F8BDEC028B10BD144890ED000A704766
:40D50000134890ED000A704753070020804500204C000020000000A046DF913F1821002084000020E80D0020000000A046DF813F2FDDE43E0AD7A33B000048430000C8C259
:40D54000F00300204400002085000020480000205400002010B50446204625F04FF910BD07B586B000200490002108980170069800786F2881F0AF82DFE810F06F00710046
:40D58000ED000D013B01AD0AB10050075B0766076901CF01E1014702BC0211036603B303080470045D048200BD042F059D05E3053206B0060D09CA0671079B097D07C30730
:40D5C000D20710081E082C0872087E088E089808A808AD0AAD0AAD0AB808C908E308890795079F07B707AB07AD0AAD0AAD0AAD0AAD0AAD0AAD0AAD0AAD0AAD0AAD0AD40462
:40D60000AD0AAD0AAD0A1109390956097E09AD0AAD0AAD0AAD0AAD0AAD0AAD0AAD0AAD0AAD0AAD0AAD0AAD0AAD0AAD0AAD0AAD0AAD0AAD0AAB09DC090D0AAD0AAD0AAD0A19
:40D640001F0A670AAD0AAD0AAD0AAD0A310A430AAD0A550A790A8B0A9D0A01F040BAF94890F841000390069890ED010ABCEEC00A10EE100AC0B20290039919F07CF8ECE7AD
:40D680000698007A032803D006210898017025E0069890ED010AF7EE000AB4EE600AF1EE10FA02D117F099F918E0069890ED010AF0EE000AB4EE600AF1EE10FA02D117F0CC
:40D6C00074F90BE0069890ED010AF0EE080AB4EE600AF1EE10FA01D116F06DFFBDE70698007A032809D1069890ED010A8DED030A9DED030A10F05CF82AE00698007A0128DF
:40D7000011D1D048B0F8BE110A22079802FB001000EE100AB8EEC00A8DED030A9DED030A10F046F814E00698007A022810D1C548B0F8BE110A22079802FB101000EE100A41
:40D74000B8EEC00A8DED030A9DED030A10F030F80120049081E70AF0CFF8C0B90698007A032811D1069890ED010A8DED030A9DED030A0BF0E0F8B448D0F8180101460390A9
:40D780008020DFF8C8C200DF0120049002E001210898017061E716F081FA30BB0698007A03281ED1069890ED010ABCEEC00A10EE100A80B203900BF09CF80BF019F880B98E
:40D7C0000821A348DFF88CC200DF012809D0A248406840F00100A04948609D48DFF87CC200DF182023F056FC02E001210898017033E716F053FA30BB0AF0FAFF18B306987C
:40D80000007A03281BD1069890ED010ABCEEC00A10EE100AC0B203900BF045F808218C48DFF830C200DF012809D08B48406840F00100894948608648DFF820C200DF1820FD
:40D8400023F028FC02E001210898017005E70698007A032817D17B4890F842000390794890F841000290069890ED010ABCEEC00A10EE100AC0B20190DDE9021212F09AFCE2
:40D880000899087046E00698007A01281FD16D4890F841105C3000EB41006A4991F84210415C0122079802FB0010C0B20190654890F842000390634890F84100029001465E
:40D8C000039A019812F076FC0899087022E00698007A02281ED15B4890F841105C3000EB4100584991F84210415C0122079802FB1010C0B20190534890F842000390514872
:40D9000090F8410002900146039A019812F052FC08990870012004909FE60698007A03280CD1069890ED010ABCEEC00A10EE100AC0B2039012F07AFC089908708DE60698F3
:40D94000007A032817D13F4890F8420003903D4890F841000290069890ED010ABCEEC00A10EE100AC0B20190DDE9021212F08AFC0899087046E00698007A01281FD1314856
:40D9800090F84110603000EB41002E4991F84210415C0122079802FB0010C0B20190294890F842000390274890F8410002900146039A019812F066FC0899087022E00698DF
:40D9C000007A02281ED11F4890F84110603000EB41001C4991F84210415C0122079802FB1010C0B20190174890F842000390154890F8410002900146039A019812F042FCA8
:40DA0000089908700120049027E60698007A032826D10C4890F8420003900A4890F841000290069890ED010ABCEEC00A10EE100AC0B20190DDE9021212F074FC0899087059
:40DA400055E000001821002060420020892304084032002051280408503200206D2704080698007A01281FD1FB4890F84110643000EB4100F84991F84210415C01220798BD
:40DA800002FB0010C0B20190F34890F842000390F14890F8410002900146039A019812F041FC0899087022E00698007A02281ED1E94890F84110643000EB4100E64991F8A0
:40DAC0004210415C0122079802FB1010C0B20190E14890F842000390DF4890F8410002900146039A019812F01DFC0899087001200490B2E50698007A032810D1D64890F886
:40DB000042000390069890ED010A8DED020A03989DED020A12F063FD089908703CE00698007A01281AD1CC4890F842107C3000EB8100D0ED000A9DED070AB8EEC00A30EE7A
:40DB4000C00A8DED020AC44890F8420003909DED020A12F044FD089908701DE00698007A022819D1BC4890F842107C3000EB8100D0ED000A9DED070AB8EEC00A30EE800A61
:40DB80008DED020AB44890F8420003909DED020A12F025FD08990870012004905DE50698007A032810D1AC4890F842000390069890ED010A8DED020A03989DED020A12F068
:40DBC00054FC089908703CE00698007A01281AD1A14890F842106C3000EB8100D0ED000A9DED070AB8EEC00A30EEC00A8DED020A994890F8420003909DED020A12F035FC62
:40DC0000089908701DE00698007A022819D1924890F842106C3000EB8100D0ED000A9DED070AB8EEC00A30EE800A8DED020A8A4890F8420003909DED020A12F016FC08996C
:40DC400008700120049008E50698007A032812D1814890F842000390069890ED010ABCEEC00A10EE100AC0B20290039912F097FB0899087032E00698007A012815D1764848
:40DC800090F842106830415C0122079802FB0010C0B20290704890F8420001460390029812F07DFB0899087018E00698007A022814D1694890F842106830415C0122079858
:40DCC00002FB1010C0B20290634890F8420001460390029812F063FB0899087001200490BBE40698007A032810D15B4890F842000390069890ED010A8DED020A03989DED58
:40DD0000020A12F0CAFC089908703CE00698007A01281AD1504890F84210843000EB8100D0ED000A9DED070AB8EEC00A30EE800A8DED020A484890F8420003909DED020A99
:40DD400012F0ABFC089908701DE00698007A022819D1414890F84210843000EB8100D0ED000A9DED070AB8EEC00A30EEC00A8DED020A394890F8420003909DED020A12F07F
:40DD80008CFC089908700120049066E40698007A032810D1304890F842000390069890ED010A8DED020A03989DED020A12F0BBFB089908703CE00698007A01281AD1264866
:40DDC00090F84210743000EB8100D0ED000A9DED070AB8EEC00A30EE800A8DED020A1E4890F8420003909DED020A12F09CFB089908701DE00698007A022819D1164890F81F
:40DE00004210743000EB8100D0ED000A9DED070AB8EEC00A30EEC00A8DED020A0E4890F8420003909DED020A12F07DFB089908700120049011E40698007A03280AD10698FE
:40DE400090ED010ABCEEC00A10EE100AC0B20390FCF799FA13E40000182100200698007A032812D1F74890F842000390069890ED010ABCEEC00A10EE100AC0B2029003999F
:40DE800012F0C0FA0899087032E00698007A012815D1EC4890F842106A30415C0122079802FB0010C0B20290E64890F8420001460390029812F0A6FA0899087018E006987F
:40DEC000007A022814D1DF4890F842106A30415C0122079802FB1010C0B20290D94890F8420001460390029812F08CFA08990870012004902EE40698007A032803D006217A
:40DF0000089801700DE0069890ED010A8DED030A9DED030A0A2009F06DFB10B901210898017017E40698007A032814D1069890ED010ABCEEC00A10EE100A80B200EE100A09
:40DF4000B8EE400A8DED030A9DED030A0FF030FC089908703EE00698007A01281BD110F0DEF9F0EE400AB748B0F8BE0100EE100AB8EE401A9DED070AF8EE401AB0EE410AD3
:40DF800000EEA10A8DED030A9DED030A0FF010FC089908701EE00698007A02281AD110F0BEF9F0EE400AA748B0F8BE0100EE100AB8EE401A9DED070AF8EE401AB0EE410A5A
:40DFC00000EEE10A8DED030A9DED030A0FF0F0FB08990870012004900AE40698007A032815D1984890F842000390964890F841000290069890ED010A8DED010ADDE9020171
:40E000009DED010A12F085F80899087050E00698007A012824D18B4890F842000290894890F841000190029910F066FADDED070AF8EE600A9FED841A01EE200A8DED030A03
:40E04000804890F8420002907E4890F84100019002999DED030A12F05CF80899087027E00698007A022823D1764890F842000290744890F841000190029910F03DFADDEDB2
:40E08000070AF8EE600A9FED701A01EE600A8DED030A6C4890F8420002906A4890F84100019002999DED030A12F033F8089908700120049030E40698007A03280BD10698EF
:40E0C00090ED010A8DED030A9DED030A12F082FB0899087032E00698007A012815D15948D0ED7E0A9DED070AB8EE401ADFED571AB0EE600A01EE810A8DED030A9DED030A4B
:40E1000012F068FB0899087018E00698007A022814D14C48D0ED7E0A9DED070AB8EE401ADFED4A1AB0EE600A01EEC10A8DED030A9DED030A12F04EFB0899087001200490A5
:40E1400062E40698007A032814D1069890ED010ABCEEC00A10EE100A80B200EE100AB8EE400A8DED030A9DED030AFCF729F90899087032E00698007A012815D13148D0ED9A
:40E18000280A079800EB8000400000EE100AB8EEC00A30EE800A8DED030A9DED030AFCF70FF90899087018E00698007A022814D12448D0ED280A079800EB8000400000EEDF
:40E1C000100AB8EEC00A30EEC00A8DED030A9DED030AFCF7F5F8089908700120049039E20698007A032835D1069890ED010ADFED180AB4EEE00AF1EE10FA06DD022108984E
:40E200000170642006F0C4FA62E0069890ED010AF2EE040AB4EEE00AF1EE10FA06D20321089801700A2006F0B3FA51E0069890ED010ABCEEC00A10EE100AC0B2039006F0B2
:40E24000A7FA45E0182100200AD7233CCDCCCC3D0000C8420698007A01281BD1FE4890F8401007984000C0F1650081420BDAFA4890F840100222079802FB0010C0B20390BC
:40E2800006F086FA24E0022108980170642006F07FFA1DE00698007A022819D1EE4890F8401007984000093081420BDDEA4890F840100222079802FB1010C0B2039006F0DE
:40E2C00067FA05E00321089801700A2006F060FA1A20FFF73FF901200490BBE10698007A032803D006210898017010E0069890ED010ABCEEC00A10EE100AC0B21FED2C0ACC
:40E30000039009F077F910B9012108980170E6E30698007A032803D00621089801707CE0069890ED010AF8EE000AB4EE600AF1EE10FA13D1C84890F842107C3000EB810081
:40E3400090ED000A8DED030A9DED030A082009F051F900BB0121089801705EE0069890ED010AFFEE000AB4EE600AF1EE10FA13D1B94890F842106C3000EB810090ED000A01
:40E380008DED030A9DED030A082009F033F910B901210898017040E0069890ED010AF7EE000AB4EE600AF1EE10FA13D1AA4890F84210743000EB810090ED000A8DED030AFE
:40E3C0009DED030A082009F015F900BB01210898017022E0069890ED010AF0EE000AB4EE600AF1EE10FA13D19B4890F84210843000EB810090ED000A8DED030A9DED030AFE
:40E40000082009F0F7F810B901210898017004E09FED920A002009F0EDF860E30020FEF767F88DED030A00209DED030AFDF708FF55E30020FEF75CF88DED030A00209DED04
:40E44000030AFDF725FF4AE30020FEF751F88DED030A00209DED030AFDF795FF3FE3069890ED010ABCEEC00A10EE100AC0B203900FF0ABFD33E3069890ED010ABCEEC00AF6
:40E4800010EE100AC0B20390FEF7D3F927E3069890ED010ABCEEC00A10EE100AC0B2039012F0F5FA1BE3069890ED010A8DED030A9DED030A12F000FB11E3069890ED010A73
:40E4C000BCEEC00A10EE100AC0B2039013F036F805E3069890ED010ABCEEC00A10EE100A80B2039012F00EFEF9E2069890ED010ABCEEC00A10EE100A80B2039012F017FE84
:40E50000EDE2069890ED010ABCEEC00A10EE100AC0B2039010F0D0FF2120FFF71BF8DEE20698007A032803D006210898017034E0069890ED010AF7EE000AB4EE600AF1EE1A
:40E5400010FA0ED10AF013FD28B1B7EE000A112009F050F821E0B7EE000A072009F04AF81BE0069890ED010AF0EE000AB4EE600AF1EE10FA05D19FED390A002009F03AF8AE
:40E580000BE0069890ED010AF0EE080AB4EE600AF1EE10FA01D100F08BFCA0E2069890ED010ABCEEC00A10EE100A80B201460390022017F0EAFE92E2069890ED010ABCEE87
:40E5C000C00A10EE100A80B201460390012017F0DCFE84E20698007A03283BD1069890ED010AB5EEC00AF1EE10FA0BD11A4890F842000390184890F84100029003990AF00E
:40E6000071FB27E0069890ED010AF7EE000AB4EE600AF1EE10FA07D10F4890F84200012103900AF0C8FA15E0069890ED010AF0EE080AB4EE600AF1EE10FA0BD1064890F841
:40E6400042000390044890F841000122029003990AF030FA43E200001821002000000000069890ED010ABCEEC00A10EE100AC0B203900AF0F1F932E20698007A03280AD1F0
:40E68000069890ED010ABCEEC00A10EE100AC0B20390FBF7BAFF22E215F000FB28B90698007A032801D10AF078F918E20698007A03280AD1069890ED010ABCEEC00A10EEE3
:40E6C000100AC0B20390FDF79BFC08E20698007A03280AD1069890ED010ABCEEC00A10EE100AC0B20390FDF7A3FCF8E10698007A03280BD1069890ED010ABCEEC00A10EE8E
:40E70000100AC0B20121039012F026FDE7E10698007A032814D1069890ED010ADFEDFE0AB4EE600AF1EE10FA0AD10DF0ECFF01200DF068FE0021F94801720020F84908709F
:40E74000CDE10698007A03280BD1069890ED010ABDEEC00A10EE100A00B20390FAF784F918E00698007A012808D1EE48B0F8AA00401C00B20390FAF777F90BE00698007AC7
:40E78000022807D1E748B0F8AA00401E00B20390FAF76AF9A3E11C20FEF7DCFE9FE10698007A03281AD1DF4890F842106C3000EB810090ED000A8DED050A9DED050AB5EE4D
:40E7C000C00AF1EE10FA03D19FEDD70A8DED050A9DED050A082008F00DFF07E00698007A20B91FED620A082008F004FF77E10698007A03280FD1CB4890F842107C3000EB65
:40E80000810090ED000A8DED030A9DED030A082008F0F0FE07E00698007A20B91FED710A082008F0E7FE5AE10698007A03281AD1BC4890F84210743000EB810090ED000A62
:40E840008DED050A9DED050AB5EEC00AF1EE10FA03D19FEDB60A8DED050A9DED050A082008F0C8FE07E00698007A20B91FED850A082008F0BFFE32E10698007A03280FD172
:40E88000A84890F84210843000EB810090ED000A8DED030A9DED030A082008F0ABFE07E00698007A20B91FED930A082008F0A2FE15E10698007A03280AD1069890ED010A85
:40E8C000BCEEC00A10EE100AC0B203900AF0A5F805E10698007A03280ED1069890ED010ABCEEC00A10EE100A80B201210390FCF76CFF089908701CE00698007A01280AD1C0
:40E90000FCF7E0FE401C80B201210390FCF75DFF089908700DE00698007A022809D1FCF7D1FE401E80B201210390FCF74EFF08990870D4E00698007A03280ED1069890ED01
:40E94000010ABCEEC00A10EE100A80B201210390FCF753FF089908701CE00698007A01280AD1FCF7ABFE401C80B201210390FCF744FF089908700DE00698007A022809D16C
:40E98000FCF79CFE401E80B201210390FCF735FF08990870A3E00698007A03280CD1069890ED010ABCEEC00A10EE100A80B20390FCF73BFF0899087091E00698007A032831
:40E9C0000CD1069890ED010ABCEEC00A10EE100A80B20390FCF740FF089908707FE00698007A03280CD1069890ED010ABCEEC00A10EE100A80B20390FCF749FF089908702E
:40EA00006DE00698007A03280CD1069890ED010ABCEEC00A10EE100A80B20390FCF766FF089908705BE00698007A03280CD1069890ED010ABCEEC00A10EE100AC0B203906F
:40EA400017F085FF0899087049E00698007A03280CD1069890ED010ABCEEC00A10EE100A80B20390FCF75DFF0899087037E00698007A03280CD1069890ED010ABDEEC00AF8
:40EA800010EE100A00B20390FCF77DFF0899087025E00698007A03280CD1069890ED010ABDEEC00A10EE100A00B20390FCF754FF0899087013E00698007A03280AD1069846
:40EAC00090ED010ABCEEC00A10EE100AC0B20390FDF7D5F803E007210898017000BF00BF049809B000BD86B04FF6FF7438211048DFF840C000DF02210F4880F808110C2202
:40EB000084210E4833F0EAFA002879D103210A4880F8081100BF13E000007E43503200203C05002018210020CDCCCCBDCDCCCC3DF010002011250408604200206C10002007
:40EB4000224605A98748DFF820C200DF012858D000208DF800008DF80D0001208DF80C0000208DF80E0005980078002839D004AA01210598FEF7F4FC05469DF8100068B18A
:40EB800000250599087824F0A7F906460598837A427A9DF81010304624F0A4F908F0ACFE08B1002504E00598007A032800D100250DB39DF80D00F0B90598007AD8B1059AFA
:40EBC00007CA8DE8070001208DF80D008DF80C004FF47A649DF80E00401CC0B28DF80E0009E008F03EFD30B16048D0F890110120DFF87CC100DF5F480599F9F781FB8AE71B
:40EC000047E09DF80000002885DD9DF80E0000283CDD9DF80E00032803D102208DF80C000EE09DF80E00052803D106208DF80C0006E09DF80E00072802D110208DF80C00C0
:40EC40009DF80E00FF2805DA9DF80E00401CC0B28DF80E009DF80C1004AA6846FEF780FC9DF8100078B100208DF80E000599087824F032F906460598837A427A9DF8101034
:40EC8000304624F02FF94FF4FA6444E74FF6FF7441E70521354880F808110020DFF8D8C000DF00BFFEE72DE9F0472DED028B0546B0EE408A0E46174698464FF001092948C0
:40ECC000DFF8B8C000DFD0B900BF284890F8090140F00201254880F80911B0F814014FF6FF71884207DA2148B0F81401401C81B21E48A0F8141100BF4FF000092CE01D48FD
:40ED0000F9F7EEFA04466CB1257084ED018A2672677284F80A800A2221461248DFF860C000DF19E000BF114890F8090140F004010E4880F80911B0F814014FF6FF718842CD
:40ED400007DA0A48B0F81401401C81B20748A0F8141100BF4FF000094846BDEC028BBDE8F0870000F0100020A126040860420020892304086C1000200D2E04080925040897
:40ED8000FD25040831B52DED020B0446FE4890EDD40ADDED000AB4EEE00AF1EE10FA00D3ACB100BF04226946F848006800F554700CF06AFB20B99DED000AF34880EDD40A6B
:40EDC00000BFF348C16B0220DFF8C8C300DF3EBD31B52DED020B0446EB4890EDD30ADDED000AB4EEE00AF1EE10FA00DCACB100BF04226946E548006800F553700CF044FB0D
:40EE000020B99DED000AE04880EDD30A00BFE048C16B0220DFF87CC300DF3EBD31B52DED020B0446D84890ED2F0ADDED000AB4EEE00AF1EE10FA00D3A4B100BF042269469C
:40EE4000D2480068BC300CF01FFB20B99DED000ACD4880ED2F0A00BFCD48C16B0220DFF834C300DF3EBD31B52DED020B0446C64890ED2E0ADDED000AB4EEE00AF1EE10FAB9
:40EE800000DCA4B100BF04226946C0480068B8300CF0FAFA20B99DED000ABB4880ED2E0A00BFBB48C16B0220DFF8E8C200DF3EBD10B54FF4F671B84830F0C9F9B24890F8F2
:40EEC0002800B54981F8E0012AF083FDB2498860012081F8DC01002081F8DD019FEDAF0A084680ED500A002007F0BFF801209FEDAB0AFFF7B8FF01209FEDA80AFFF78EFF0E
:40EF000001209FEDA60AFFF763FF01209FEDA30AFFF738FF10BD10B517F037FDA04880ED000A90ED000AF2EE000A20EE200ADFED9D0A80EE201A9C4880ED001A984890EDDD
:40EF4000000AF0EE080A20EE200ADFED960A80EE201A964880ED001A914890ED000AF3EE010A20EE200ADFED8F0A80EE201A904880ED001A10BD10B5002428F055F940B3E7
:40EF80008C4800680078012800D128E0894800680078022801D1142421E0864800680078052801D128241AE0824800680078032801D13C2413E07F4800680078062801D121
:40EFC00050240CE07B4800680078082807D1642405E028F041F910B16F4890F8E141204610BD10B56C4890F8DD0173490978884203D0FFF7C0FF7149087010BD70B52DED46
:40F00000028B044614F04AFE00287DD1002596E05D48C03000EB8400D0ED000AB0EE600A284611F013FC5848C03000EB8400D0ED000AB0EE600A284611F017FA5248C8306B
:40F0400000EB8400D0ED000AB0EE600A284611F021FC4D48C83000EB8400D0ED000AB0EE600A284611F05FFA4748D03000EB8400D0ED000AB0EE600A284611F02FFC424842
:40F08000D03000EB8400D0ED000AB0EE600A284611F0A5FA3C48D83000EB8400D0ED000AB0EE600A284611F03DFC3748D83000EB8400D0ED000AB0EE600A284611F0EDFA77
:40F0C0003149E031085D294611F050FC2E49E231085D294611F068FC28F0A6F808B32A49E0310A5D891C095D501800EBD071491000EE101AB8EEC00AB0EE408ABCEEC80AE1
:40F1000010EE101AC8B200E01DE0214611F047F9BCEEC80A10EE101AC8B2214611F072F90BE01949E031085D214611F038F91649E231085D214611F065F9681CC5B2022D94
:40F14000FFF666AFAFE01048C03000EB8400D0ED000AB0EE600A204611F078FB0A48C03000EB8400D0ED000AB0EE600A204611F07CF90548C83000EB8400D0ED000AB0EE21
:40F18000600A20461CE0000018210020F003002060420020892304082811002000000000700300200000C84274030020780300207C03002048030020800300206E03002037
:40F1C00011F068FBFE4800EB8400D0ED000AB0EE600A204611F0A7F9F948083000EB8400D0ED000AB0EE600A204611F077FBF448083000EB8400D0ED000AB0EE600A204678
:40F2000011F0EDF9EE48103000EB8400D0ED000AB0EE600A204611F085FBE948103000EB8400D0ED000AB0EE600A204611F035FAE3491831085D214611F098FBE0491A31BE
:40F24000085D214611F0B0FB27F0EEFFF8B1DC4918310A5D891C095D501800EBD071491000EE101AB8EEC00AB0EE408ABCEEC80A10EE101AC8B2214611F091F8BCEEC80A21
:40F2800010EE101AC8B2214611F0BCF80BE0CC491831085D214611F082F8C9491A31085D214611F0AFF8BDEC028B70BD01B500BF01226946C348006800F5E9700CF0E4F8EC
:40F2C00028B99DF80000BE49C83981F8D20100BF08BD10B5032006F0C8FE1FED500A002008F088F90120FFF7E1FFB549C83991F84200FFF783FE1C2021F0CCFE10BD01B54B
:40F30000B8B000203590349033903290319030902F902E901FED5F0A389880ED530A1FED610A389880ED560A1FED640A389880ED540A1FED660A389880ED580A1FED690A67
:40F34000389880ED550A1FED6B0A389880ED590A01203790FEE3379834F0B6F99FED9A0B53EC102BCDE926019DED260B51EC100B33F0A2FFCDE92C0137983690389890ED41
:40F380006A0B8DED200B9DED2C0B53EC102B9DED200B51EC100B34F0E7F9CDE92401389890ED680B8DED1A0B9DED2C0B53EC102B9DED1A0B51EC100B34F0D6F9CDE91C01A5
:40F3C0009DED2C0B53EC102B9DED1C0B51EC100B34F0CAF9CDE92001389890ED660B8DED140B9DED2C0B53EC102B9DED140B51EC100B34F0B9F9CDE916019DED2C0B53ECD5
:40F40000102B9DED160B51EC100B34F0ADF9CDE918019DED2C0B53EC102B9DED180B51EC100B34F0A1F9CDE91C01389890ED640B8DED0E0B9DED2C0B53EC102B9DED0E0BF7
:40F4400051EC100B34F090F9CDE910019DED2C0B53EC102B9DED100B51EC100B34F084F9CDE912019DED2C0B53EC102B9DED120B51EC100B34F078F9CDE914019DED2C0BC3
:40F4800053EC102B9DED140B51EC100B34F06CF9CDE91801389890ED620B8DED080B9DED2C0B53EC102B9DED080B51EC100B34F05BF9CDE90A019DED2C0B53EC102B9DED04
:40F4C0000A0B51EC100B34F04FF9CDE90C019DED2C0B53EC102B9DED0C0B51EC100B34F043F9CDE90E019DED2C0B53EC102B9DED0E0B51EC100B34F037F9CDE910019DED3C
:40F500002C0B53EC102B9DED100B51EC100B34F02BF9CDE91401389890ED600B8DED020B9DED2C0B53EC102B9DED020B51EC100B34F01AF9CDE904019DED2C0B53EC102B74
:40F540009DED040B51EC100B34F00EF9CDE906019DED2C0B53EC102B9DED060B51EC100B34F002F9CDE908019DED2C0B53EC102B9DED080B51EC100B34F0F6F8CDE90A01A3
:40F580009DED2C0B53EC102B9DED0A0B51EC100B34F0EAF8CDE90C019DED2C0B53EC102B9DED0C0B51EC100B34F0DEF8CDE91001389890ED5E0B8DED000B9DED2C0B07E078
:40F5C000E0210020F0030020000000000000244053EC102B9DED000B51EC100B34F0C4F8CDE902019DED2C0B53EC102B9DED020B51EC100B34F0B8F8CDE904019DED2C0BF9
:40F6000053EC102B9DED040B51EC100B34F0ACF8CDE906019DED2C0B53EC102B9DED060B51EC100B34F0A0F8CDE908019DED2C0B53EC102B9DED080B51EC100B34F094F851
:40F64000CDE90A019DED2C0B53EC102B9DED0A0B51EC100B34F088F8CDE90C019DED2C0B53EC102B9DED0C0B51EC100B34F07CF8CDE90E019DED100B53EC102B9DED0E0BDD
:40F6800051EC100B33F05CFDCDE912019DED140B53EC102B9DED120B51EC100B33F050FDCDE916019DED180B53EC102B9DED160B51EC100B33F044FDCDE91A019DED1C0B3E
:40F6C00053EC102B9DED1A0B51EC100B33F038FDCDE91E019DED200B53EC102B9DED1E0B51EC100B33F02CFDCDE922019DED240B53EC102B9DED220B51EC100B33F020FD7B
:40F70000CDE92601389890ED6C0B8DED240B9DED240B53EC102B9DED260B51EC100B33F00FFDCDE92A01389890ED7A0B8DED200B9DED2C0B53EC102B9DED200B51EC100B6A
:40F7400034F012F8CDE92401389890ED780B8DED1A0B9DED2C0B53EC102B9DED1A0B51EC100B34F001F8CDE91C019DED2C0B53EC102B9DED1C0B51EC100B33F0F5FFCDE9CE
:40F780002001389890ED760B8DED140B9DED2C0B53EC102B9DED140B51EC100B33F0E4FFCDE916019DED2C0B53EC102B9DED160B51EC100B33F0D8FFCDE918019DED2C0BEA
:40F7C00053EC102B9DED180B51EC100B33F0CCFFCDE91C01389890ED740B8DED0E0B9DED2C0B53EC102B9DED0E0B51EC100B33F0BBFFCDE910019DED2C0B53EC102B9DEDCB
:40F80000100B51EC100B33F0AFFFCDE912019DED2C0B53EC102B9DED120B51EC100B33F0A3FFCDE914019DED2C0B53EC102B9DED140B51EC100B33F097FFCDE9180138985D
:40F8400090ED720B8DED080B9DED2C0B53EC102B9DED080B51EC100B33F086FFCDE90A019DED2C0B53EC102B9DED0A0B51EC100B33F07AFFCDE90C019DED2C0B53EC102B9C
:40F880009DED0C0B51EC100B33F06EFFCDE90E019DED2C0B53EC102B9DED0E0B51EC100B33F062FFCDE910019DED2C0B53EC102B9DED100B51EC100B33F056FFCDE91401FE
:40F8C000389890ED700B8DED020B9DED2C0B53EC102B9DED020B51EC100B33F045FFCDE904019DED2C0B53EC102B9DED040B51EC100B33F039FFCDE906019DED2C0B53EC29
:40F90000102B9DED060B51EC100B33F02DFFCDE908019DED2C0B53EC102B9DED080B51EC100B33F021FFCDE90A019DED2C0B53EC102B9DED0A0B51EC100B33F015FFCDE938
:40F940000C019DED2C0B53EC102B9DED0C0B51EC100B33F009FFCDE91001389890ED6E0B8DED000B9DED2C0B53EC102B9DED000B51EC100B33F0F8FECDE902019DED2C0B4E
:40F9800053EC102B9DED020B51EC100B33F0ECFECDE904019DED2C0B53EC102B9DED040B51EC100B33F0E0FECDE906019DED2C0B53EC102B9DED060B51EC100B33F0D4FE09
:40F9C000CDE908019DED2C0B53EC102B9DED080B51EC100B33F0C8FECDE90A019DED2C0B53EC102B9DED0A0B51EC100B33F0BCFECDE90C019DED2C0B53EC102B9DED0C0BC0
:40FA000051EC100B33F0B0FECDE90E019DED100B53EC102B9DED0E0B51EC100B33F090FBCDE912019DED140B53EC102B9DED120B51EC100B33F084FBCDE916019DED180B09
:40FA400053EC102B9DED160B51EC100B33F078FBCDE91A019DED1C0B53EC102B9DED1A0B51EC100B33F06CFBCDE91E019DED200B53EC102B9DED1E0B51EC100B33F060FB59
:40FA8000CDE922019DED240B53EC102B9DED220B51EC100B33F054FBCDE92601389890ED7C0B8DED240B9DED240B53EC102B9DED260B51EC100B33F043FBCDE92801642154
:40FAC000369890FBF1F201FB120008BB9DED2A0B51EC100B33F002FB01466422369890FBF2F2521E389800F5027040F822109DED280B51EC100B33F0F1FA014664223698E9
:40FB000090FBF2F2521E389800F50C7040F82210389890ED000AB1EE400A8DED250A259834F018F9CDE926019DED2A0B53EC102B9DED260B51EC100B33F014FF2AD2359838
:40FB4000401C80B235909DED350AB8EE400ADFEDFE0A00E028E2B4EEE00AF1EE10FA1BDD389890ED530AB5EEC00AF1EE10FA13D19DED2C0B51EC100B33F0B0FA00EE100A7C
:40FB8000B1EE400AF3EE040A30EE200A389880ED530A01E000203590389890ED000AB1EE400A8DED250A259834F0D4F8CDE926019DED2A0B53EC102B9DED260B51EC100B06
:40FBC00033F0D0FE26D23498401C80B234909DED340AB8EE400ADFEDDC0AB4EEE00AF1EE10FA19DD9DED2C0B51EC100B33F076FA00EE100AF1EE400A9DED340AB8EE400A94
:40FC0000B2EE041AC0EE011A30EEA10A389880ED520A01E000203490389890ED010AB1EE400A8DED250A259834F094F8CDE926019DED2A0B53EC102B9DED260B51EC100B96
:40FC400033F090FE28D23198401C80B231909DED310AB8EE400AF1EE040AB4EEE00AF1EE10FA1BDD389890ED540AB5EEC00AF1EE10FA13D19DED2C0B51EC100B33F02EFA69
:40FC800000EE100AB1EE400AF6EE000A30EE200A389880ED540A01E000203190389890ED030AB1EE400A8DED250A259834F052F8CDE926019DED2A0B53EC102B9DED260BD8
:40FCC00051EC100B33F04EFE28D22F98401C80B22F909DED2F0AB8EE400AF1EE040AB4EEE00AF1EE10FA1BDD389890ED550AB5EEC00AF1EE10FA13D19DED2C0B51EC100B23
:40FD000033F0ECF900EE100AB1EE400AF6EE000A30EE200A389880ED550A01E000202F9038980068259034F015F8CDE926019DED280B53EC102B9DED260B51EC100B33F0D0
:40FD4000D7FC26D23398401C80B233909DED330AB8EE400ADFED7C0AB4EEE00AF1EE10FA19DD389890ED560AB5EEC00AF1EE10FA11D19DED2C0B51EC100B33F0AFF900EE71
:40FD8000100AF3EE040A30EE600A389880ED560A01E00020339038980068259033F0DAFFCDE926019DED280B53EC102B9DED260B51EC100B33F09CFC24D23298401C80B238
:40FDC00032909DED320AB8EE400ADFED5F0AB4EEE00AF1EE10FA17DD9DED2C0B51EC100B33F07CF900EE900A9DED320AB8EE400AB2EE041AC0EE011A30EEE10A389880ED31
:40FE0000570A01E00020329038984068259033F0A1FFCDE926019DED280B53EC102B9DED260B51EC100B33F063FC26D23098401C80B230909DED300AB8EE400AF1EE040A56
:40FE4000B4EEE00AF1EE10FA19DD389890ED580AB5EEC00AF1EE10FA11D19DED2C0B51EC100B33F03BF900EE100AF6EE000A30EE600A389880ED580A01E000203090389812
:40FE8000C068259033F066FFCDE926019DED280B53EC102B9DED260B51EC100B33F028FC26D22E98401C80B22E909DED2E0AB8EE400AF1EE040AB4EEE00AF1EE10FA19DD5B
:40FEC000389890ED590AB5EEC00AF1EE10FA11D19DED2C0B51EC100B33F000F900EE100AF6EE000A30EE600A389880ED590A01E000202E90389890ED5C0AB1EE400A8DEDF2
:40FF0000250A259833F026FFCDE926019DED2A0B53EC102B9DED260B51EC100B33F022FD19D29DED2A0B51EC100B33F0D7F83899C1F870019DED2C0B51EC100B33F0CEF831
:40FF400000EE100A02E0000000004843B1EE400A389880ED5A0A3898D0F87401259033F0F9FECDE926019DED280B53EC102B9DED260B51EC100B33F0BBFB11D29DED280B06
:40FF800051EC100B33F0AAF83899C1F874019DED2C0B51EC100B33F0A1F83899C1F86C013798401C80B237903798B0F57A7F7FF7D2A9389890ED540AB5EEC00AF1EE10FAD6
:40FFC0000BD0389890ED540A80ED5A0A389890ED010AB1EE400A80ED5C0A389890ED580AB5EEC00AF1EE10FA09D0389890ED580A80ED5B0A389890ED010A80ED5D0A38983B
:020000040801F1
:4000000090ED530AB5EEC00AF1EE10FA61D0389890ED560AB5EEC00AF1EE10FA59D0389890ED5A0AD0ED530AB7EE001A70EEC10AB4EEE00AF1EE10FA4BDC389890ED5B0A32
:40004000D0ED560AB7EE001A70EE810AB4EEE00AF1EE10FA3DD3389890ED530AD0ED520A30EE600A8DED230A239833F073FECDE924019DED240B30F047FA8DED260B9FEDC9
:40008000F80B53EC102B9DED260B51EC100B33F069FC1ED3389890ED560AD0ED570A30EE600A8DED230A239833F054FECDE924019DED240B30F028FA8DED260B9FEDE80B0D
:4000C00053EC102B9DED260B51EC100B33F04AFC03D22320E44981F8DA01389890ED550AB5EEC00AF1EE10FA04D19FEDE00A389880ED550A389890ED590AB5EEC00AF1EE8C
:4001000010FA04D19FEDDA0A389880ED590A39B000BD70B52DED088B064600246FE09FEDD50BB0EE408AF0EE608A9FEDD20BB0EE409AF0EE609A002551E006F1400000EBCC
:40014000850090ED000A10EE101A084633F002FE41EC1B0B04EB440000EBC400C74901EBC00000EBC50090ED001BB0EE410AF0EE610A53EC102B51EC1B0B33F0F5FA53EC41
:40018000182B32F0DDFF41EC180B06F16C0000EB850090ED000A10EE101A084633F0DAFD41EC1B0B04EB440000EBC400B34901EBC00000EBC50090ED001BB0EE410AF0EEF8
:4001C000610A53EC102B51EC1B0B33F0CDFA53EC192B32F0B5FF41EC190B681CC5B20B2DABDB06F5BC7000EBC40080ED008B06F5DC7000EBC40080ED009B601CC4B2082C78
:400200008DDBBDEC088B70BD70B504469C4890F82850022D14D19FED9B0A84ED000A9FED9A0A84ED010A9FED990A84ED020A9FED980A84ED030A9FED970A84ED040A89E0C1
:400240000D2D14D19FED8F0A84ED000A9FED8E0A84ED010A9FED8D0A84ED020A9FED8E0A84ED030A9FED8B0A84ED040A72E00C2D14D19FED840A84ED000A9FED830A84EDAE
:40028000010A9FED820A84ED020A9FED830A84ED030A9FED800A84ED040A5BE0032D14D19FED780A84ED000A9FED770A84ED010A9FED760A84ED020A9FED780A84ED030AFB
:4002C0009FED740A84ED040A44E0012D14D19FED6D0A84ED000A9FED6C0A84ED010A9FED6B0A84ED020A9FED6C0A84ED030A9FED6C0A84ED040A2DE00B2D17D126F0ACFFD5
:40030000A0B19FED600A84ED000A9FED5F0A84ED010A9FED5E0A84ED020A9FED5F0A84ED030A9FED600A84ED040A13E09FED550A84ED000A9FED540A84ED010A9FED530A89
:4003400084ED020A9FED540A84ED030A9FED540A84ED040A70BD70B52DED028B04465248FFF752FF5048FFF7D4FE4F48FEF7C7FF4D48D0ED550AB0EE600A204610F02FF912
:400380004948D0ED550AB0EE600A204610F0A6FA4548D0ED590AB0EE600A204610F07DF94148D0ED590AB0EE600A204610F0BAFA3D4890ED000AFFEE000A20EE200AB0EE4D
:4003C000408A90ED5A0AD0ED530A30EE600AD0ED5C0A70EEC80A80EE801A80ED7E1AD0ED7E0A90ED531AB0EE480A00EEC10A80ED7F0A90ED000AB0EE408A90ED5B0AD0EDF4
:40040000560A30EE600AD0ED5D0A70EEC80A80EE801A80ED801AD0ED800A90ED561AB0EE480A00EEC10A80ED810A90ED040AD0ED7E0A80EE201AB0EE418A9FED0D0A28EE02
:40044000000AB0EE408A9FED190AB4EEC08AF1EE10FA2DDD9FED150AB0EE408A33E00000000000000000F03F281100200000C8C20000C84200000000000000008800002092
:400480001821002035FA0E3DC2B8323E00000000C2B8B23E8FDAA53B920A063F7CD9A03E88C3643B35FA0E3C1813002000007F43B7EE000AB4EEC08AF1EE10FA03D2B7EE4A
:4004C000000AB0EE408AB6EE000A38EE000ABCEEC00A10EE100AC5B2214628460FF05FFF2146284610F042FAFE4890ED040AD0ED800A80EE201AB0EE418A1FED230A28EEEE
:40050000000AB0EE408A1FED170AB4EEC08AF1EE10FA04DD1FED1B0AB0EE408A0AE0B7EE000AB4EEC08AF1EE10FA03D2B7EE000AB0EE408AB6EE000A38EE000ABCEEC00A21
:4005400010EE100AC5B2214628460FF05BFF2146284610F029FABDEC028B70BD2DE9F04F2DED088BC5B005468A4600241FED390AB0EE408A1FED3B0AF0EE408A1FED3D0AAA
:40058000B0EE409A1FED3F0AF0EE409A032101A816F091FEBAF1000F0DD1DFF84C8308F12C0905F1400605F16C0708F11C0B08F14800449024E0BAF1010F0FD1DFF82883ED
:4005C00008F1580808F12C0905F1980605F1C40708F11C0B08F14800449011E0BAF1020F0ED1DFF8048308F1B00808F12C0905F1F00605F58E7708F11C0B08F14800449001
:400600001FED5E0A86ED000A1FED600A87ED000A1FED620A85ED050A032201A9584616F05EFE032101A816F0BCFEF0EE409A032201A9449816F053FE032101A816F0B1FE44
:40064000B0EE409AB6EE080A29EE80AABEEE000A69EE80AAB6EE080A29EE00BABEEE000A69EE00BA012476E000EE104AB8EE400AF2EE040A20EE200A05F1140000EB840034
:4006800080ED000A601E08EB800090ED000AB5EEC00AF1EE10FA06DD1FED840A06EB840080ED000A08E0601E08EB800090ED000A06EB840080ED000A601E09EB800090EDD1
:4006C000000AB5EEC00AF1EE10FA06D21FED910A07EB840080ED000A08E0601E09EB800090ED000A07EB840080ED000A06EB840090ED000A601E06EB8000D0ED000A30EE10
:40070000600AB0EE408A07EB840090ED000A601E07EB8000D0ED000A30EE600AF0EE408AB4EECA8AF1EE10FA0ED3B4EEEA8AF1EE10FA09DCF4EECB8AF1EE10FA04DCF4EE7D
:40074000EB8AF1EE10FA04D223206749283981F8DA01601CC4B20B2C86DB45B0BDEC088BBDE8F08F10B500215E48FFF7F7FE10BD10B52DED028B5D4890F828400E2C34D239
:40078000DFE804F0330B080712333333191A1B220A0900BF00BF00BF00BF9FED550A5248283880ED500A27E09FED520A4E48283880ED500A20E000BF00BF9FED4D0A4A48BC
:4007C000283880ED500A17E026F02EFD30B1B3EE040A4548283880ED500A05E09FED450A4148283880ED500A06E01FEDD80A3E48283880ED500A00BF00BF08F0C7FB70B10C
:40080000FAF7D2FFB0EE408AFAF754FF00EE100AB8EE400AB4EEC08AF1EE10FA10DC08F0A6FB30B1FAF7D6FDB5EEC00AF1EE10FA06DC15F0F9FEB5EEC00AF1EE10FA09DDE3
:400840002948283890ED500AFFEE000A20EE200A80ED500ABDEC028B10BD73B52DED020B04460D460A2C21D200BF05EB85022249096801F5177101EBC20101EB84000422ED
:4008800069460AF001FE50B99DED000A05EB85011A4800EBC10000EB840080ED000A00BF1748C16B0220DFF85CC000DF7FBD10B5FAF749FB10BD73B52DED020B04460D465C
:4008C0000A2C34D200BF05EB85020B49096801F59A7101EBC20101EB8400042269460AF0D3FD11E018130020501100201821002000008C4200004842F003002074230020CA
:40090000604200208923040850B99DED000A05EB8501F84800EBC10000EB840080ED000A00BFF548C16B0220DFF8D0C300DF7FBD73B52DED020B04460D460A2C22D200BFB4
:4009400005EB8502EE49096801F5037101EBC20101EB8400042269460AF096FD58B99DED000A05EB8501E348D83000EBC10000EB840080ED000A00BFDF48C16B0220DFF882
:400980007CC300DF7FBD10B5FAF7DDFA10BD73B52DED020B04460D460A2C21D200BF05EB8502D7490968E43101EBC20101EB8400042269460AF068FD58B99DED000A05EBAA
:4009C0008501CC48503800EBC10000EB840080ED000A00BFC848C16B0220DFF820C300DF7FBD70B50446C74890F828500E2D27D2DFE805F0260B0807112626262626261797
:400A00000A0900BF00BF00BF00BF1FED470ABE4880ED500A1AE01FED490ABB4880ED500A14E026F001FC28B19FEDB80AB64880ED500A04E01FED520AB34880ED500A05E074
:400A40009FEDB20AB04880ED500A00BF00BF032C08D1AD4890ED500AFFEE000A20EE200A80ED500A70BDA74A92F82810062905D19FEDA70AA44A82ED500A0CE0042905D15F
:400A80001FED640AA04A82ED500A04E01FED680A9D4A82ED500A062808D19B4A92ED500AFFEE000A20EE200A82ED500A7047B5EEC00AF1EE10FA01D2012070470020FCE77F
:400AC000B5EEC00AF1EE10FA01DD012070470020FCE72DE9F04106460C4615464FF00408884890F828702868A8B928F072FF2860002088490870884890ED000A15F0DFFEC8
:400B000020B1BFEE000A854880ED000A15F08CFD834880ED000A0E2F37D2DFE807F0360B0807153636363636361F0A0900BF00BF00BF00BF794890ED000A5FED930A20EEFF
:400B4000200A84ED000A2AE0744890ED000A5FED970A20EE200A84ED000A20E026F064FB48B16E4890ED000ADFED680A20EE200A84ED000A08E0694890ED000A5FEDA40A2D
:400B800020EE200A84ED000A09E0644890ED000ADFED5E0A20EE200A84ED000A00BF00BF41F28831286828F01AFF28B1212030704FF00108002599E040F6C411286828F001
:400BC0000EFFF0B153480078D8B9564890ED000A15F075FE28B9534890ED000A15F0E7FD78B101204B4908704C4890ED000AFFEE000A20EE200A80ED000A28F0EAFE28607B
:400C000074E0D4ED000AB0EE600AFFF759FF68B115F00AFD4248D0ED000A30EE600ADFED420AB4EEE00AF1EE10FA14DCD4ED000AB0EE600AFFF73BFFB0B115F0F5FC3848EA
:400C4000D0ED000A30EE600ADFED380AB4EEE00AF1EE10FA08D24FF003089FED2C0A84ED000A0020286041E0D4ED000AB0EE600AFFF726FF68B115F0D7FC2948D0ED000A61
:400C800030EE600ADFED290AB4EEE00AF1EE10FA14D3D4ED000AB0EE600AFFF708FF28B315F0C2FC1E48D0ED000A30EE600ADFED1E0AB4EEE00AF1EE10FA17DD114890F8F0
:400CC0009C0018B90120F9F75EFB07E00D4890F89C00012802D10020F9F755FB4FF003089FED0A0A84ED000A002028604046BDE8F08100004C2200206042002089230408B0
:400D0000F003002018210020281100200000000000002042820300207C030020840300208803002074030020C2B8B23DC2B8B2BD70B52DED048B0425FE4890F8DC010A2839
:400D40007DD2DFE800F00506EF477CEE487CEDEC00BFF84890F8DD0120B1102821D0112835D110E01120F34981F8DD0115F05CFCF04880ED080AB6EE000A80ED500A00202A
:400D8000EC49086024E0EB4A02F5A07101F19A00FFF79FFE032803D11020E64981F8DD0116E00620E34981F8DC01022081F8DD010A2081F8E3010020086015F035FCDD4800
:400DC00080ED080AB6EE000A80ED500A00E000BF00BF0AE300BFD74890F8DD01801E0B287BD2DFE800F0067AA0FC60C87A7A7A7A7B00D048006870B928F0EBFDCD490860CD
:400E0000084690F8E1010A2805DD084690F8E101C01F81F8E101C74991F8DC01FFF723FEC44908684FF47A6128F0D9FDB0B115F0FBFBC048D0ED080A30EEC00A00E0F4E30C
:400E4000B0EEC00ADFEDBC0AB4EEE00AF1EE10FA04D22120B74981F8DA0123E0B74890ED000A15F02CFD20B1B24890F8DC0103280AD0B24890ED000A15F099FC90B1AD485B
:400E800090F8DC0106280DD1B6EE000AA94880ED500A0620A74981F8DD010C2081F8DF0100200860A0E2B6EE000AA24880ED500A006818B928F08DFD9E4908609D49086880
:400EC000C82128F08CFD38B19A4890F8DF01994981F8DD010020086086E284E2954991F8DC01FFF77EFD9348006818B928F071FD904908608F490868C82128F070FD68B147
:400F0000B6EE000A8B4880ED500A0620894981F8DD0100200860042081F8DF0164E2FDE3FDE363E263E215F07FFBF0EE409A4FF6FF71834816F025FB7E48006818B928F091
:400F400048FD7C4908607B4908684FF4FA7128F046FD78B1774890ED680A80ED080A0720744981F8DD010020086001F5C07000210162416238E26F48006818B928F029FD14
:400F80006C4908606B4890F8E30100EB8000400000EE100AB8EEC00A664880ED500A90F8DC01032808D1634890ED500AFFEE000A20EE200A80ED500A604890ED000A15F048
:400FC0007EFC20B15B4890F8DC0106280CD05B4890ED000A15F0EBFBC0B1564800E030E090F8DC01032811D10220524981F8DD0101F5C07000210162416215F015FB4D4803
:4010000080ED080A00204B49086019E0494908684FF4FA7128F0E3FC90B1B6EE000A454880ED500A0620434981F8DD01086828F0F8FC4049C86100200860052081F8DF01F5
:40104000D2E115F0F1FAF0EE409A4FF6FF713C4816F097FA3748006818B928F0BAFC35490860344908684FF4FA7128F0B8FC00285FD0304890ED680AD0ED080A30EE608ADD
:40108000B0EEC80AF0EE409A15F091FB20B1294890F8DC01032821D0284890ED000A15F086FB20B1234890F8DC01032816D0B0EEC80AF0EE409A15F002FC20B11D4890F89C
:4010C000DC0106280AD01D4890ED000A15F0F7FB98B1184890F8DC0106280ED10220154981F8DD01084690ED680A80ED080A00F5C0700021016241620DE007200D4981F84B
:40110000DD01084690ED680A80ED080A00F5C070002101624162074890F8E301401E054981F8E301084690F8DC01032862D1084608E057E12811002035FA0E3D740300201C
:40114000C812002090ED070AF8EE400A9FEDFE1A80EE810AC8EE000A90F8E311283000EB8100C0ED000AF94A92F84210F84A92F8E30192F8E331283202EB8302D2ED000A61
:40118000B0EE600AFFF703FCF14890F8E311283000EB8100D0ED000AB0EE600A0020FDF762FEFFF7F0FBEA4890F8E311803000EB810080ED000AE54A92F84210E44A92F891
:4011C000E30192F8E331803202EB8302D2ED000AB0EE600AFFF7ACFBDD4890F8E311803000EB8100D0ED000AB0EE600A0020FDF7EFFD57E0D64890ED070AF8EE400A9FEDB0
:40120000D21A80EE810AC8EE000A90F8E311543000EB8100C0ED000ACC4A92F84210CC4A92F8E30192F8E331543202EB8302D2ED000AB0EE600AFFF73EFBC54890F8E31151
:40124000543000EB8100D0ED000AB0EE600A0020FDF7E4FDFFF72BFBBD4890F8E311AC3000EB810080ED000AB84A92F84210B84A92F8E30192F8E331AC3202EB8302D2ED63
:40128000000AB0EE600AFFF7E8FAB14890F8E311AC3000EB8100D0ED000AB0EE600A0020FDF796FDAA4890F8E301002813D1A84890F8DC0106280FD10320A54981F8DC01DD
:4012C000022081F8DD01B6EE000A084680ED500A0A2081F8E30182E0B7EE000A9C4880ED4E0A09209B49087026E099485430994991F9001000EB810090ED000A5FED720A4A
:40130000B4EEE00AF1EE10FA10D2924890F9000000EE100AB8EEC00AF2EE040A20EE200A8B4880ED4E0AFF208A49087089480078401E40B287490870864890F900000028F3
:40134000D3DAB7EE000A824880ED4D0A09208149087026E07E4828307E4991F9001000EB810090ED000ADFED7C0AB4EEE00AF1EE10FA10DD774890F9000000EE100AB8EEF6
:40138000C00AFAEE040A20EE200A714880ED4D0AFF20704908706F480078401E40B26D4908706C4890F900000028D3DA684890ED4E0A80ED4F0A0520654981F8DC010D2008
:4013C00081F8DD01B6EE000A084680ED500A002081F8E3019FED610A084680ED4C0A00205B49086000E000BF00BFD9E100BF584890F8DD0106281DD00D2802D00E287DD19F
:4014000032E0FFF7B5F9564890ED000A15F0FFF978B1B6EE000A4E4880ED500A06204C4981F8DD010E2081F8DF0128F0D2FA484908608EE1B6EE000A454880ED500A014672
:4014400008684FF4FA7128F0CAFA60B1404890F8DF013F4981F8DD010020086015F0E4F83B4880ED080A74E1394890F8DC01052807D115F0D9F83648D0ED080A70EE608A7C
:4014800006E015F0D1F83248D0ED080A70EEC08A2F48006860B928F09CFA2D49086008460068C1F8E4019FED2D0A084680ED7A0A264890F8430001282FD128F08AFA244942
:4014C000D1F8E411441A224890ED7A0A30EE280A80ED7A0AB4F57A7F1AD3D0ED7A0A00EE104AB8EE400A80EE801AF0EE418A9FED1B0A80ED7A0A28F06CFA00E028E1144905
:40150000C1F8E40115F090F8114880ED080A03E09FED120AF0EE408A00BF0C4890ED6E0AB4EEE80AF1EE10FA7ED2094890ED4C0AD0ED500A30EE200A80ED4C0A90F8E301EE
:40154000401C03490EE0000000007A4418210020281100208103002035FA0EBD000000007803002081F8E301B6EE000A084680ED500A0D2081F8DD01086828F052FA00EEC6
:40158000100AB8EE400A5FED100A80EE209AFE4890F8DC01052816D1FB4890ED4F0A30EE090AF1EE040A30EE600A80ED4F0A90ED4F0AB5EEC00AF1EE10FA1AD21FED190A08
:4015C00080ED4F0A15E0F04890ED4F0A30EE490AF1EE040A30EE200A80ED4F0A90ED4F0AB5EEC00AF1EE10FA03DD1FED240A80ED4F0AE54890F8E30103283ADBE248D0EDEA
:401600004C0A90F8E30100EE100AB8EE400A80EE801ADD4880ED4C1A90F8DC01052829D1DA4991F8420001E03FE0B8E0D649D1ED4C0AB0EE600A0FF02DF91FED380AD24816
:4016400080ED4C0AB6EE000A80ED500A0020CE4981F8E301022081F8DC010D2081F8DD0128F0B7F9C8490860084690ED4D0A80ED4F0A6CE0C54991F84200C349D1ED4C0A34
:40168000B0EE600A0FF0E2F81FED4C0ABE4880ED4C0AB6EE000A80ED500A0820BA4981F8DC010F2081F8DD0151E0B74890ED500AB0EEC00ADFEDB60AB4EEE00AF1EE10FA32
:4016C00007DA0146086828F0ACF94EF66021884207D92120AC4981F8DA01092081F8DC0135E0A94890F8DC01022819D1A649086828F097F900EE100AB8EE400AFFEE000AA8
:4017000020EE200A1FED701AC0EE010A9E4890ED4F0A30EE800A80ED500A18E01BE021E09949086828F07DF900EE100AB8EE400AF7EE000A20EE200A1FED7D1AC0EE010AA8
:40174000914890ED4F0A30EE800A80ED500A00E000BF00BF24E002251FED800A8A4880ED500A1DE0FEF7FEFF874890F8DA0120B10920854981F8DC0110E0844991F84200CC
:40178000FEF7E9FD1020804981F8DD0103251FED8D0A084680ED500AFDF79BFD00E000BF00BF794890F8DE01774991F8DD11884214D0754890F8E101401C734981F8E1018D
:4017C000084690F8E101642802DD642081F8E1016D4890F8DD016C4981F8DE016A4890ED500AB5EEC00AF1EE10FA08D0D0ED500AB0EE600A01210846F8F765FE08E0624895
:40180000D0ED500AB0EE600A00210120F8F75BFE2846BDEC048B70BD2DE9F0412DED048B042607F0B3FB10B1B3EE090A01E0B1EE040AB0EE409A07F0A9FB08B1554800E021
:401840005548044607F0A2FB08B1544800E0544807464D4890F8DC010A2872D2DFE800F00506D77171D67171F9F800BF464890F8DD0120B110287DD011280ED000BF11202B
:40188000414981F8DD01B6EE000A084680ED500A28F09FF83C490860B6E03B49086828F0C0F8B0F5FA7F04D2A047374880ED090A89E03549086828F0B4F840F6B8318842B0
:4018C00005D29FED380A304880ED500A7BE02E49086828F0A6F840F6AC51884217D2B6EE000A294880ED500AA0472748D0ED090A30EE600AB4EEC90AF1EE10FA63DD1E20B6
:40190000214981F8DA01092081F8DC015BE01E49086828F086F8B0F57A6F04D2A0471A4880ED090A4FE01849086828F07AF841F66411884206D29FED160A134880ED500AEF
:4019400041E059E21049086828F06BF841F6583188422CD2B6EE000A0B4880ED500AA0470948D0ED090A30EE600AF1EE490AB4EEE00A00E028E0F1EE10FA24D21E200249D9
:4019800081F8DA0109200FE0281100201821002000008C42A9B70008D5B30008B5B90008F7B3000800008CC281F8DC010BE0B6EE000AFE4880ED500A28F00BF8FB4908600A
:4019C000102081F8DD011FE00520F84981F8DC010D2081F8DD01B6EE000A084680ED500A002081F8E30127F0F4FFF04908609FEDF00A084680ED4C0A9FEDED0A80ED4F0A56
:401A0000002081F8E10100BF00BFF6E100BFE74890F8DD0106282DD00D2802D00E287CD141E0FEF7A5FEB0EE000AB84790B1B6EE000ADE4880ED500A0620DC4981F8DD01EF
:401A40000E2081F8DF0127F0C4FFD849086010E068E16EE1D549086827F0E3FF44F62061884206D92120D14981F8DA01092081F8DC0155E1B6EE000ACC4880ED500A0146D5
:401A800008684FF4FA7127F0AAFF58B1C74890F8DF01C64981F8DD0100200860A047C34880ED090A3CE1C14890F8DC01052806D1A047BE48D0ED090A70EE608A05E0A04708
:401AC000BA48D0ED090A70EEC08AB848006818B927F07FFFB5490860F4EEC98AF1EE10FA7EDDB24890F8E301002808DDAF4890ED4C0AD0ED500A30EE200A80ED4C0AAB486D
:401B000090F8E301401CA94981F8E301B6EE000A084680ED500A0D2000E000E181F8DD01086827F07EFF00EE100AB8EE400ADFEDA10A80EE208A9D4890F8E301012804D1AC
:401B4000B1EE040A28EE000A03E0B6EE000A28EE000AB0EE408A27F03CFF94490860084690F8DC01052816D1084690ED4F0A30EE080AF2EE040A30EE600A80ED4F0A90ED14
:401B80004F0AB5EEC00AF1EE10FA1AD29FED880A80ED4F0A15E0854890ED4F0A30EE480AF2EE040A30EE200A80ED4F0A90ED4F0AB5EEC00AF1EE10FA03DD9FED7D0A80ED16
:401BC0004F0A7A4890F8E30103283DDD7748D0ED4C0A90F8E30100EE100AB8EE400A00E04EE0B7EE001A30EE410A80EE801A6F4880ED4C1A90F8DC01052826D16E4991F852
:401C000042006A49D1ED4C0AB0EE600A0EF042FE9FED670A654880ED4C0AB6EE000A80ED500A0020614981F8E301022081F8DC010D2081F8DD0127F0CCFE5C4908609FEDD6
:401C40005C0A084680ED4F0A68E05B4991F842005649D1ED4C0AB0EE600A0EF0F7FD9FED540A524880ED4C0AB6EE000A80ED500A08204E4981F8DC010F2081F8DD014DE002
:401C80004A4890ED500AB0EEC00ADFED4C0AB4EEE00AF1EE10FA07DA0146086827F0C1FE4EF66021884207D92120404981F8DA01092081F8DC0131E03C4890F8E30110B978
:401CC000B1EE040A01E0B6EE000AF0EE409A3749086827F0A6FE00EE100AB8EE400A20EE290ADFED340A80EE201A304880ED501A90F8DC01022808D12C4890ED500AFFEE6B
:401D0000000A20EE200A80ED500A284890ED500AD0ED4F0A30EE200A80ED500A00E000BF00BF6AE002269FED220A204880ED500A63E01E4890F8DA0120B109201B4981F894
:401D4000DC0158E06425A8461B4991F84200694200EE101AB8EEC00A0EF041FC164991F84200694200EE101AB8EEC00A0EF0B6FD114991F8420000EE105AB8EE400A0EF0C1
:401D80008CFC0D4991F8420000EE105AB8EE400A0EF0C8FD084890F8421040460EF0FFFA054890F8421040460AE00000281100200000000000007A44182100200000A042DF
:401DC0000EF0D4FDFE4890F8421040460EF01AFBFB4890F8421040460EF0E6FD1020F94981F8DD0103261FED0E0A084680ED500AFDF76FFA00BF00E000BF00BFF14890F871
:401E0000DE01F04991F8DD11884214D0ED4890F8E101001DEB4981F8E101084690F8E101642802DD642081F8E101E64890F8DD01E44981F8DE01E34890ED500AB5EEC00A90
:401E4000F1EE10FA08D0D0ED500AB0EE600A01210846F8F738FB08E0DA48D0ED500AB0EE600A00210120F8F72EFB3046BDEC048BBDE8F081002070471FED330AD14880ED03
:401E8000720A1FED350A80ED740A1FED370A80ED6C0A1FED390A80ED6A0A1FED3B0A80ED700A1FED3D0A80ED6E0A704770B52DED048B0446F0EE408AB0EE609AF0EE419AD8
:401EC0000D46BF4890F83000702804D0BC4890F8300093280CD1F7EE000A80EEA80A5FED4B0A89EE201A20EE010A20EE298A6AE0B34890F83000912809D0B14890F8300095
:401F0000922804D0AE4890F8300071280CD1F0EE000A80EEA80A5FED590A89EE201A20EE010A20EE298A4EE0A81E0C283DD2DFE800F02D3C063C13203C3C3C3C2F2EF0EEB6
:401F4000080A80EEA80A5FED650A89EE201A20EE010A20EE298A35E0DFED9B0A80EEA80A5FED6C0A89EE201A20EE010A20EE298A28E0DFED960A80EEA80A5FED720A89EE23
:401F8000201A20EE010A20EE298A1BE000BF00BFDFED8F0A80EEA80A5FED7A0A89EE201A20EE010A20EE298A0CE0DFED8A0A80EEA80A5FED800A89EE201A20EE010A20EE9A
:401FC000298A00BF00BFB2EE040AB4EEC08AF1EE10FA04D2B2EE040AB0EE408A0AE09FED7E0AB4EEC08AF1EE10FA03DD9FED7A0AB0EE408A012C0AD1714A92F84210BCEECD
:40200000C80A10EE102AD0B20EF0B0FC09E06C4A92F84210BCEEC80A10EE102AD0B20EF0C3FCBDEC048B70BD00B52DED028B95B0644890ED500A8DED140A27F0CAFC0E9060
:4020400004200C9014F096FA5E4880ED520AC0685C4948610846006988616048007829F05EFC5849C86027F0B4FC56490861084680690B9027F0D5FC4FF47A71B1FBF0F0E8
:402080000F905048C0684F494969401A00EE100AB8EEC00AF7EE000A20EE200A9FED501AC0EE010A9DED0F0AB8EEC00A20EE800A8DED130A05214B489DED130A15F061FACD
:4020C0000521484808309DED140A15F05AFA1EF08BFA8DED0B0A1E21424818389DED0B0A15F04FFA404890ED000A8DED0B0A1E213C4820389DED0B0A15F043FA3A4890ED30
:40210000000A304880ED510A3848007810F042FA8DED0B0A0521334808389DED0B0A15F030FA3348007810F0F2FB8DED050A059831F010FECDE906019DED060B2EF0E4F95B
:402140008DED080B9DED080B51EC100B30F0C6FF05210B90234810389DED0B0A15F011FA1748B0F8BE014FF4967190FBF1F000EE100AB8EEC00A8DED0D0A114890F8280047
:4021800006284ED00E4890F82800072849D00D4890F8DC01042804D00A4890F8DC0107283FD1084890ED740ADFED120AB4EEE00AF1EE10FA36DD90ED721A9DED0D0A1BE075
:4021C0001821002028110020CDCC4C406666A6408FC2753E9A99193F00007F435407002052EC2F45F0120020804500200F0700206007002000004842F2EE040AF1EE041A9F
:4022000041EEC00AB4EEE01AF1EE10FA79D20920FE4981F8DC01242081F8DA01002081F8DD016EE0F94890ED740ADFEDF90AB4EEE00AF1EE10FA19D290ED721A9DED0D0A9D
:40224000FAEE040AF1EE041A41EE800AB4EEE01AF1EE10FA55DD0920EC4981F8DC01242081F8DA01002081F8DD014AE0E748D0F8D001079031F06EFDCDE908019DED080BC7
:402280002EF042F98DED0A0B9FEDE20B53EC102B9DED0A0B51EC100B31F066F931D1DDED0D0AB1EE040AB1EE041A01EE200A8DED070A079831F04EFDCDE90A01D348D0F82C
:4022C000C801059031F046FDCDE906019DED060B2EF01AF98DED080B9DED0A0B53EC102B9DED080B51EC100B31F03CFB09D20920C64981F8DC01242081F8DA01002081F806
:40230000DD01C24890F8DD01062813D1BF48806801460B900E9827F093FBBC494968884241F2D483B94890F8DF01B84981F8DD0101F0CCBBB54890F8DC010A2881F0C48392
:40234000DFE810F030000A0040004F04C20B49022C07C20BB80BA30BAC4890F8DB0180B1AA4890F8DB01A94981F8DC01062081F8DD01002081F8DF01192048600E988860B4
:402380000EE00020A14981F8DC01062081F8DD01002081F8DF014FF47A7048600E98886001F093BB0220994981F8DC01062081F8DD01002081F8DF014FF47A7048600E986C
:4023C0008860EDE7914890F8DC01904981F8DB01084690F8DD0108287ED003DC38B105287BD165E1092879D00B28F9D10BE00620864981F8DD010B2081F8DF0119204860E9
:402400000E988860E5E18148806801460B900E9827F016FB41F28831884207D909207B4981F8DC01262081F8DA0170E07B4890F8280006280ED0794890F82800072809D02C
:40244000724890ED520ADFED760AB4EEE00AF1EE10FA13DC714890F82800062804D06F4890F8280007280FD1684890ED520ADFED6D0AB4EEE00AF1EE10FA05DDBBEE0E0A54
:40248000624880ED500A42E0644890F8280006280ED0624890F82800072809D05B4890ED520ADFED610AB4EEE00AF1EE10FA17D35A4890F82800062804D0584890F8280009
:4024C000072813D1514890ED520ADFED580AB4EEE00AF1EE10FA02E032E073E118E005D2B3EE0E0A494880ED500A10E00620474981F8DD01092081F8DF014FF47A70486038
:402500000E9888609FED4A0A084680ED500A60E106203E4981F8DD01082081F8DF01192048600E988860BAEE000A084680ED500A4048007829F0F3F93449C1F8880148E12F
:40254000364890F82800062804D0344890F82800072810D12D48C0682C49D1F88811401A00EE100AB8EEC00ADFED330AB4EEE00AF1EE10FA3BD3294890F8300091280AD061
:40258000264890F83000922805D0244890F83000712800D010E01D48C0681C49D1F88811401A00EE100AB8EEC00ADFED240AB4EEE00AF1EE10FA1AD3184890F82800062829
:4025C00052D0164890F8280007284DD00F48C0680E49D1F88811401A00EE100AB8EEC00ADFED150AB4EEE00AF1EE10FA3CD20B4890F842000B909DED140A0EF027F9062043
:40260000024981F8DD0105201AE0000028110020000048C2000000000000204018210020CDCCCC3CCDCC4C3DCDCCCCBCCDCC4CBD00000000540700206CE7DBC57390EAC418
:4026400081F8DF014FF47A7048600E9888609DED140A084680ED500AFA48007829F05FF9F949C1F8880122E0F74890ED500A5FED180AB4EEE00AF1EE10FA0BD81FED140A2A
:4026800080ED500A0920F04981F8DC01272081F8DA010CE09DED140ADFEDEC0A30EE600A8DED140A9DED140AE74880ED500A90E0E548D0ED500A9FEDE61A80EE810A8DED39
:4026C000010A019831F046FBCDE902019DED020B2DF01AFF8DED060BDB48D0F8C001039031F038FBCDE904019DED060B53EC102B9DED040B51EC100B31F036F89FEDD50BB4
:4027000053EC102BCDE908019DED080B51EC100B30F0D2FDCDE90A019DED0A0B51EC100B30F0DCFCC849C1F85801084690ED6E0ADFEDCA0A80EE201A80ED5A1AC84890F8A5
:402740003000912809D0C64890F83000922804D0C34890F83000712804D1B3EE090A8DED100A03E0B1EE040A8DED100A9DED100ADFEDBC0A80EE201A9FEDBB0A21EE000A5E
:40278000BDEEC00AB8EEC00AAF4880ED5E0AB0F8D80140F00400AC49A1F8D801052081F8DC01062081F8DD01002081F8DF014FF47A7048600E9888601FED630A084680ED44
:4027C000500A06E00020A049A1F8D80181F8DC0100BF00BFE4E59C4890F8DC019A4981F8DB01084690F8DD0108287CD003DC38B1052879D162E1092877D00B28F9D10BE0EE
:402800000620914981F8DD010B2081F8DF01192048600E988860E2E18B48806801460B900E9827F00DF941F28831884207D90920854981F8DC01282081F8DA0170E088488C
:4028400090F8280006280ED0854890F82800072809D07D4890ED520A5FED8F0AB4EEE00AF1EE10FA13DC7E4890F82800062804D07B4890F8280007280FD1734890ED520AA2
:402880005FED980AB4EEE00AF1EE10FA05DDBBEE0E0A6D4880ED500A42E0714890F8280006280ED06E4890F82800072809D0664890ED520A5FEDA40AB4EEE00AF1EE10FA9B
:4028C00017D3674890F82800062804D0644890F82800072813D15C4890ED520A5FEDAD0AB4EEE00A02E034E072E11AE0F1EE10FA05D2B3EE0E0A544880ED500A10E00620DD
:40290000514981F8DD01092081F8DF014FF47A7048600E9888601FEDBA0A084680ED500A5DE10620484981F8DD01082081F8DF01192048600E988860B2EE000A084680ED3B
:40294000500A4048007828F0EAFF3F49C1F8880145E1434890F82800062804D0404890F82800072810D13848C0683749D1F88811401A00EE100AB8EEC00ADFED3C0AB4EE77
:40298000E00AF1EE10FA3BDC354890F8300091280AD0334890F83000922805D0304890F83000712800D010E02748C0682649D1F88811401A00EE100AB8EEC00ADFED2C0ADE
:4029C000B4EEE00AF1EE10FA1ADC254890F8280006284FD0224890F8280007284AD01A48C0681949D1F88811401A00EE100AB8EEC00ADFED1E0AB4EEE00AF1EE10FA39DD00
:402A0000174890F842000B909DED140A0DF042FF06200D4981F8DD01052081F8DF014FF47A7048600E9888609DED140A084680ED500A0448007828F072FF0349C1F88801A0
:402A40003BE000005407002028110020CDCCCC3D0000C8420000000000408F4000007A4418210020000070428DED24486CE7DB457390EA44F74890ED500ADFEDF70AB4EED4
:402A8000E00AF1EE10FA0BDB9FEDF40A80ED500A0920F04981F8DC01292081F8DA010CE09DED140A5FED170A30EE200A8DED140A9DED140AE74880ED500A90E0E548D0EDDE
:402AC000500A1FED1D1A80EE810A8DED010A019831F040F9CDE902019DED020B2DF014FD8DED060BDB48D0F8C001039031F032F9CDE904019DED060B53EC102B9DED040BCB
:402B000051EC100B30F030FE1FED2E0B53EC102BCDE908019DED080B51EC100B30F0CCFBCDE90A019DED0A0B51EC100B30F0D6FAC849C1F86001084690ED6E0A5FED390AF0
:402B400080EE201A80ED5C1AC54890F83000912809D0C34890F83000922804D0C04890F83000712804D1B3EE090A8DED100A03E0B1EE040A8DED100A9DED100A5FED470A47
:402B800080EE201A1FED480A21EE000ABDEEC00AB8EEC00AAF4880ED600AB0F8D80140F02000AC49A1F8D801032081F8DC01062081F8DD01002081F8DF014FF47A704860C7
:402BC0000E9888609FEDA50A084680ED500A06E00020A049A1F8D80181F8DC0100BF00BFF8E59C4890F8DC019A4981F8DB01084690F8DD0130B105287ED007287DD00A28A6
:402C00007CD10BE00620934981F8DD010A2081F8DF01192048600E988860BDE28D48806801460B900E9826F00BFF42F21071884207D90920874981F8DC01262081F8DA01C5
:402C4000BCE0874890F8280006280ED0844890F82800072809D07F4890ED520A5FED850AB4EEE00AF1EE10FA13DC7D4890F82800062804D07A4890F8280007282AD17548FA
:402C800090ED520ADFED770AB4EEE00AF1EE10FA20DD734890F82800062804D0704890F8280007280BD100BF6D4890ED300AF0EE040A30EE600A674880ED500A7EE0684879
:402CC00090ED300AF2EE0E0A30EE600A614880ED500A73E0624890F82800062812D0604890F8280007280DD05A4890ED520ADFED5E0AB4EEE00A02E061E0F0E145E2F1EED7
:402D000010FA13D3564890F82800062804D0544890F8280007282AD14E4890ED520A5FEDB50AB4EEE00AF1EE10FA20D24C4890F82800062804D04A4890F8280007280BD169
:402D400000BF474890ED320AF0EE040A30EE200A404880ED500A31E04148D0ED320AB2EE0E0A30EE800A3B4880ED500A26E00620384981F8DD01052081F8DF0140F6B830EC
:402D800048600E988860364890F8280007280AD1334890ED320ADFED350A20EE200A084680ED500A04E09FED2D0A2A4880ED500A00202849C1F88801C1F89401ECE12548DE
:402DC000D0F88801D0BB2A48007828F0A8FD2149C1F88801084690ED6A0A80ED630A90ED6C0A80ED640A062081F8DD01072081F8DF011B4890F82800072803D14FF47A707D
:402E0000486003E04FF47A701249486011490E988860134890F82800062804D0104890F8280007280BD10E4890ED300AF2EE0E0A30EE600A074880ED500A4FE11AE00848B2
:402E400090ED300ADFED040A30EE600A014880ED500A43E128110020000048420000000018210020CDCC4C3ECDCC4C3D9A99193F54070020FE48D0F8940100287ED1FD481F
:402E8000007828F04CFDFA49C1F89401084690ED6A0A80ED660A90ED6C0A80ED670AD0F89401D1F88811401A0B9014F0D5FD00EE100AF8EE400A9FEDF00A20EE800ADFED0F
:402EC000EE0A80EE201AEA4880ED5F1AD0F89411D0F88801081A00EE100AB8EEC00ADFEDE70AB4EEE00AF1EE10FA7DD2E44890F82800062804D0E24890F82800072804D185
:402F00009FEDE00A8DED130A04E0D94890ED6C0A8DED130ADA4890F82800072839D1D44890F8E0010B90D64890ED0F0A8DED0A0ACF4890ED660A8DED090A0B989DED0A1AA6
:402F4000DDED130A9DED090A12F070FBC84880ED550A90F8E0010B90C94890ED0F0A8DED0A0AC34890ED630A8DED090A0B989DED0A1ADDED130A9DED090A00E0AEE012F084
:402F800055FBBB48D0ED550A30EEC00A80ED550A38E0B74890F8E0010B90B94890ED0F0A8DED0A0AB24890ED660A8DED090A0B989DED0A1ADDED130A9DED090A12F036FB32
:402FC000AB4880ED550A90F8E0010B90AC4890ED0F0A8DED0A0AA64890ED630A8DED090A0B989DED0A1A00E06CE0DDED130A9DED090A12F01BFB9E48D0ED550A30EEC00A8E
:4030000080ED550A9A4890F8E0010B90984890ED570AB1EE400A8DED0A0A90ED550A8DED090A0B999DED0A1ADFED930A9DED090A0120FEF73BFF8E4890ED550AF7EE000AF7
:4030400080EE201A1FED7B0A31EE408A8E4800780FF0A0FADFED880A80EE201A844890ED570AB1EE400AC0EE010A854890ED300A9FED861A10EE810AC8EE000A7C48C0ED8B
:40308000530AB0F8D80140F008007949A1F8D8010846B0F8D80140F01000A1F8D801062081F8DC0181F8DD01002081F8DF014FF47A7048600E9888601FED980A084680ED2D
:4030C000500A0BE01FED9B0A694880ED500A0920674981F8DC012B2081F8DA015CE00620634981F8DD01052081F8DF010A2048600E9888600846D0ED500A9FED641A80EE74
:40310000810A8DED010A019830F024FECDE902019DED020B2DF0F8F98DED060B5448D0F8C001039030F016FECDE904019DED060B53EC102B9DED040B51EC100B30F014FBDF
:403140009FED530B53EC102BCDE908019DED080B51EC100B30F0B0F8CDE90A019DED0A0B51EC100B2FF0BAFF4149C1F85C01084690ED6E0ADFED400A80EE201A80ED5B1A5C
:40318000BAEE000A80ED500A06E000203849A1F8D80181F8DC0100BF00BFFDE3344890F8DC01334981F8DB01084690F8DD0130B105285CD0072873D00A2872D10BE0062051
:4031C0002B4981F8DD010A2081F8DF01192048600E988860FAE32648806801460B900E9826F02EFC42F21071884207D90920204981F8DC01282081F8DA01D4E0204890F890
:40320000280006280ED01E4890F82800072809D01748D0ED520A9FED200AF4EEC00AF1EE10FA13D3164890F82800062804D0144890F82800072846D10D48D0ED520A9FED37
:40324000170AF4EEC00AF1EE10FA3CD20C4890F82800062804D00A4890F82800072827D100BF074890ED320AF0EE040A1AE09BE0281100205407002000007A44FF4680C616
:403280001821002039B400400F0700200000C8420000000000408F40CDCCCCBDCDCC4CBE95E3E4E330EE200AFE4880ED500A7AE0FD4890ED320AF2EE0E0A30EE200AF94807
:4032C00080ED500A6FE0F84890F8280006280ED0F54890F82800072809D0F248D0ED520A9FEDF20AF4EEC00AF1EE10FA13DCEE4890F82800062804D0EB4890F8280007286E
:403300002AD1E84890ED520A5FED1D0AB4EEE00AF1EE10FA20DDE44890F82800062804D0E14890F8280007280BD100BFDE4890ED300AF0EE040A30EE600ADA4880ED500AE9
:4033400031E0D94890ED300AF2EE0E0A30EE600AD44880ED500A26E00620D24981F8DD01052081F8DF0140F6B83048600E988860CD4890F8280007280AD1CB4890ED300AF8
:40338000DFEDCB0A20EE200A084680ED500A04E09FEDC80AC34880ED500A0020C149C1F88801C1F894016EE3BE48D0F88801D0BBC148007828F0B3FABA49C1F88801084645
:4033C00090ED6A0A80ED630A90ED6C0A80ED640A062081F8DD01072081F8DF01B24890F82800072803D14FF47A70486003E04FF47A70AC494860AB490E988860AA4890F80C
:403400002800062804D0A84890F8280007280BD1A54890ED320AF2EE0E0A30EE200AA14880ED500AD2E20AE09F4890ED320ADFEDA30A30EE200A9B4880ED500AC6E29948EF
:40344000D0F894010028EDD19B48007828F067FA9449C1F89401084690ED6A0A80ED660A90ED6C0A80ED670AD0F89401D1F88811401A0B9014F0F0FA4FF47A71B0FBF1F0C1
:4034800000EE100AB8EE400A5FED850A20EE200A844880ED610AD0F894018249D1F88811401A00EE100AB8EEC00ADFED850AB4EEE00AF1EE10FA7DDD7B4890F82800062836
:4034C00004D0794890F82800072804D11FED930A8DED130A04E0734890ED6C0A8DED130A714890F82800072837D16E4890F8E0010B906D4890ED0F0A8DED0A0A694890EDB9
:40350000660A8DED090A0B989DED0A1ADDED130A9DED090A12F08AF8624880ED550A90F8E0010B90604890ED0F0A8DED0A0A5D4890ED630A8DED090A0B989DED0A1ADDEDB8
:40354000130A9DED090A12F071F85648D0ED550A30EEC00A80ED550A38E0524890F8E0010B90514890ED0F0A8DED0A0A4D4890ED660A8DED090A0B989DED0A1ADDED130AFE
:403580009DED090A12F052F8464880ED550A90F8E0010B90444890ED0F0A8DED0A0A414890ED630A8DED090A0B989DED0A1ADDED130A00E0FEE19DED090A12F037F83948CE
:4035C000D0ED550A30EEC00A80ED550A354890F8E0010B90334890ED590A8DED0A0A90ED550A8DED090A0B999DED0A1A5FEDDE0A9DED090A0220FEF759FC2A4890ED550A4B
:40360000F7EE000A80EE201A9FED2A0A31EE408A2C4800780EF0BEFF5FEDE90A80EE201A204890ED590AC0EE010A1F4890ED320A1FEDEA1A10EE810AC8EE000A1948C0ED34
:40364000540AB0F8D80140F040001649A1F8D8010846B0F8D80140F08000A1F8D8010846D0ED560A90ED580A30EE800A80ED560A90ED560AF0EE000A80EE201A80ED561A30
:4036800090ED570AD0ED590A30EE200A80ED570A90ED570AF0EE000A80EE201A80ED571A12E000002811002018210020CDCC4CBD9A99193F000000005407002000004842D4
:4036C000FF4680460F07002090ED5A0AD0ED5C0A30EE200A80ED5A0A90ED5A0AF0EE000A80EE201A80ED5A1A90ED5B0AD0ED5D0A30EE200A80ED5B0A90ED5B0AF0EE000A30
:4037000080EE201A80ED5B1A90ED5E0AD0ED600A30EE200A80ED5E0A90ED5E0AF0EE000A80EE201A80ED5E1A90ED5E0ADFEDF90A20EE200A80ED5E0A90ED5F0AD0ED610AAD
:4037400030EE200A80ED5F0A90ED5F0AF0EE000A80EE201A80ED5F1A90ED5F0ADFEDED0A20EE200A80ED5F0A90ED5B0AD0ED5A0A70EE600A90ED570A90ED561A30EE411A09
:4037800080EE810A8DED0B0A9DED0B0A0AF0D1F8E14890ED5B0AE148D0ED700ADE4890ED571A00EEC10A8DED0B0A9DED0B0A0AF0A6F8D94890ED5F0AD0ED5E0A70EE600A2D
:4037C00090ED570A90ED561A30EE411A80EE810A8DED0B0A9DED0B0A0AF077F8CE4890ED5F0ACE48D0ED720ACB4890ED571A00EEC10A8DED0B0A9DED0B0A0AF04CF8C84874
:4038000000780EF0C7FE9FEDC71AC0EE010AC34890ED700A20EE800AD0ED710AB2EE001A71EE600A80EE801A9FEDBF0A21EE000A8DED130A90F82800062804D19FEDBB0AC1
:403840008DED110A17E0B54890F83000912809D0B24890F83000922804D0B04890F83000712804D19FEDB10A8DED110A03E09FEDB00A8DED110AA848D0ED530A9DED110ACE
:4038800080EE201AA54890ED300A31EE400A8DED120A9DED130ADFEDA40AB4EEE00AF1EE10FA10DD9DED120ADFED9F0AB4EEE00AF1EE10FA07DD90F842009FED9E0A0B902D
:4038C0000DF00CF81DE09DED130ADDED120AB4EEE00AF1EE10FA0ADD904890F842000B909DED120AB1EE400A0CF0F8FF09E08B4890F842000B909DED130AB1EE400A0CF075
:40390000EDFF8548D0ED540A9DED110A80EE201A824890ED320A31EE000A8DED120A9DED130ADFED810AB4EEE00AF1EE10FA10DD9DED120ADFED7C0AB4EEE00AF1EE10FA57
:4039400007DD90F842009FED780A0B900CF0EAFF19E09DED130ADDED120AB4EEE00AF1EE10FA08DD6D4890F842000B909DED120A0CF0D8FF07E0694890F842000B909DED11
:40398000130A0CF0CFFF0820634981F8DC01062081F8DD01002000E097E081F8DF014FF47A7048600E9888601FEDBE0A084680ED500A0BE01FEDC10A574880ED500A09200C
:4039C000554981F8DC012B2081F8DA015BE00620514981F8DD01052081F8DF010A2048600E9888600846D0ED500A9FED4F1A80EE810A8DED030A039830F0ACF9CDE904010F
:403A00009DED040B2CF080FD8DED080B4248D0ED700A9FED441A80EE810A8DED050A059830F098F9CDE906019DED080B53EC102B9DED060B51EC100B2FF096FECDE90A0111
:403A40009DED0A0B51EC100B2FF048FB3249C1F86401084690ED6E0ADFED320A80EE201A80ED5D1AB2EE000A80ED500A0BE000202949A1F8D80181F8DC011FEDF20A084671
:403A800080ED500A00BF00BF1FE002200C900620214981F8DD01002081F8DF01192048600E9888601FEDFD0A084680ED500AFEF7E3F90AE003200C909FED1F0A164880ED13
:403AC000500AFBF706FC00E000BF00BF124890ED500AB5EEC00AF1EE10FA0AD090ED500A8DED0B0A012108469DED0B0AF6F7EBFC0AE0094890ED500A8DED0B0A002101208D
:403B00009DED0B0AF6F7DFFC0C9815B0BDEC028B00BD00005F43BA3928110020182100200F07002000007A440000C8423333B33F3333B33E0000C8C20000000010B501245A
:403B4000FB4890F8DA0170BB23F06EFB68B1F94991F8300005F0EEF918B1FDF75DFE04461FE0FEF761FA04461BE023F075FBC0B1F04890F82800072803D1FEF77BF9044680
:403B80000FE005F0F4F928B9EA4991F8300005F0D1F918B1FDF740FE044602E0FDF7C8F80446FBF71EFA204602F05FFAE04890F8DA0120B1DE4991F8DA0102F05FFF20462B
:403BC00010BD10B5DA4890F8DC010A284CD2DFE800F04C4D20054B21064B4B4E00BF0220D34981F8DD010020086012F01DFDD04880ED080A90F8E301401CCD4981F8E301C7
:403C0000084690F8E3010A2802DD0A2081F8E30130E000BF0D20C64981F8DD0125F0D9FEC34908601FED3C0A084680ED4C0A002081F8E30105F09BF970B1BD4890F8E10177
:403C4000322804DD3220BA4981F8E1010BE00020B74981F8E10106E0B54890F8E101C01EB34981F8E10105E000BF00BF00BFFBF71FF900BF00BFB048002101624162002088
:403C8000AB4981F8DA01B6EE000A084680ED500A10BD10B523F0C8FA10B302F0EBFE2B2802D1FBF705F91DE0A14890F8DB01A04981F8DC01062081F8DD01002081F8DF015F
:403CC0004FF47A70486025F084FE994988601FED660A084680ED500A002081F8DA0101E0FFF76FFF10BDB7EE000A7047904890F8DA01704710B59148FCF786FA8F48FCF744
:403D000008FA8E48FBF7FBFA10BD10B58B48FCF77BFA8A48FCF7FDF98848FBF7F0FA10BD834890F8DC017047814890F8DD01704710B504247E4890F8DC01012804D10620BA
:403D40007B4981F8DC0186E04FF4FA717C48008825F045FE00287ED025F03BFE78490880734890F8DC01801E072872D2DFE800F0450571440471700000BF6D4890F8DD01BE
:403D8000801E0B2835D2DFE800F00634151F0B1A3434343410000620654981F8DD0129E00C20634981F8DD0124E00420604981F8DD011FE007205E4981F8DD011AE0052033
:403DC0005B4981F8DD0115E0594890F8DC01062807D10320564981F8DC01022081F8DD0106E00520524981F8DC010D2081F8DD0100E000BF00BF2DE000BF4D4890F8DD0191
:403E0000062804D00D2807D00E281ED109E00D20474981F8DD0119E00E20454981F8DD0114E0434890F8DC01052809D10220404981F8DC01062081F8DD0105E00BE008E025
:403E400008203B4981F8DC0100E000BF00BF01E000E000BF00BF204610BD10B52DED088BB0EE408A05F092F818B3F7F723FC00EE100AB8EE400A38EE400A10EE104A204619
:403E80002FF068FF41EC1B0BB0EE4B0AF0EE6B0A2CF03AFBB0EE40AAF0EE60AA9FED290B53EC102B51EC1A0B2FF006FA41EC100B0BE018EE100A2FF04DFF41EC1A0BB0EEB9
:403EC0004A0AF0EE6A0A2CF01FFBB0EE409AF0EE609A51EC190B2FF001F900EE100ABDEC088B10BD01B500BF0122694617480068433007F0C9FA20B99DF800000D4981F893
:403F0000430000BF08BD10B52DED020B00BF042269460E48006800F5DC7007F0B5FA20B99DED000A034880ED6E0A00BF1CBD00002811002018210020A81200201813002089
:403F40008C0300200000000000005940F003002010B5044623F068F900287DD0092C7CD005DC4CB1032C31D0062C77D158E00B2C75D00C2CF9D1E5E00120FE490870FA2070
:403F80008861FA21FB48C16125F023FDF94948620121F84880F82810D0ED080AB0EE600AF548007827F060FD0020F24948604FF47A71F0488160416A0161002101759FEDEB
:403FC000EF0AEF48007827F04FFDF5E00120E9490870FA204860FA21E648816025F0F9FCE44908610121E3480175D0ED030AB0EE600AE348007827F037FD0020DD498861D8
:404000004FF47A71DB48C16101694162002180F828109FEDDA0AD848007827F025FDCBE00120D44908704FF47A7088610021D148C16125F0CEFCCF4948620121CD4880F8CB
:404040002810D0ED080AB0EE600ACB48007827F00BFD0020C74903E0AFE011E0ABE03AE048604FF47A71C3488160416A0161002101759FEDC20AC248007827F0F5FC9BE08C
:404080000120BC4908704FF47A7048600021B948816025F09EFCB74908610121B5480175D0ED030AB0EE600AB548007827F0DCFC0020B04988614FF47A71AE48C1610169F5
:4040C0004162002180F828109FEDAC0AAA48007827F0CAFC70E00220A6490870642048600021A448816025F074FCA24908610121A0480175D0ED030AB0EE600AA048007845
:4041000027F0B2FC64209B49886100219948C16101694162002180F828109FED980A9648007827F0A1FC0020924981F87C000121904880F87D10022180F88B10002180F871
:404140008C1039E002208B4908704FF47A70486001468848816025F03CFC86490861012184480175D0ED030AB0EE600A8448007827F07AFC4FF47A707E49886101467D48DA
:40418000C16101694162002180F828109FED7B0A7948007827F068FC0020764981F87C000121744880F87D10022180F88B10002180F88C1000E000BFDDE223F04DF800283A
:4041C000FAD0102C75D2DFE804F074083E75ABFA74E7E6E5E47474E3E2E10120654908704FF4FA70C86201466248016325F0F1FB6049886301215F4880F83C106148007895
:4042000023F054F800205B4948604FF47A7159488160816B0161002101750020554908644FF47A7153484164816BC164002180F850105348007823F039F8002152480078F2
:4042400023F034F896E201204A4908704FF4FA70086401464748416425F0BBFB4549C8640121444880F850104748007823F01EF80020404948604FF47A713E488160C16C79
:4042800001610021017500203A49C8624FF47A7138480163C16C8163002180F83C103848007823F003F800213648007822F0FEFF60E25EE201202F4908704FF4FA7048601C
:4042C00001462C48816025F084FB2A4908610121284801752A48007822F0E8FF0020254908644FF47A71234841640169C164002180F8501000201F49C8624FF47A711D48C2
:40430000016301698163002180F83C101D48007822F0CCFF00211C48007822F0C7FF29E20120144908704FF4FA70C86201461148016325F04EFB0F49886301210D4880F8EB
:404340003C101048007822F0B1FF4FF4FA700949086401460748416425F03BFB0549C8640121044880F850100748007822F09EFF002013E038160020290700200000000067
:404380002A0700208107002078070020B5E172E129E1EEE0B7E080E049E010E0F74948600021F648816025F014FBF44908610021F2480175F248007822F078FFDAE10120BA
:4043C000EE4908703220C8623221EC48016325F000FBEA4988630121E84880F83C10E948007822F063FF3220E44908643221E348416425F0EEFAE149C8640121DF4880F824
:404400005010E148007822F051FF0020DB4948600021DA48816025F0DCFAD84908610021D6480175D648007822F040FFA2E10120D24908704FF47A70C8620021CF480163CE
:4044400025F0C7FACD4988630121CC4880F83C10CC48007822F02AFF0020C84948604FF47A71C6488160816B0161002101750020C24908644FF47A71C0484164816BC16446
:40448000002180F85010BE48007822F00FFF0021BD48007822F00AFF6CE10120B74908704FF47A7008640021B448416425F091FAB249C8640121B14880F85010B24800783F
:4044C00022F0F4FE0020AD4948604FF47A71AB488160C16C0161002101750020A749C8624FF47A71A5480163C16C8163002180F83C10A348007822F0D9FE0021A148007855
:4045000022F0D4FE36E101209C4908704FF47A70486000219948816025F05BFA974908610121964801759648007822F0BFFE0020924908644FF47A71904841640169C1645B
:40454000002180F8501000208C49C8624FF47A718A48016301698163002180F83C108948007822F0A3FE00218748007822F09EFE00E10120814908704FF47A70C8620021BE
:404580007E48016325F025FA7C49886301217B4880F83C107B48007822F088FE4FF47A707649086400217548416425F012FA7349C8640121714880F850107348007822F095
:4045C00075FE00206D49486000216C48816025F000FA6A4908610021684801756848007822F064FEC6E00220644908704FF47A70486000216148816025F0EBF95F4908618F
:4046000001215E48017500215D48007822F04EFE4FF47A705949C86200215848016301698163012180F83C1000215648007822F03DFE4FF47A705149086400214F4841643A
:404640000169C164012180F8501000214E48007822F02CFE0020494981F87C000221474880F87D10032180F87E1080F88B10002180F88C107EE002204049087064204860C9
:4046800000213E48816025F0A4F93C49086101213A4801753A48007822F008FE64203749C86200213548016301698163012180F83C103448007822F0F9FD64202F490864DE
:4046C00000212E4841640169C164012180F850102D48007822F0EAFD0020284981F87C000221264880F87D10032180F87E1080F88B10002180F88C103CE001201F49087064
:404700004FF47A70486001461C48816025F061F91A49086100211948017501211948007822F0C4FD4FF47A701449C86200211348016325F04EF91149886301210F4880F8F1
:404740003C101048007822F0B1FD00200B4908644FF47A710948416425F03BF90749C8640021064880F850100748007822F09EFD00E000BF00BF0548047010BD381600207F
:404780002A07002081070020780700208E03002001B59DF8000000EE100AB8EE400AFE4880ED030A9DF8000000EE100AB8EE400AF94880ED080A00BF01226946F748006828
:4047C000403006F061FE20B99DF80000F44981F8400000BF0120F349087008BD08B506464FF4C8774FF000080121EF4880F8A8119421E9482AF02BFD307818B94620FFF7DE
:40480000C7FF11E0E64890F84050642D03DD6420FFF7BEFF08E00A2D03DA0A20FFF7B8FF02E02846FFF7B4FF0020DB4981F88D0022F0FAFCE8B10020FFF78AFBDB48DFED92
:40484000DC0A9FEDDC0A01230022DB490090DB48007826F06BFDD548DFEDD50A9FEDD50A01230022D6490090D648007826F05EFD05E022F0F1FC10B10120FFF769FB03215A
:40488000C94880F8A81100BF012239464FF6FF70DFF834C300DF25F09CF80446BE4890F88D00002874D1012017F021FB18BB22F0BBFC68B1C548007818B9BA480078012887
:4048C00005D10020FFF744FB0020B64908709EE022F0C2FC0028FAD0BC480078052803D1B04800780128F2D10520FFF731FB0020AC4908708BE001F0F5FA20BB22F094FC41
:4049000070B1B2480078092803D1A648007801287DD10920FFF71CFB0020A249087076E022F09AFC002872D0A8480078022803D19C48007801286AD10220FFF709FB00207F
:404940009849087063E022F06FFC70B19F480078062803D193480078012858D10620FFF7F7FA00208F49087051E022F075FC28B396480078042803D18A480078012846D10B
:404980000420FFF7E5FA0020864908703FE0FFE7814890F88D00012823D122F045FC70B18A4800780C2803D17E48007801282ED10C20FFF7CDFA00207A49087027E022F00E
:4049C0004BFC20B3814800780D2803D17548007801281CD10D20FFF7BBFA00207149087015E06D4890F88D00022810D122F034FC68B1764800780F2803D16A480078012825
:404A000005D10F20FFF7A4FA00206649087062480078012802D002287ED115E15E48007D28BB5D48406810B35B480169204625F007F85949896888423FD3012156480175C8
:404A4000046122F0F1FB48B15348D0ED030AB0EE600A5C48007827F007F82EE022F0FCFB10B301215748007822F020FC25E04A48007D012821D148488068A8B14648016902
:404A8000204624F0DDFF44494968884215D3002141480175046122F0C7FB30B19FED4C0A4848007826F0E0FF07E022F0D5FB20B100214448007822F0F9FB374890F82800A3
:404AC000C8B935488069B0B13348416A204624F0B7FF3149C96988422BD301212E4880F828104462D0ED080AB0EE600A3348007826F0BAFF1DE0284890F82800012818D1EE
:404B00002548C069A8B12448416A204624F098FF21498969884200E0F6E10AD300211E4880F8281044629FED2A0A2448007826F09BFF194890F85000A8B91748006C90B1CD
:404B40001548C16C204624F07BFF1349496C884245D30121104880F85010C4641D48007822F0A4FB3BE00C4890F85000012836D10948406C80B30848C16C204624F060FFBF
:404B80000549096C88422AD30021034880F85010C4641048007820E038160020F0030020182100208F0300206042002030DC00200000FA4300247449001C004029070020EB
:404BC000002000402A070020E92304088E030020000000007807002001E022F067FBD84890F83C00A8B9D648C06A90B1D448816B204624F025FFD249096B884223D3012162
:404C0000CF4880F83C108463CE48007822F04EFB19E0CB4890F83C00012814D1C848006B88B1C748816B204624F00AFFC449C96A884208D30021C24880F83C108463C148F5
:404C4000007822F033FB5FE1BD4890F88C107C30405C78BBBA48007D01282CD1B8480169204624F0EDFEB6494968884221D30021B3480175046122F0D7FA30B11FED2C0AB9
:404C8000B148007826F0F0FE0DE022F0E5FA50B11FED310AAC48007826F0E6FE0021AA48007822F003FBA6488068002801D14FF00108C1E00BE0A2480169204624F0C0FE28
:404CC0009F498968884201D34FF00108B4E09C4890F88C107C30405C01282BD1984890F8280001281AD19648416A204624F0A8FE93498969884210D30021914880F828107A
:404D000044621FED4D0A9148007826F0ADFE8C48C069002801D14FF001088DE08848416A204624F08DFE8649C969884201D34FF0010881E0824890F88C107C30405C022884
:404D400036D17F4890F83C00012825D17C48816B204624F075FE7A49C96A88426CD30021774880F83C1084637648007822F09EFA22F072FA50B100217248007822F096FA07
:404D80001FED6D0A6F48007826F06EFE6C48006B90BB4FF001084FE06948816B204624F04FFE6749096B884246D34FF0010843E0634890F88C107C30405C03283CD1604811
:404DC00090F8500001282CD15D48C16C204624F037FE5B49096C88422ED30021584880F85010C46422F020FA38B11FED870A5748007826F039FE0EE01EE022F02DFA50B153
:404E00001FED8D0A5248007826F02EFE00215048007822F04BFA4A48406C68B94FF001080AE04748C16C204624F00AFE4449496C884201D34FF00108B8F1010F63D14FF0D0
:404E400000083F4890F88C00401CC1B23C4880F88C1090F88C1090F88B00814203DB0021374880F88C10364890F88C107C30405C022809D10121324880F83C1084633148EE
:404E8000007822F013FA3EE02D4890F88C107C30405C01280DD10121294880F828104462D0ED080AB0EE600A2848007826F0DCFD29E0234890F88C107C30405C032809D1D9
:404EC00001211F4880F85010C4642148007822F0EDF918E001211A480175046122F0A4F948B11748D0ED030AB0EE600A1648007826F0BAFD07E022F0AFF920B1012112488F
:404F0000007822F0D3F900BFBEE42DE9F04106460C4617469846069D2078642803DD6420FFF736FC09E020780A2803DA0A20FFF72FFC02E02078FFF72BFCBDE8F0810000BF
:404F400038160020810700202A070020290700207807002070B543201CE0C41700EBD4646511CD4C54F82540C51700EBD5656D11A0EB45160125B5402C40C51700EBD5652C
:404F80006D11A0EB45160125B540AC4200D103E0411EC8B20028E0DC00BF70BD30B5C31700EBD3635C11BC4B183353F824300246C41700EBD4646411A0EB44150124AC4039
:404FC00023430146C41700EBD4646511B24C183444F8253030BD13B50C4600BFAF49096801F5B07108190122694606F04DFA18B99DF80010AA48015500BF1CBD13B50C46CF
:4050000000BFA649096801F25F2108190122694606F03AFA20B99DF80010A148FF30015500BF1CBD70B504469E480470E21704EBD2625311984A52F823202146E31704EB35
:40504000D3635B11A4EB43150123AB409A432046E31704EBD3635D118F4B43F82520E21704EBD26253118C4A0C3252F82320E31704EBD3635B11A4EB43150123AB409A43EF
:40508000E31704EBD3635D11834B0C3343F82520E21704EBD26253117F4A183252F82320E31704EBD3635B11A4EB43150123AB409A43E31704EBD3635D11774B183343F883
:4050C00025200020FFF79AFF70BD30B50146CB1701EBD3635C11704B53F82430CC1701EBD4646411A1EB44150124AC4023400BB1012030BD0020FCE76B49087070476A4861
:405100000078704770B52DED048B04460025442C6FD2DFE804F02223282D2E2F3038404850586068727B8790ABB0FDFCFBFAF9F8F7F6F5F4F3F2F1F0EFEEEDECEBEAE9E80A
:40514000E7E6E5E4E3E2E1E0DFDEDDDCDBDAD9D8D7D6D5D4D3D2D1D0CF9CFEE20EF09EFD80F00105F9E222F057F880F00105F4E2F3E2F2E2F1E20FF063FC18B1F8F7E9F846
:4051800000B10125E9E20FF05BFC18B1F8F7D9F800B10125E1E20FF053FC18B1F8F7E1F800B10125D9E20FF04BFC18B1F8F7EAF800B10125D1E20FF043FC18B1F8F7DAF831
:4051C00000B10125C9E20FF03BFC18B1F8F7E2F800B10125C1E211F0A2FB012800D100E000200546B9E211F09AFB032802D1012001E0B1E200200546AFE22C4890F8380014
:40520000012800D100E000200546A6E20FF018FC38B1264890F8380008B9012000E0002005469AE2214890F89000012800D100E00020054691E20FF003FC38B11B4890F8C3
:40524000900008B9012000E00020054685E2174890F83800022804D0144890F89000022801D1012000E00020054676E20CF041F980F0010571E20E48007D60B90648001F61
:40528000006900F48020B0F5802F42D002F034FB08B101203EE03CE0DC180020F80300201827002098030020990300203C290020D02B00204CE23EE210E203E2FAE1EDE1E3
:4052C000E1E1D5E1CCE1C3E1B7E1AEE1A2E199E190E187E17EE175E16CE163E15AE151E148E13FE136E12AE11EE10CE1E3E0D6E0C9E0BCE0AFE0A2E095E08BE080E075E07A
:405300005DE050E043E032E025E018E00FE00BE002E00020054620E2F748007D08B9012000E00020054618E2F448057815E2F5F7B3F908B1012000E0002005460DE20EF068
:4053400041FAB0EE408A9FEDEE1ADFEDEE0A0EF0B8F9054601E20EF035FAB0EE408A9FEDEA1ADFEDEA0A0EF0ACF90546F5E102F0A9FFB0F57B4F07DB02F0A4FF4FF6FF7177
:40538000884201DA012000E000200546E5E102F05AFF28B1DE488078FE2801D0012000E000200546D9E1DA488078FE2806D0F7F7F6FE18B101250020D6490872CDE1D4484D
:4053C0008078FE2805D0D448007810B103F05CFD20B101251C20FFF78FFE06E0FFF78FFE1C2802D10020FFF787FEB6E1CB48007800F0B40008B1012000E000200546ACE1D0
:40540000C648007800F0480008B1012000E000200546A2E1C2480088102801D0012000E00020054699E10EF01CFAB0EE408A9FEDB41ADFEDB60A0EF044F905468DE10EF031
:4054400018FAB0EE408A9FEDAE1ADFEDB00A0EF038F9054681E10EF014FAB0EE408A9FEDA81ADFEDAA0A0EF02CF9054675E10EF0D1F9B0EE408A9FEDA21ADFEDA40A0EF006
:4054800020F9054669E10DF03AFAB0EE408A9FED9C1ADFED9E0A0EF014F905465DE10EF0C1F9B0EE408A9FED961ADFED980A0EF008F9054651E121F0B7FE18B3F5F743FD58
:4054C000B0EE408AF5F714FD38EE400A10EE106A30462EF03FFC41EC190BB0EE490AF0EE690A2BF011F8B0EE408AF0EE608A9FED8D0B53EC102B51EC180B2EF033FA00D28E
:40550000012500BF29E1F5F71EFDDFED880AB4EEE00AF1EE10FA04DDF4F718FB08B1012000E00020054618E102F0E6F920B903F04BF908B9012000E0002005460DE102F0B7
:40554000DBF920B108F0D4FC08B1012000E00020054602E10FF074FA18B103F08AFD80F00105FAE0F5F7A3F808B1012000E000200546F2E0F5F7BAF808B1012000E00020C0
:405580000546EAE0F5F73FF908B1012000E000200546E2E0F5F777F908B1012000E000200546DAE0F5F7ACF908B1012000E000200546D2E0F5F7F8F908B1012000E0002071
:4055C0000546CAE0F5F730FA08B1012000E000200546C2E0F5F764FA08B1012000E000200546BAE0F5F798FA08B1012000E000200546B2E0F5F7D0FA08B1012000E000200B
:405600000546AAE0F5F704FB08B1012000E000200546A2E00FF014FA30B1F5F76DFB08B1012000E00020054697E0F5F783FB08B1012000E0002005468FE00FF001FA30B14C
:40564000F5F796FB08B1012000E00020054684E0F5F7B4FB08B1012000E0002005467CE0F5F7CAFB08B1012000E00020054674E00FF0E6F930B1F5F7DDFB08B1012000E0A1
:405680000020054669E00FF0DBF930B1F5F7F0FB08B1012000E0002005465EE00EF07DF906460EF0FDF906430EB1012000E00020054652E00EF02CFA08B1012000E00020F0
:4056C00005464AE00FF0BCF938B108F0A7FE012803D103F035FC00B901253EE0F4F77BFF28B9F5F76AFC10B9F5F781FC00B303F027FCE8B901201CE0E82B0020DD03002059
:4057000000FF7F4700A0254600007A460000000058CA0020503200203C050020ED030020BE070020000000000070A7400000FA450020054611E00EF091FA20B9FE4800788D
:4057400022F0B6F908B1012000E00020054604E003F069F8054600E000BF00BF05B100BF3DB9F6480078002807DDF4480078844203D10120BDEC048B70BD0020FAE74FF021
:405780000008C1464FF0010A4FF0500B0321EC4880F8B810002491E0EA48005D04EB840101EBC401E84A02EB810189680870E548FF30005D00287FD0E21704EBD26253115B
:4057C000E24A52F82320E31704EBD3635B11A4EB431C012303FA0CF31A43E31704EBD3634FEA631CD94B43F82C20E21704EBD2625311D64A0C3252F82320E31704EBD363EE
:405800005B11A4EB431C012303FA0CF31A43E31704EBD3634FEA631CCC4B0C3343F82C2004EB840000EBC400C74901EB8000007BE0B1E21704EBD2625311C44A183252F811
:4058400023202146E31704EBD3635B11A4EB431C012303FA0CF31A432046E31704EBD3634FEA631CB94B183343F82C2024F0B1F8B74941F8240000BFE21704EBD26253111C
:40588000B24A243252F823202146E31704EBD3635B11A4EB431C012303FA0CF39A432046E31704EBD3634FEA631CA84B243343F82C2000E000E000BF601CC4B2442CFFF648
:4058C0006BAF4FF47A60DFF88CC200DF9C48D0F8DC100120DFF880C200DF4FF47A60DFF874C200DF00BF002259460320DFF86CC200DF0646022E21D1DFF864C200DF074695
:4059000007F00200D0B1002416E0002004EB840101EBC4018C4A02EB81018968087004EB840101EBC40102EB8101896808782146FFF751FB601CC4B2442CE6DB0024AAE25F
:405940002046FFF7DFFB05462046FFF7BEFBA8427ED0002D7DD1A946E31704EBD3634FEA631C7A4B0C3353F82C304FEAE47C04EBDC6C4FEA6C1CA4EB4C1E4FF0010C0CFA91
:405980000EFC03EA0C034FEAE47C04EBDC6C4FEA6C1CA4EB4C1E4FF0010C0CFA0EFC634501D04FF0010904EB840000EBC400664901EB800090F8330000F0010008B14FF058
:4059C000010904EB840000EBC4005F4901EB800090F8330000F0020020B10BF046FC08B14FF0010904EB840000EBC400564901EB800090F8330000F0040038B108F080FA73
:405A000010B921F03CFC08B14FF0010904EB840000EBC4004C4901EB800090F8330000F0080020B1BAF1000F01D04FF0010904EB840000EBC400444901EB800090F8330001
:405A400000F0100038B14748005D012803D101E00FE00FE08146B9F1010F0AD10020414908554FF001082046FFF7DCFA3720F7F771FD03E1E31704EBD3634FEA631C334BCC
:405A800053F82C304FEAE47C04EBDC6C4FEA6C1CA4EB4C1E4FF0010C0CFA0EFC03EA0C034FEAE47C04EBDC6C4FEA6C1CA4EB4C1E4FF0010C0CFA0EFC6345DAD00020294993
:405AC000085500BF01F018FFE8B1E21704EBD26253111E4A243252F823202146E31704EBD3635B11A4EB431C012303FA0CF31A432046E31704EBD3634FEA631C134B2433CF
:405B000043F82C2035E0E21704EBD26253110F4A243252F823202146E31704EBD3635B11A4EB431C012303FA0CF39A432046E31704EBD36318E000008E0700209A03002041
:405B400060420020182700203C3F0408DC180020C81700202923040889230408E923040831230408841700204FEA631CF74B43F82C20E21704EBD2625311F44A243A52F840
:405B80002320E31704EBD3635B11A4EB431C012303FA0CF31A43E31704EBD3634FEA631CEA4B243B43F82C2023F013FFE84941F8240004EB840000EBC400E64901EB80004A
:405BC00080680078401C04EB840101EBC401E14A02EB81018968087004EB840000EBC400114601EB8000806800787E2808DD7E2004EB840101EBC40102EB81018968087056
:405C000000BF00BF01F078FE01281BD1E21704EBD2625311CD4A52F823202146E31704EBD3635B11A4EB431C012303FA0CF31A432046E31704EBD3634FEA631CC34B43F863
:405C40002C201AE0E21704EBD2625311BF4A52F823202146E31704EBD3635B11A4EB431C012303FA0CF39A432046E31704EBD3634FEA631CB54B43F82C2000BF002D7DD0EE
:405C8000E21704EBD2625311B04A183A52F82320E31704EBD3635B11A4EB431C012303FA0CF31A40002A53D104EB840000EBC400A84901EB8000406AE8BBE21704EBD26262
:405CC0005311A24A183A52F82320E31704EBD3635B11A4EB431C012303FA0CF31A43E31704EBD3634FEA631C984B183B43F82C204FF0010804EB840000EBC40001EB800015
:405D0000806800787E2811DA04EB840000EBC40001EB800080680078401C04EB840101EBC4018C4A02EB81018968087021460120FFF764F900E00CE004EB840101EBC40189
:405D4000844A02EB8101896808782146FFF743F95BE004EB840202EBC4027E4B03EB8202516A7B4A52F8240023F039FEF0B3E21704EBD2625311754A183A00E083E052F845
:405D80002320E31704EBD3635B11A4EB431C012303FA0CF31A43E31704EBD3634FEA631C6A4B183B43F82C204FF0010804EB840000EBC400674901EB8000806800787E28B8
:405DC00011DA04EB840000EBC40001EB800080680078401C04EB840101EBC4015D4A02EB8101896808702146012000E00DE0FFF705F904EB840101EBC401564A02EB81014D
:405E0000896808782146FFF7E6F804EB840202EBC402504B03EB8202127BA2B3E21704EBD2625311494A0C3A52F82320E31704EBD3635B11A4EB431C012303FA0CF31A40C6
:405E40000ABB01F059FD10B901F00BFCE0B104EB840000EBC4003F4901EB8000806A68B104EB840202EBC4020B4603EB8202916A374A52F8240023F0B2FD20B12046FFF7E7
:405E80008DF84FF0010804E02046FFF787F84FF00108601CC4B2442CFFF652ADB8F1010F0BD12D48D0F8DC100120DFF8B0C000DF4FF000083720F7F74DFB4FF0000AFFF7A0
:405EC00049F804460FE5002108E02048243850F8210008B101207047481CC1B20329F4DB0020F8E7002108E018480C3850F8210008B101207047481CC1B20329F4DB0020F2
:405F0000F8E770B543201DE0C41700EBD46465110E4C0C3C54F82540C51700EBD5656D11A0EB45160125B5402C40C51700EBD5656D11A0EB45160125B540AC4200D103E028
:405F4000411EC8B20028DFDC00BF70BD00190020C81700203C3F0408604200208923040870B5002401F0C8FC78B343242AE0E31704EBD3635D11364B53F82530E51704EB0D
:405F8000D5656D11A4EB45160125B5402B40E51704EBD5656D11A4EB45160125B540AB420ED104EB840303EBC4032A4D05EB830393F83330102B03D1274B1B5D03B903E0A7
:405FC000601EC4B2002CD2DC00BF204670BD0121214A1154704701460020FF2906DA1E4A525C0AB1012200E000221046704700B5002304E01846FFF7EAFF581CC3B2442B15
:40600000F8DB00BD0EB5154A07CA8DE807001CF04BFB1DF0DDFB0C226946FF201CF010FB0EBD014601EB810000EBC100094A52F820007047014601EB810000EBC100054AC9
:4060400002EB8000007970477047054908707047E81800203C3F0408841700200C4D04089A030020FE48007B7047FD490873704770B52DED068B04460D46284623F0D1FC20
:4060800000EE100AB8EE400AB0EE408A9FEDF50AC8EE000AB0EE608A94ED000AD4ED020A00EE880ADFEDF00A68EE200A20EE200A10EE101A08462DF04DFE41EC1A0BB0EE89
:4060C0004A0AF0EE6A0A2BF0DFF8B0EE409AF0EE609A51EC190B2DF001F808EE100A94ED040A20EE080AB0EE408AB0EE480ABDEC068B70BD10B52DED088BF0EE409AF0EEBB
:40610000608A04469FEDD90AF0EE40AA9FEDD50AC0EE290AB0EE608AB1EE000A28EE800AC0EE080AB0EE60AA9FEDD00AB0EE40BA204623F076FCBCEEC80A10EE101AB0FB37
:40614000F1F201FB120000EE100AB8EE400AB0EE409AB5EE000A28EE000AB4EEC90AF1EE10FA15D8B6EE080A28EE000AB4EEC90AF1EE10FA0CDDBFEE000A2AEE000AB0EE12
:4061800040AAB0EE000A28EE800AB0EE40BA0EE0B6EE080A28EE000AB4EEC90AF1EE10FA05D8B9EE000A28EE800AB0EE40BAB0EE4B0A0AEE090AF0EE40AAB0EE6A0ABDECAC
:4061C000088B10BD2DE9F0412DED028B05460F4690460024002600BF32E0322108FB01F000EE100AB8EEC00ADFED9E0A80EE201A05F1300000EB840090ED000A30EE410A60
:4062000005F1300000EB840080ED000A08FB01F000EE100AB8EEC00ADFED920A80EE201A05F1700000EB840090ED000A30EE410A05F1700000EB840080ED000A601CC4B2D3
:40624000082CCADB0024D8E007F1300000EB840090ED000A07F1700000EB8400D0ED000A30EE600AF0EE000A20EE200AB0EE408A05F1300000EB840090ED000A07F1300059
:4062800000EB8400D0ED000A30EE600A05F1900000EB860080ED000A05F1900000EB860090ED000AC0EE080A9FED710A20EE800A05F1CC0000EB860080ED000A05F15000E5
:4062C00000EB840090ED000A05F1100000EB8400D0ED000A30EE600A07F1500000EB8400D0ED000A07F1100000EB840090ED001A70EEC10A80EE201A05F5847000EB860028
:4063000080ED001AB7EE000AC0EE080A05F5A27000EB8600C0ED000A701CC6B20F2E6ADA07F17000611C00EB810090ED000A07F1300000EB8400D0ED000A30EE600AF0EE12
:40634000000A20EE200AB0EE408A05F1700000EB810090ED000A07F1700000EB8100D0ED000A30EE600A05F1900000EB860080ED000A05F1900000EB860090ED000AC0EE5D
:40638000080A9FED3B0A20EE800A05F1CC0000EB860080ED000A05F1500000EB810090ED000A05F1100000EB8400D0ED000A30EE600A07F1500000EB8100D0ED000A07F148
:4063C000100000EB840090ED001A70EEC10A80EE201A05F5847000EB860080ED001AB7EE000AC0EE080A05F5A27000EB8600C0ED000A701CC6B2601CC4B2082CFFF624AF3B
:406400001C4B0F221C4901F13C0013F080FC1B4B0F2219493C3901F1780013F078FC154890ED010A0E4880ED1D0A124890ED000A0B4880ED230A114890ED010ADFED100AFF
:4064400030EEC00AD0ED000A80EE201A044880ED261A0F210848783813F03FFC004811E02019002000007A44DB0FC940000000000000B443A0030020D01A0020A80300208C
:406480000000344380ED200ABDEC028BBDE8F08170B52DED028B0446B0EE408A0D46207800F0100000280AD094ED020A84ED030A84ED028AA078082802D10420208086E0CA
:4064C000207800F00100D8B394ED020AD4ED030AB4EEE00AF1EE10FA20DD94ED020AFE48817804F1500000EB810080ED000AFB49486823F096FA00EE100AB8EE400A5FEDEC
:40650000270A80EE201AF448817804F1700000EB810080ED001A0020E07002E0E078401CE070E0782179884251DD208840F002002080208820F0010020800020E07046E04C
:40654000FFE7207800F00200F0B394ED020AD4ED030AB4EEE00AF1EE10FA1ED294ED020AA17804F1100000EB810080ED000ADB49486823F056FA00EE100AB8EE400A5FED3F
:40658000470A80EE201AA17804F1300000EB810080ED001A0020E07002E0E078401CE070E0782179884212DD208840F001002080208820F002002080A078401CA070002039
:4065C000E0700DB1207900E001E0401E2071BDEC028B70BD10B52DED028BF0EE408AB0EE608ABE49486823F01CFAB0F57A7F0BD90121B0EE480ABA48FFF74AFF0021B0EED1
:40660000680AB548FFF744FFB548008804280DD1B1480088042809D10222AF49B048FFF7D1FD2020AE490880AB490880BDEC028B10BD70B52DED0C8B044602F063FD60B103
:40664000F6F7E5FEB0EE408AD4ED098AF1EE009AB1EE00AAB0EE009A57E002F08CFD40B3F5F72CF80546F5F72DF8281A00EE100AB8EEC00ADFED9B0A20EE200AB0EE40BA88
:40668000F5F792F8DFED980A20EE208A94ED090ADFED950A60EE208AB1EE000A6BEE009AB1EE000A2BEE00AAB0EE000A2BEE009A2BE00FF05FFFB0EE408A8C4991F828008E
:4066C00091ED0F0AF0EE400AB0EE480A0FF039FEDFED870A20EE200AB0EE408A834991F8280091ED0F1AF0EE410A94ED091AB0EE410A0FF026FEDFED7E0A60EE208AF0EE91
:40670000009AB0EE00AAB7EE009A4020005D40B994ED0B0A38EEC00A84ED0E0A01214020015519EE900A2DF015FB41EC1B0B94ED0B0A30EE480A10EE101A08462DF00AFBDC
:4067400041EC1D0BB0EE4D0AF0EE6D0A29F0DCFEB0EE40CAF0EE60CA53EC1B2B51EC1C0B2DF000F90ED24C20005D58B9606823F058F900EE100AB8EE400A84ED110A01214C
:406780004C2001551AEE100A2DF0E4FA41EC1B0B38EEC80A10EE101A08462DF0DBFA41EC1C0BB0EE4C0AF0EE6C0A29F0ADFEB0EE40DAF0EE60DA53EC1B2B51EC1D0B2CF011
:4067C00097FF0ED25820005D58B9606823F029F900EE100AB8EE400A84ED140A01215820015519EE100A2DF0B5FA41EC1B0B38EEC80A10EE101A08462DF0ACFA41EC1C0B04
:40680000B0EE4C0AF0EE6C0A29F07EFEB0EE40DAF0EE60DA53EC1B2B51EC1D0B2DF0A2F80DD8002164200155607B324951F8200000EE100AB8EE400A84ED170A31E019EEC9
:40684000100A2DF087FA41EC1B0B38EEC80A10EE101A08462DF07EFA41EC1C0BB0EE4C0AF0EE6C0A29F050FEB0EE40DAF0EE60DA53EC1B2B51EC1D0B2CF03AFF11D2642091
:40688000005D70B9012164200155606823F0C9F800EE100AB8EE400A84ED170A23F099F8A06078EEC8AA94ED0E0AB5EEC00AF1EE10FA0BD2B4EEE88AF1EE10FA06D294ED92
:4068C0001B0AB4EEEA0AF1EE10FA24D394ED0E0AB5EEC00A10E00000481B002020190020C819002017B7D1380AD7233C18210020E02E6542184D0408F1EE10FA25DDB4EE07
:40690000E88AF1EE10FA20DD94ED1B0AB4EEEA0AF1EE10FA19DDC4ED1BAA94ED1B0A10EE101A08462DF016FA41EC1C0BB0EE4C0AF0EE6C0A29F0E8FDB0EE40BAF0EE60BAFB
:4069400051EC1B0B2CF0CAFBA066BDEC0C8B70BD00200022002100BF33E0FE4B03EB820393ED000AB5EEC00AF1EE10FA01D14B1C99B2F84B403303EB820393ED000AB5EEB5
:40698000C00AF1EE10FA01D14B1C99B2F24B03EB820393ED000AB5EEC00AF1EE10FA01D14B1C99B2EC4B403303EB820393ED000AB5EEC00AF1EE10FA01D14B1C99B2531C9C
:4069C000DAB2082AC9DB00224FE0E44B93ED1D0ADFEDE30AB4EEE00AF1EE10FA06DC93ED1D0AB5EEC00AF1EE10FA01D24B1C99B2DA4B93ED230ADFEDDA0AB4EEE00AF1EE8F
:406A000010FA08DC93ED230ADFEDD60AB4EEE00AF1EE10FA01D24B1C99B2D04B93ED260ADFEDCF0AB4EEE00AF1EE10FA06DC93ED260AB5EEC00AF1EE10FA01D24B1C99B2C3
:406A4000C64B93ED200ADFEDC60AB4EEE00AF1EE10FA06DC93ED200AB5EEC00AF1EE10FA01D24B1C99B2531CDAB20F2AADDB01B901207047B94890F8A4007047B74981F838
:406A8000A4007047B548407B0C2823D0B348407B0B281FD0B148407B07281BD0AF48407B112817D0AD48407B082813D0AB48407B0A280FD0A948407B04280BD0A748407B45
:406AC000052807D0A548407B0F2803D0A348407B102801D1012070470020FCE79F48407B08281BD09D48407B042817D09B48407B052813D09948407B0A280FD09748407BF0
:406B00000B280BD09548407B0F2807D09348407B102803D09148407B112801D1012070470020FCE78D48407B082817D08B48407B042813D08948407B05280FD08748407B20
:406B40000A280BD08548407B0B2807D08348407B102803D08148407B0F2801D1012070470020FCE77D48407B082803D07B48407B0A2801D1012070470020FCE770B5002454
:406B800028F01AF8002872D101F05DFB18B10720FFF774FF80E00AF0ACFC30B9FFF7E2FF18B90220FFF76AFF76E019F03DFDB5EEC00AF1EE10FA06D2FFF7B4FF18B9092020
:406BC000FFF75CFF68E019F02FFDDFED670AB4EEE00AF1EE10FA02D2FFF780FF60B15F48407B0F280CD119F023FDDFED5F0AB4EEE00AF1EE10FA03D20420FFF73FFF4BE01A
:406C000019F012FDDFED590AB4EEE00AF1EE10FA06DDFFF763FF18B90520FFF72FFF3BE05348007D18B90120FFF728FF34E0F3F7D2FC50B102F084F938B94848407B0F2852
:406C400003D10D20FFF71AFF26E007F059FA28B107F056FA0546FFF711FF1DE0F6F7A3FB30B1F6F7A0FB0546FFF708FF14E01AE007F03EF938B13948407B0B2803D024207F
:406C8000FFF7FCFE08E0FFF72DF928B1FFF7FAFE10B90A20FFF7F2FEFFF7ECFE18B10120FFF7E3F90124204670BDC9B1DFED310AC0ED000ADFED300AC0ED010A2F4AD2EDBE
:406CC000060AB8EE601ADFED2E1AC1EE210A9FED2D1AC1EE201AC0ED021A80ED040A1CE0DFED290AC0ED000ADFED280AC0ED010A224AD2ED0D0AB8EE601ADFED211AC1EEF6
:406D0000210ADFED231A81EEA01AF6EE000A61EE200AC0ED020A80ED040A704710B501219FED1C0A0D481030FFF7BFFF4FF4C0710848303828F08BFA4FF4C07106483038CF
:406D400028F085FA0A2003493039087102493039087121E0F8190020781B00202019002000409C4500409CC52FDDE43E2FDDE43FE82B0020CDCCCC3D14AE473F184D04080C
:406D800000007A447A142E3FCDCC4C3E0000204233331F42C2B8B23E1120FC490880FC49088010BD2DED028B84B04FF47A66A821F84828F04CFA1421F74828F048FA00BFDA
:406DC000002231460320DFF8D4C300DF0546022D70D1DFF8CCC300DF0446022C6BD1EE480078002867D0EC480078122863DC0120EC490870E8480078E649487322F0E9FD4C
:406E0000E4494860E44890ED010A084680ED090A407BE54908700020DE498860084600218166C1660167C165016641668163C163016441648164C164016541658165002024
:406E4000D44981F8A4000846407BD84951F82000D04908600846407B122877D2DFE800F0A5505354555609454D4E4CA0412C3A515246C848002141678167C1678030C1601B
:406E8000016141618161C1610162016041608160FFF744FF04208DF8040003208DF8050005208DF80600022201A9FF201BF0C8FB04267BE0B0E07DE000219FEDBD0AB548A3
:406EC0001030FFF7F2FE9FEDBB0AB24880ED090A04266BE09FEDB80AAE4880ED090A042664E0F8F718F8C82660E000BFF8F713F8FCF7CFFEC82659E000BF00BF042655E050
:406F000000BF00BF00BF00BF00BF00BF02F0FAF850B1F6F77CFAB0EE408A9E4880ED0B8A012180F834102BE002F025F978B1F4F73BFCDFEDA20A20EE200AB0EE408A954806
:406F400080ED0B8A012180F8341019E02DE00FF011FBB0EE408A9A4991F8280091ED0F0AF0EE400AB0EE480A0FF0EBF9DFED950A20EE200A874880ED0B0A012180F83410C0
:406F800004208DF8040003208DF8050005208DF80600032201A9FF201BF052FB042605E04FF4C87607F0A5F900E000BF00BF042078490873012C2FD10020764948730021B6
:406FC00001209FED7C0AF3F77EFA0020754908709FED780A704880ED010A9FED760A6D4880ED090A012180F864104FF47A665820F6F7B0FA5920F6F7ADFAFFF733F804288D
:4070000002D10020FFF731F811201AF043F8002201A9FF201BF014FB5E48407B00287DD05C4A1168506822F0DAFC18BBFFF71AF804280FD05748407B07281BD05548407B7C
:40704000112817D05348407B0B2813D05148407B0C280FD0FFF792FD60B94E4890F8640001286DD14B49886840F6C41122F0B7FC002865D04748407B022807D04548407B52
:40708000012803D04348407B032819D1414890F8640030B93F4890ED000AB8EE400A80ED170A3C4890F8580030B93A4890ED000AB8EE400A80ED140A5920F6F74BFA1FE014
:4070C0003448407B06281BD1FFF742FC80B99FED3E0A304880ED1D0A9FED3B0A80ED230A9FED390A80ED260A9FED370A80ED200A002026490880264908805820F6F72AFA20
:40710000112019F0C7FF002022494873FEF7AAFF042802D10020FEF7A8FF00E010E0002101209FED240AF3F7CEF900201D4908709FED200A184880ED010A4FF47A663FE65F
:407140001448407B122879D2DFE800F0095279F5F3F2F1F0EFEEEDECEBEAE90A0BE81CE200BF02F008F888B3F4F7BCFB00EE100AB8EE400A074880ED090AD0ED090AB0EEFB
:40718000600A0121032008F04BFF2DE0C8190020481B0020201900200C190020E9230408312304089C030020B8030020184D04080000A04200000000000070420AD7233C58
:4071C00018210020E02E6542003C1C46FFE71FED070AFC4880ED090AD0ED090AB0EE600A0121032008F090FDF648FFF722FAD4E101F0C1FF88B1F4F75DFA00EE100AB8EE9B
:40720000400AF04880ED090AD0ED090AB0EE600A0121032008F004FF0CE01FED1A0AE94880ED090AD0ED090AB0EE600A0121032008F06AFDE348FFF7FCF9AEE193E101F0E1
:4072400061FF68B19FEDE00ADE4880ED090AD0ED090AB0EE600A0121032008F025FE59E001F089FF00B3F4F725FA00EE100AF8EE408AF4F71FFA8046F4F724FAA8EB0000B4
:4072800000EE100AB8EEC00ADFEDD00A40EEC08ACC48C0ED098AD0ED090AB0EE600A0121032008F0BDFE35E01FF0E9FFD8B1C84890ED640ADFEDC70A20EE200A5FED410A18
:4072C00020EE200AB0EE408A014691F8280091ED0F0AF0EE400AB0EE480A0EF077FAB94880ED090A0DE0BA4991F8280091ED0F0AF0EE400A9FEDB80A0EF068FAB14880EDE3
:40730000090AB048D0ED090AB0EE600A0121032008F0FAFCAB48FFF78CF93EE1F9E0D0E0E5E00BE104E1F7E001E1F6E0F0E08FE07FE06FE0FFE701F0E5FE68B19FEDA50A01
:40734000A04880ED090AD0ED090AB0EE600A0121032008F0A9FD59E001F00DFF00B3F4F7A9F900EE100AF8EE408AF4F7A7F98046F4F7A0F9A8EB000000EE100AB8EEC00ADC
:40738000DFED920A40EE808A8E48C0ED098AD0ED090AB0EE600A0121032008F041FE35E01FF06DFFD8B18A4890ED650ADFED890A20EE200A5FED7F0A20EE200AB0EE408AE0
:4073C000014691F8280091ED0F0AF0EE400AB0EE480A0EF0FBF97B4880ED090A0DE07C4991F8280091ED0F0AF0EE400A9FED7B0A0EF0ECF9734880ED090A7248D0ED090AD6
:40740000B0EE600A0121032008F07EFC6D48FFF710F9C2E06E4890F84210D03000EB8100D0ED000AB0EE600A01210846F3F74BF8B3E0674890F84210D83000EB8100D0ED82
:40744000000AB0EE600A01210846F3F73CF8A4E05C4841681030FEF70BFE5A4880ED090A5B4991F8280091ED0F1AF0EE410A554991ED091AB0EE410A0EF0A8F9F0EE408AA7
:407480000121032008F040FC4E4890F82900B8B100204C4981F829000FF0C2F8F0EE408A03214F4810F06DF84D4890ED001AF0EE410A444890ED091AB0EE410AFFF78AF8E9
:4074C0006BE0404948684749D1ED000A464991ED000AFEF70FFE3B4880ED090AD0ED090AB0EE600A01210846F2F7EDFF55E0354841681030FEF7BCFD324880ED090AD0ED77
:40750000090AB0EE600A01210846F2F7DCFF44E000BFFCF713FB40E000BF2A48D0ED090AB0EE600A01210846F2F7CDFF35E034E006F001FE8046FEF798FD2EE0214A0832A9
:4075400002F11C0101F18000F9F7C3FA8046FEF78CFD1C48D0ED090AB0EE600A01210846F2F7B1FF19E00020164948730873002101201FEDF00AF2F7A6FF00201B490870D3
:407580001FEDF40A1A4880ED010A002201A9FF201BF056F84FF47A6600BF00BFFEF762FD04287FF4CCAD4FF4FA71384622F017FA00283FF4C4AD22F00CFA0746112019F0DC
:4075C00069FDBCE52019002000008CC23333333F1821002000008C42C2B8B2BEC2B8B23EB0030020C0030020BC0300209C0300200C19002070B52DED028B0446B0EE408A73
:407600000025B5EEC08AF1EE10FA0AD04CB1122C07DCAF4890ED010AB4EE480AF1EE10FA0DD1AC48D0F890110120DFF8ACC200DF9FEDAA0AA64880ED010A00250DE00CB106
:40764000A3480470A24880ED018AA248D0F890110220DFF884C200DF01252846BDEC028B70BD9F480078704701209E4981F8290070477A2303709B4BD3ED0E0A9FED9A0AEC
:40768000B2EE041A00EE810ABDEEC00A10EE103A1AB24270130A8370924B93ED110ABCEEC00A10EE103A99B2C1700B0A03718D4B93ED140ABCEEC00A10EE103A99B24171E0
:4076C0000B0A8371874B93ED170ABCEEC00A10EE103A99B2C1710B0A0372824BD3ED1A0A9FED810AB2EE041A00EE810ABDEEC00A10EE103A1AB24272130A837270477B23A8
:407700000370784BD3ED1D0A9FED781A9FED760A00EE810ABDEEC00A10EE103A19B241700B0A83706F4BD3ED230A9FED701A9FED6E0A00EE810ABDEEC00A10EE103A19B286
:40774000C1700B0A0371674BD3ED260A9FED671A9FED650A00EE810ABDEEC00A10EE103A19B241710B0A83715E4B93ED200ADFED600A20EE200ABCEEC00A10EE103A9AB220
:40778000C271130A0372704710B500245548407B122813D2DFE800F013141718191A1B091E1F1D0E121C1215160A00BFFCF7B8FA044611E006F097FD04460DE000BF00BFCE
:4077C00000BF00BF00BF00BF00BF00BF00BF00BF00BF00BF00BF00BF00BF204610BD10B500244048407B122813D2DFE800F013141718191A1B091E1F1D0E121C1215160A17
:4078000000BFFCF791FA044611E006F06CFD04460DE000BF00BF00BF00BF00BF00BF00BF00BF00BF00BF00BF00BF00BF00BF00BF204610BD2B48407B70472A4890F8640093
:40784000704710B500242748407B122816D2DFE800F01718191A1B1C1D0920211F16151E150E0F0A00BFF7F786FB044613E000BFFFF7E3FF642110FB01F40CE000BF00BFD0
:4078800000BF00BF00BF00BF00BF00BF00BF00BF00BF00BF00BF00BF204610BD002011490873704713480078704710B500F0CEFF044644F6206122F092F838B900F0C6FFA2
:4078C00040F2DC51884201D9012010BD0020FCE70C1900206042002089230408000000009C03002020190020000000470000C84200007A44B8030020FE490979042901D10B
:40790000012100E000210846704770B50023012113E0CC1701EBD4646511F74C54F82540CD1701EBD5656D11A1EB45160125B5402C4004B10B46481CC1B24029E9DB1846F3
:4079400070BD70B504460D46E21704EBD2625311E94A52F823202146E31704EBD3635B11A4EB43160123B3401A432046E31704EBD3635E11E04B43F826202846FDF7BCFBD1
:40798000002C37D00821DD48DFF874C300DF012813D0DA482038817F807F401CD74A203A907710464454807F1E2802DB002011468877D248DFF84CC300DF0821D248DFF877
:4079C00040C300DF012815D022F003F8CF4901EBC4014860CD4810F83400FF2806DACB4810F83400401CC94901F83400C648DFF814C300DF70BDC6490870704710B5BD4807
:407A0000007905287BD2DFE800F003152581DE00FEF768FA10B90220B6490871BD48007838B10120BC490870FFF7E5FF0020B94908701AE1FEF756FA10B90220AD49087134
:407A4000B448007828B10120B34908700020B14908700AE1FEF746FA18B10020A549087153E0AC48007898B30120AB490870FEF739FA50B1FEF745FA044621460920FFF77E
:407A800060FF0120FFF7B7FF3FE006F031FA38B129210320FFF755FF0120FFF7ACFF34E09E48007800F0080038B91A213120FFF748FF0120FFF79FFF27E003208D490871A6
:407AC00021F087FF964908600020FDF715FB1CE0FFE7FFF7B2FEC0B909F009F8A8B1FFF7C0FD90B9FFF7E1FE78B118F0A1FDDFED8D0AB4EEE00AF1EE10FA06DD00E0B3E062
:407B00009FED890A0F20FFF775FDAEE08148007800284DD006F0ECF950B129210320FFF710FF0120FFF767FF01207B49087049E0FEF7D8F968B10120FFF75DFF01207649F8
:407B40000870FEF7DEF9044621460920FFF7F9FE38E04FF47A717248006821F040FF90B16E48007800F0020008BB0120FFF743FF1A213120FFF7E5FE0120674908700020F7
:407B80005C4908711EE06548007800F00B0070B1FFF767FD30B16548D0F890110120DFF890C100DF04205349087109F082FB09E01A210220FFF7C5FE0120574908700220E6
:407BC0004C49087151E05348007850B91A210220FFF7B7FE01205049087002204549087137E006F085F968B129210320FFF7A9FE0220404908710120FFF7FDFE0120464933
:407C0000087026E0FEF76EF980B10020394908710120FFF7F0FEFEF774F9044621460920FFF78FFE01203C49087012E0F5F7C8FB78B100202F4908710120FFF7DCFEF5F784
:407C4000BFFB044621460920FFF77BFE01203249087028480079042805D021F0BAFE2549086009F025FB00E000BF00BF214800792049487110BD2048001F00210160416072
:407C80008160C16070472B490870704710B52A4991F8300001F01EF930B1002213466421264813F091FC11E0234991F8300001F033F928B9204991F8300001F035F928B162
:407CC0000022134631211D4813F07EFC10BD10B50024194991F8300001F0FCF848B9164991F8300001F018F918B9134991F8300026E028E0C8030020681F0020541F0020EB
:407D0000512804086D270408F01C0020341D0020D2030020D3030020D4030020DC030020D80300202FDDE43E0000C8426042002089230408D00300201821002098CF002020
:407D400001F0F2F800B10124204610BDFE480078704710B50446FD480078844204D0FB480470162019F096F910BD00EE900AB8EE601ADFEDF70AF5EE001A51EE210AB0EE78
:407D8000600ADFEDF40A80EE201AB0EE410A7047F1480078704710B52DED028BFFF7F8FF022807D0FFF7F4FF032803D0FFF7F0FF052812D10CF02FFE30B10CF026FE022855
:407DC00002D19FEDE68A0AE00CF025FE10B19FEDE48A04E01FED2D8A01E01FED2E8AB0EE480ABDEC028B10BD10B52DED028B18F0FFFBB0EE408AFFF7CEFFB4EEC08AF1EE4D
:407E000010FA03DB0120BDEC028B10BD0020FAE710B52DED048BF0EE408AB0EE609A0446F0EE689AFFF7E0FF00EE100AB8EE400AB4EEC90AF1EE10FA07DDFFF7D5FF00EE96
:407E4000100AB8EE400AB0EE409A29EE090ADFEDC50A80EE808AECB1F4EEC88AF1EE10FA05DDF0EE489A0120BF49087015E0B1EE480AF4EEC08AF1EE10FA07D2B1EE480A81
:407E8000F0EE409A0120B849087006E00020B649087002E00020B4490870B0EE690ABDEC048B10BD10B504460020206060606071207121F08EFD206010BD2DED048B92B0C1
:407EC0004FF05008002405E04FF6FF702DF81400601CC4B2022CF7DB0020FFF7D4FE00208DF80400A1490870FFF785FD0020A0490870A048DFF880C200DFA048DFF878C23E
:407F000000DF9F48DFF870C200DF00209949183908759C48FFF7C6FF03219B4880F8441100BF002241460720DFF860C200DF0746022F7AD1DFF858C200DF054605F002000E
:407F4000002873D010218B48DFF848C200DF012809D028228749183908A827F01CF98548DFF834C200DFBDF82060FFF7C5FC08B1012000E00020814618F03AFBF0EE408A9E
:407F80003046FFF7F2FEB0EE409A4846F0EE680AFFF73EFFB0EE408AFFF7AEFC00B375481838007D01280BD1DDED0A0AB0EE600A0121042007F01DFF8146FFF7CAFE2FE0BF
:407FC0006C481838007D02280BD1DDED090AB0EE600A0121052007F067FF8146FFF7B9FE1EE064481838007D03280BD1DDED0B0AB0EE600A0121062008F012F88146FFF791
:40800000A8FE0DE05B481838007D042808D101210220B0EE480A07F077FE8146FFF799FE9DF83500012802D102E047E032E000205A4908709DF8350040B95948007840F01C
:408040000800574908700020FFF7D5FC4FF6FF7086421FD05248007800F00200D0B95048007800F00800A8B1002410E03DF81410711A08B20FF0E9FC022806DC48480078F6
:4080800040F002004649087003E0601CC4B2022CECDB00BF05F0040080B1424801889DF80420501CC0B28DF804002DF812109DF80400022802DB00208DF804001CF069F9A3
:4080C00088B10BF0EBFD70B1FFF740FE58B9364813F0BCFA38B1FFF7FAFD08B1FFF7D6FD0120FFF7D0FD9DF8360090B10C9821F098FCB0F5C87F0CD301201C490870224803
:40810000D0F8B4100120DFF8A4C000DF0CF0A4FC02E00020154908702548007D012854D19DF81C0028B900201D49087021F051FC824640F2E241504621F051FCD0B31FF03B
:408140009EF8B8BB012036E0D0030020C60300200000FB4500007A44C40300200AD7A33C9A99193ED222FB3FD5030020D1030020DD030020181D00205D270408541F002022
:40818000F01C0020C803002060420020E923040831230408512804086D270408D3030020DC030020281D002040D1002089230408B82B002028E0FE490870FE48D0F8B4106A
:4081C0000120DFF8F4C300DF1EE09DF81C0001281AD1FA48007DB8B90020F5490870FFF74AFDF448D0F8B4100120DFF8CCC300DFF348007840F00100F14908700120F149CC
:40820000087021F0E6FB82461822EC4902A826F0C2FFFFF7F3FBEB480078012809D1FFF774FBE94908700020E6490870172018F031FFFFF761FB08B1012000E00020814652
:40824000F3F753FC6DE6E14800787047E04800787047E0480078704770B50025DE48007D012801D1002405E0DB48007D08B9012400E002242543D948C472FDF733FE08B94A
:40828000012400E0002445EA8400C5B2D3484472D348007D08B9012406E0D148007D012801D1002400E0022445EA0410C5B2CB488472FFF7CEFF044645EA8415C74804725E
:4082C000284670BDC748008870472DE9F04105460C4617469846069EB5F52D4F28D12821C0481830DFF800C300DF012820D0A078BC49C875A07800F00300487520786178F5
:4083000040EA0120B749088021F063FBB54908610120887504200875A648D0F840110220DFF894C200DFAF481830DFF8C0C200DFBDE8F081F0EE400A9FEDAD0A30EEC01AB0
:40834000DFEDAC1A81EE210A70472DE9F0412DED028B04460D4616461F462078AD2833D12821A0481830DFF880C200DF01282AD0E0789C49C875E07800F00300487560786F
:40838000A17840EA012000EE100AB8EEC00AB0EE408AB0EE480AFFF7CDFF924880ED020A21F017FB8F4908610120887508758148D0F840110220DFF800C200DF89481830E0
:4083C000DFF828C200DF6BE02078A92834D1282184481830DFF810C200DF012860D0E0788049C875E07800F0030048756078A17840EA012000EE100AB8EEC00AB0EE408A64
:40840000B0EE480AFFF796FF764880ED010A21F0E0FA7449086101208875022008756548D0F840110220DFF890C100DF6D481830DFF8B8C100DF33E02078AF2830D12821D6
:4084400068481830DFF8A0C100DF012828D0E0786449C875E07800F0030048756078A17840EA012000EE100AB8EEC00AB0EE408A5C4880ED038A21F0ACFA5A4908610120E4
:408480008875032008754B48D0F840110220DFF828C100DF53481830DFF850C100DF00BFBDEC028BBDE8F0811FEDD61A5FEDD80A40EE010AF1EE001AB6EE001A00EEA11A3A
:4084C000FCEEC10A10EE901A88B2704710B52DED028B0EF04FF8B0EE408A9FED470AB4EE408AF1EE10FA06D0B0EE480AFFF7DCFF3A49088003E04FF6FF70384908802D482C
:40850000D0F840110420DFF8B0C000DF33480088BDEC028B10BD70B58CB006460025002E6ED01EF0ACFE002878D040F2B240012102220023CDE90532CDE9071004201721C9
:408540000193CDE902310490972013460022114600900AA812F03AFE0AA9304612F019FB044640F292400440844204D11DB9042022490870012540F2B240012102220023E9
:40858000CDE90532CDE90710042017210193CDE902310490972001230022114600900AA812F014FE0AA9304612F0F3FA044629E0DD0300206042002089230408B82B002002
:4085C000DC030020D4030020C5030020D1030020C6030020D2030020E82B0020281D0020F8290020001D0020512804086D27040800401C460000C84200FF7F47C403002038
:408600000BE00BE040F292400440844205D1002DFCD105208F4908700125B7E040F2B240012102220023CDE90532CDE9071017210193CDE902319720049300900123002234
:4086400011460AA812F0C2FD0AA9304612F0A1FA044640F292400440844204D11DB903207C490870012540F2B240012102220023CDE90532CDE9071017210193CDE90231E5
:408680009720049300901346002211460AA812F09DFD0AA9304612F07CFA044640F292400440844204D11DB902206A490870012540F2B240012102220023CDE90532CDE975
:4086C000071017210193CDE902319720049300900323002211460AA812F078FD0AA9304612F057FA044640F292400440844204D11DB9032057490870012540F2B2400121E2
:4087000002220023CDE90532CDE9071017210193CDE902319720049300900423002211460AA812F053FD0AA9304612F032FA044640F292400440844204D11DB902204549F7
:408740000870012540F2B240012102220023CDE90532CDE9071017210193CDE9023197201A461946049300900AA812F02FFD0AA9304612F00EFA044640F292400440844257
:4087800004D11DB9012033490870012515B15620F4F7E0FE28460CB070BD10B52E4890F8280007280DD117F023FFDFED2C0AB4EEE00AF1EE10FA01DB012000E00020044698
:4087C00000E00124204610BD10B517F011FFDFED240AB4EEE00AF1EE10FA01D8012010BD0020FCE79FED1F0A70479FED1F0A70471848007803280FD01648007802280BD097
:4088000014480078012807D012480078042803D010480078052801D1012070470020FCE712480079704710B500F056FC10B11048047800E00024204610BDF0EE400A1FED58
:40884000931A1FED950A00EE810A70470748006870470000C4030020182100202FDDE43E83C00041B81E4141A2454841C8030020D503002010B5044600BF28222146FE48A0
:40888000006802F001FE20B928222146FB4826F03DFC00BF10BD10B504462822F749204626F034FC10BD01B500BF04226946F2480068283002F0E8FD18B99DF80000EF49EC
:4088C000886200BFEE48C16B0220DFF8B8C300DF08BD01B500BF04226946E74800682C3002F0D2FD18B99DF80000E449C86200BF08BD01B5E14890F830000099884219D033
:4089000000BF04226946DC480068303002F0BCFD10B9DA490098086300BFD84890F83000922804D0D54890F83000932802D101201AF066FF08BD10B52DED020B00BF04226F
:408940006946CD4800683C3002F09EFD20B99DED000ACA4880ED0F0A00BF04F048F8C848C16B0220DFF81CC300DF0220F4F7F2FD5020F4F7EFFD1CBD01B500BF0122694684
:40898000BD480068483002F07FFD20B99DF80000BA4981F8480000BF08BD08B5002000901EF05AFCA0B10021B74800781EF07EFCB64800781FF07CF828B10220FFF7DCFFA7
:4089C0000120009004E00120FFF7D6FF0220009000BF01226946A8480068493002F054FD20B99DF80000A54981F8490000BFA448016D0120DFF88CC200DF08BD01B500BF09
:408A0000042269469C480068443002F03DFD10B99A490098486400BF08BD01B5974890F841009DF80010884215D000BF0122694691480068413002F027FD20B99DF8000088
:408A40008E4981F8410000BF19F02EFE08F05EF81F20F4F77FFD08BD01B500BF0122694685480068423002F00FFD20B99DF80000824981F8420000BF19F016FE2620F4F7CB
:408A800069FD7F48C16B0220DFF8F8C100DF08F03DF808BD01B500BF042269467C480068AC3002F0F1FC18B974480099C0F89C1400BF08BD70B52DED028B04460D461646D2
:408AC0001EF0B2FBF8B16D49E0314A5D891C495D501800EBD071491000EE101AB8EEC00AB0EE408ABCEEC80A10EE101AC8B2294607F055FCBCEEC80A10EE101AC8B229461A
:408B000007F080FC0EE01EF0A7FB58B15B49E031485D294607F043FC5849E231485D294607F070FC5B4800EB8400D0ED000AB0EE600A2946204607F0ECFA56490831085D21
:408B40002A46214607F036FB52490A31085D2A46214607F097FB4F490C31085D2A46214607F0E0FB46B11D2018F094FA4448016D0120DFF810C100DFBDEC028B70BD70B584
:408B800000240CE0002506E0002229462046FFF791FF681CC5B2022DF6DB601CC4B2022CF0DB1D2018F076FA3548016D0120DFF8D4C000DF70BD70B52DED028B04460D4696
:408BC0001EF032FB00B32D48D03000EB840090ED000AB1EE400A2948D83000EB8400D0ED000A30EE200AF0EE000A80EE201AB0EE418A2046B1EE480A07F0F1FC2046B0EE04
:408C0000480A07F04AFD18E01EF026FBA8B11B48D03000EB8400D0ED000AB0EE600A204607F0DDFC1548D83000EB8400D0ED000AB0EE600A204607F030FD1048C03000EBED
:408C40008400D0ED000AB0EE600A204607F00DFC0A48C83000EB8400D0ED000AB0EE600A204607F060FCFDB1192018F013FA1D2018F010FA19200FE0F0030020182100201B
:408C800060420020892304087307002093070020F4030020FC22002018F0FCF9F848016D0120DFF8E0C300DFBDEC028B70BD10B5002405E000212046FFF77DFF601CC4B250
:408CC000022CF7DB192018F0E5F91D2018F0E2F9192018F0DFF9EA48016D0120DFF8A4C300DF10BD70B505460C4600212046FFF762FF002221462846FFF7DCFE70BD70B5B8
:408D00002DED028B05460024A1E0DF4890F8491005F1380000EB81100E3030F9140000EE900AF8EEE00AB0EE600A204607F08EFDD54890F8491005F1380000EB811012303D
:408D400030F9140000EE900AF8EEE00AB0EE600A204607F09FFDCC4890F8491005F1380000EB8110163030F9140000EE900AF8EEE00AB0EE600A204607F0B0FDC24890F83F
:408D8000491005F1380000EB81101A3030F9140000EE900AF8EEE00AB0EE600A204607F0C1FDB94991F8492005F1380101EB82110A31085D214607F0D9FDB34991F849204A
:408DC00005F1380101EB82110C31085D214607F0EBFDAD4890F8491005F1380000EB8110401C005D00EE100AB8EE400ADFEDA70A80EE201AB0EE418A2046B0EE480A07F0D1
:408E0000F1FDA14991F8492005F1380101EB8211091D085D214607F0FEFD9B4991F8492005F1380101EB8211891D085D214607F006FE954991F8492005F1380101EB821167
:408E40000831085D214607F00EFE601CC4B2022CFFF65BAF8C4890F8491005F1380000EB8110D0ED080AB0EE600A07F0B3FC864991F8492005F1380101EB8211C87807F049
:408E8000D5F9BDEC028B70BD7F4890F8280008B9012070470020FCE710B501201AF0EFFC01467B4880F8391000201AF0E8FC7849487401201AF0E3FC04462146012011F060
:408EC00059FE00201AF0DBFC04462146002011F051FE10BD01460020282901D1012200E00022402901D1012300E000231A43492901D1012300E000231A434A2901D101238D
:408F000000E000231A434B2901D1012300E000231A4302B10120704701460020562901D0782900D10120704701460020592900D10120704701460020712900D1012070473F
:408F400010B50024504890F83000912809D04E4890F83000922804D04B4890F83000712803D11EF079F900B10124204610BD464890F82810082905D0092903D00A2901D0AC
:408F80000E2901D1012070470020FCE73E4890F828100A2901D1012070470020FCE73A4890F82810082901D1012070470020FCE7354890F82810092901D10120704700204E
:408FC000FCE7314890F828100E2901D1012070470020FCE710B504461EF03EF970B11EF04EF900B92CB901212A4800781EF05EF904E00021274800781EF058F910BD224816
:4090000090F8300000EBC00101EB0010224901EB0010408E70470246012109E001EB01101E4B13F81000904201D1C8B27047491C2229F3DB0020F9E7134890ED0F0A704715
:40904000114890F84900022801D1012070470020FCE70D4890F84900012800D170470020FCE7094890F8490008B9012070470020FCE710B50024FFF7F4FF88B1012429E01E
:409080006042002089230408182100200000C84218D100206E070020E4510408604D04081EF0DAF8B0B1FFF7D4FF20B1624800781EF0FEFC68B9FFF7C3FF58B1F1F798FADA
:4090C00038B9F1F795FA28B95B4800781EF0F0FC00B90124204610BD584890F8970020B1564890F89700012801D1012070470020FCE7524890F82800072801D101207047BB
:409100000020FCE74D4890F89700022804D04B4890F89700032801D1012070470020FCE7464890F89700032801D1012070470020FCE7424890F89700022801D101207047EE
:409140000020FCE73D4890F8970008B9012070470020FCE7394890F89700012800D170470020FCE7354890F89700042801D1012070470020FCE7314890F89700042801D14D
:40918000012070470020FCE701B500BF012269462B480068973002F077F920B99DF80000264981F8970000BF08BD01B500BF012269462348006800F2853002F065F920B92E
:4091C0009DF800001D4981F8850300BF08BD10B500241A4890F83000282827D0174890F83000402822D0154890F8300049281DD0124890F830004A2818D0104890F8300045
:409200004B2813D00D4890F8300059280ED00B4890F830005C2809D0084890F83000782804D0064890F830001D2800D101242046FFF7BBFF204610BD9307002018210020EB
:40924000F00300201FB51EF02EF8062808D01EF02AF8072804D01EF026F8082841F077821EF00DF800287DD0002000900190029003460122FE4903901EF0EFF800200090CE
:409280000190029003460322FA49039001201EF0E4F8002000900190029003460322F649039002201EF0D9F8002000900190029003460322F149039010461EF0CEF80020D0
:4092C00000900190029003460322ED49039004201EF0C3F8002000900190029003460422E849039005201EF0B8F8002002220123CDE901200093039003460322E24906208A
:409300001EF0ABF8002000900190029003460246DE49039007201EF0A0F8002000900190029003460322DA49039008201EF095F8002000900190029003460122D5490390E7
:4093400009201EF08AF8002000900190029003460122D14903900A201EF07FF800200090019000E0E0E3029003460122CB4903900B201EF072F8002001210090CDE90101E3
:4093800003460A46C64903900C201EF066F8002000900190029003460246C249039011201EF05BF8002000900190029003460322BD49039012201EF050F800200222CDE9EA
:4093C000000202900346B949039016201EF045F8002001210090CDE9010103460A46B449039017201EF039F8002000900190029003460222AF49039019201EF02EF80020F9
:409400000222CDE9000202900346AB4903901A201EF023F8002000900190029001230222A64903901B201EF018F8002000900190029001230222A24903901C201EF00DF8AD
:4094400000200222CDE90002029003469D4903901E201EF002F800200222CDE90002029003460246984903901F201DF0F6FF00200090019002900346032294490390212090
:409480001DF0EBFF0020009001900290034603228F49039022201DF0E0FF0020009001900290034603228B49039023201DF0D5FF002000900190029003460322864903906C
:4094C00024201DF0CAFF0020009001900290034603228249039025201DF0BFFF0020009001900290034603227D49039026201DF0B4FF002000900190029003460122794902
:40950000039027201DF0A9FF0020009001900290034601227449039028201DF09EFF0020009001900290034601227049039029201DF093FF00200090019002900346022268
:409540006B4903902B201DF088FF002000900190029003460222674903902C201DF07DFF002000900190029003460122624903902D201DF072FF0020009001900290034609
:4095800001225E4903902E201DF067FF002000900190029003460122594903902F201DF05CFF0020009001900290034601225549039031201DF051FF002000900190029071
:4095C000034601225049039032201DF046FF00200121CDE9000103460A46CDE902104B4936201DF03AFF002000900190029003460122474903903B201DF02FFF00200090FD
:409600000190029003460122424903903C201DF024FF00200122CDE90002029003463E4903903D201DF019FF00200122CDE9000202900346394903903E201DF00EFF0020FC
:4096400001210090CDE9010103460A463449039041201DF002FF0020009001900290034601223049039042201DF0F7FE00205BE0370700205407002053070020970700204D
:40968000980700205707002058070020A3070020550700206B0700206A070020690700208B070020200700205D070020130700202A070020140700201907002099070020B2
:4096C0009A070020180700201D0700200D0700200F070020600700206107002062070020630700206507002064070020660700206707002068070020590700205B070020D7
:409700005A0700206C0700206D0700206E07002070070020710700207207002073070020740700203E07002000900190029003460122FE49039043201DF08FFE00200090E4
:409740000190029003460122F949039044201DF084FE002001210090CDE9010103460A46F449039048201DF078FE002001210090CDE9010103460A46EF4903904B201DF04E
:409780006CFE002001210090CDE9010103460A46EA4903904D201DF060FE002000900190029003460322E64903904F201DF055FE012000220092CDE9012013460246E14935
:4097C000039050201DF049FE002001210090CDE9010103460A46DC49039051201DF03DFE002000900190029003460122D749039052201DF032FE00200090019002900346C1
:409800000322D349039054201DF027FE002000900190029003460322CE49039055201DF01CFE002000900190029003460322CA49039056201DF011FE0020009001900290DB
:4098400003460322C549039057201DF006FE00200222CDE90002029003460246C049039057201DF0FAFD002000900190029003460322BC49039058201DF0EFFD0020009021
:409880000190029003460322B749039059201DF0E4FD002000900190029003460322B34903905A201DF0D9FD002000900190029003460322AE4903905B201DF0CEFD0020B2
:4098C00001210090CDE9010103460A46A94903905C201DF0C2FD002000900190029003460122A54903905D201DF0B7FD002000900190029003460122A04903905E201DF054
:40990000ACFD0020009001900290034601229C4903905F201DF0A1FD00200222CDE900020290034601229749039061201DF095FD00200222CDE9000202900346012292493B
:40994000039062201DF089FD0020009001900290034601228D49039064201DF07EFD0020009001900290034601228949039065201DF073FD002001210090CDE90101034612
:409980000A468449039067201DF067FD002001210090CDE9010103460A467F49039069201DF05BFD00200222CDE900020290034602467A4903906A201DF04FFD01200021F9
:4099C000009101910B460246CDE9021074496B201DF043FD00200222CDE9000202900346704903906D201DF038FD00200222CDE90002029003466C4903906E201DF02DFD78
:409A000000200222CDE9000202900346674903906F201DF022FD002001210090CDE9010103460A466249039073201DF016FD00200222CDE900020290034602465D490390E5
:409A400079201DF00AFD002000900190029003460222594903907A201DF0FFFC002000900190029003460122544903907B201DF0F4FC002000900190029003460122504943
:409A800003907C201DF0E9FC0020009001900290034601224B4903907D201DF0DEFC002001210090CDE9010103460A46464903907E201DF0D2FC00200090019002900346C1
:409AC0000122424903907F201DF0C7FC002001210090CDE90101034602223D49039082201DF0BBFC002001210090CDE90101034602223849039083201DF0AFFC0020012198
:409B00000090CDE90101034602223349039084201DF0A3FC01200021009101910B460222CDE902102D495BE0DAE0000075070020760700209B0700209C0700208A07002095
:409B400056070020770700207807002079070020A0070020A1070020A2070020A4070020250700207E0700207F070020800700201B070020810700208307002084070020EB
:409B8000820700205F0700205E070020850700208607002087070020890700204B070020380700209D0700209E0700209F0700208C0700208E0700208F07002031070020A4
:409BC0003207002090070020910700208D0700203B0700203C0700203D0700209307002086201DF03AFC01200021009101910B460222CDE90210FE4987201DF02EFC012035
:409C00000021009101910B460246CDE90210F94988201DF022FC002000900190029003460322F54903908E201DF017FC002000900190029003460322F04903908F201DF0C1
:409C40000CFC002000900190029003460322EC4903908F201DF001FC012009F040FD0021E84800781DF022FB0021E74800781DF01DFB0021E54800781DF018FB0021E448B0
:409C800000781DF013FB01200021009101910B460222CDE90210DF4986201DF0DEFB01200021009101910B460222CDE90210DA4987201DF0D2FB0121D84800781DF07BFF34
:409CC0000121D74800781DF076FF0121D54800781DF071FF0121D44800781DF06CFFE1E3002000900190029003460122CF4903901DF0B3FB0020009001900290034603221D
:409D0000C649039001201DF0A8FB002000900190029003460322C249039002201DF09DFB002000900190029003460322C049039010461DF092FB0020009001900290034621
:409D40000322BC49039004201DF087FB002000900190029003460422B749039005201DF07CFB002002220123CDE901200093039003460322B14906201DF06FFB00200090DB
:409D80000190029003460322A749039007201DF064FB002000900190029003460322A149039008201DF059FB002000900190029003460122A249039009201DF04EFB002059
:409DC000009001900290034601229E4903900A201DF043FB002000900190029003460122994903900B201DF038FB002001210090CDE9010103460A46944903900C201DF06A
:409E00002CFB0020009001900290034603229049039011201DF021FB0020009001900290034603228B49039012201DF016FB00200222CDE90002029003468749039016208C
:409E40001DF00BFB002001210090CDE9010103460A466E49039017201DF0FFFA0020009001900290034602227C49039019201DF0F4FA00200222CDE90002029003467849C1
:409E800003901A201DF0E9FA002000900190029001230222734903901B201DF0DEFA0020009001900290012302226F4903901C201DF0D3FA00200222CDE900020290034608
:409EC0006A4903901E201DF0C8FA00200222CDE90002029003460246654903901F201DF0BCFA00200222CDE900020290034602466049039020201DF0B0FA0020009001901A
:409F00000290034603225C49039021201DF0A5FA0020009001900290034603225749039022201DF09AFA0020009001900290034603225349039023201DF08FFA00200090AC
:409F400001900290034603224E49039024201DF084FA0020009001900290034603224A49039025201DF079FA0020009001900290034603224549039026201DF06EFA0020EE
:409F8000009001900290034601224149039027201DF063FA0020009001900290034601223C49039028201DF058FA0020009001900290034601223849039029201DF04DFAC6
:409FC000002000900190029003460222334903902B201DF042FA0020009001900290034602222F4903902C201DF037FA002059E09407002095070020440700204507002002
:40A000004307002081070020780700202A0700206D07002027070020260700205407002053070020550700205207002037070020970700209807002057070020580700202D
:40A040006B0700206A070020690700208B070020210700205D070020130700201407002019070020990700209A070020180700201D070020240700200D0700200F07002041
:40A0800060070020610700206207002063070020650700206407002066070020670700206807002000900190029003460122FE4903902D201DF0D1F90020009001900290CD
:40A0C00003460122F94903902E201DF0C6F9002000900190029003460122F54903902F201DF0BBF9002000900190029003460122F049039031201DF0B0F900200090019092
:40A10000029003460122EC49039032201DF0A5F900200121CDE9000103460A46CDE90210E64936201DF099F9002000900190029003460122E24903903B201DF08EF90020D2
:40A1400000900190029003460122DE4903903C201DF083F900200122CDE9000202900346D94903903D201DF078F900200122CDE9000202900346D54903903E201DF06DF963
:40A18000002001210090CDE9010103460A46D049039041201DF061F9002000900190029003460122CB49039042201DF056F9002000900190029003460122C749039043201F
:40A1C0001DF04BF9002000900190029003460122C249039044201DF040F9002001210090CDE9010103460A46BD49039048201DF034F9002001210090CDE9010103460A4606
:40A20000B84903904B201DF028F9002001210090CDE9010103460A46B34903904D201DF01CF9002000900190029003460322AF4903904F201DF011F9012000220092CDE9D3
:40A24000012013460246AA49039050201DF005F9002001210090CDE9010103460A46A549039051201DF0F9F8002000900190029003460122A049039052201DF0EEF80020C8
:40A28000009001900290034603229C49039054201DF0E3F80020009001900290034603229749039055201DF0D8F80020009001900290034603229349039056201DF0CDF8AB
:40A2C0000020009001900290034603228E49039057201DF0C2F80020009001900290034603228A49039058201DF0B7F80020009001900290034603228549039059201DF072
:40A30000ACF8002000900190029003460322814903905A201DF0A1F80020009001900290034603227C4903905B201DF096F8002001210090CDE9010103460A467749039096
:40A340005C201DF08AF8002000900190029003460122734903905D201DF07FF80020009001900290034601226E4903905E201DF074F80020009001900290034601226A49D1
:40A3800003905F201DF069F800200222CDE900020290034601226549039061201DF05DF800200222CDE900020290034601226049039062201DF051F800200090019002901E
:40A3C000034601225B49039064201DF046F80020009001900290034601225749039065201DF03BF8002001210090CDE9010103460A465249039067201DF02FF80020012166
:40A400000090CDE9010103460A464D49039069201DF023F800200222CDE90002029003460246484903906A201DF017F801200021009101910B460246CDE9021042496B209C
:40A440001DF00BF800200222CDE90002029003463E4903906D201DF000F800200222CDE90002029003463A4903906E201CF0F5FF00200222CDE900020290034635490390E6
:40A480006F201CF0EAFF002001210090CDE9010103460A463049039073201CF0DEFF002002225BE053E10000590700205B0700205A0700206C0700206D0700206E0700207B
:40A4C00070070020710700207207002073070020740700203E07002075070020760700209B0700209C0700208A07002056070020770700207807002079070020A00700206A
:40A50000A1070020A2070020A40700207E0700207F070020800700201B070020810700208307002084070020820700205F0700205E070020850700208607002087070020D3
:40A54000890700204B070020380700209D0700209E0700209F0700208C070020CDE90002029003460246FE49039079201CF075FF002000900190029003460222F949039075
:40A580007A201CF06AFF002000900190029003460122F54903907B201CF05FFF002000900190029003460122F04903907C201CF054FF002000900190029003460122EC49FD
:40A5C00003907D201CF049FF002001210090CDE9010103460A46E74903907E201CF03DFF002000900190029003460122E24903907F201CF032FF002001210090CDE90101A8
:40A6000003460222DD49039082201CF026FF002001210090CDE9010103460222D849039083201CF01AFF002001210090CDE9010103460222D349039084201CF00EFF01202A
:40A640000021009101910B460222CDE90210CE4986201CF002FF01200021009101910B460222CDE90210C94987201CF0F6FE01200021009101910B460246CDE90210C44961
:40A6800088201CF0EAFE002000900190029003460322C04903908E201CF0DFFE002000900190029003460322BB4903908F201CF0D4FE002000900190029003460322B749E4
:40A6C00003908F201CF0C9FE012009F008F80021B34800781CF0EAFD0021B24800781CF0E5FD0021B04800781CF0E0FD0021AF4800781CF0DBFD01200021009101910B467F
:40A700000222CDE90210AA4986201CF0A6FE01200021009101910B460222CDE90210A54987201CF09AFE0121A34800781DF043FA0121A24800781DF03EFA0121A0480078EF
:40A740001DF039FA01219F4800781DF034FA1FBD1FB50020009001900290034603229A49039001201CF079FE0020009001900290034603229549039002201CF06EFE002066
:40A78000009001900290034603229149039010461CF063FE0020009001900290034603228C49039004201CF058FE0020009001900290034604228849039005201CF04DFEF7
:40A7C0000020009001900290034603228349039006201CF042FE0020009001900290034603227F49039007201CF037FE0020009001900290034603227A49039008201CF078
:40A800002CFE0020009001900290034602225549039009201CF021FE0020009001900290034602227049039017201CF016FE0020009001900290034602466C490390192061
:40A840001CF00BFE0020009001900290034603226749039021201CF000FE0020009001900290034603226349039022201CF0F5FD0020009001900290034602224D490390CB
:40A8800027201CF0EAFD0020009001900290034602224749039028201CF0DFFD0020009001900290034602465349039029201CF0D4FD01200021009101910B460A46CDE956
:40A8C00002104E492A201CF0C8FD0020009001900290034602464A4903902B201CF0BDFD002000900190029003460122454903902D201CF0B2FD0020009001900290034675
:40A900000246414903902E201CF0A7FD0020009001900290034602463C4903902F201CF09CFD0020009001900290034602463849039030201CF091FD00200090019002900F
:40A94000034602463349039046201CF086FD0020009001900290034602462F4903905DE08E0700208F070020310700203207002090070020910700208D0700203B070020F5
:40A980003C0700203D07002093070020940700209507002044070020450700204307002081070020780700202A0700206D07002027070020260700205407002053070020A2
:40A9C0005507002052070020600700200D0700200E0700200F070020100700206307002011070020120700203F070020170700201A0700201B07002028070020210700204C
:40AA00001E07002048070020490700204A0700204B0700201C0700204D07002047201CF01CFD002000900190029003460246F649039048201CF011FD002000900190029041
:40AA400003460122F149039057201CF006FD002000900190029003460222ED49039059201CF0FBFC002000900190029003460222E84903905A201CF0F0FC002000900190DB
:40AA8000029003460122E44903905B201CF0E5FC002000900190029003460122DF4903905C201CF0DAFC002000900190029003460122DB4903905D201CF0CFFC002000901E
:40AAC0000190029003460122D64903905E201CF0C4FC002000900190029003460122D24903905F201CF0B9FC002000900190029003460122CD49039060201CF0AEFC002060
:40AB000000900190029003460122C949039061201CF0A3FC002000900190029003460122C449039064201CF098FC002000900190029003460122C049039065201CF08DFC2D
:40AB4000002000900190029003460122BB49039066201CF082FC002000900190029003460122B749039067201CF077FC002000900190029003460122B249039068201CF0B6
:40AB80006CFC002000900190029003460122AE49039069201CF061FC002000900190029001231A46A94903906A201CF056FC002000900190029003460122A54903906C2062
:40ABC0001CF04BFC002000900190029003460122A04903906D201CF040FC0020009001900290034601229C4903906E201CF035FC01200021009101910B460A46CDE9021022
:40AC000096497C201CF029FC01200021009101910B460A46CDE9021091497D201CF01DFC002001210090CDE9010103460A468D49039081201CF011FC0020009001900290E5
:40AC4000034602228849039082201CF006FC0020009001900290034602228449039083201CF0FBFB0020009001900290034602227F49039084201CF0F0FB00200090019097
:40AC80000290034602227B49039086201CF0E5FB0020009001900290034602227649039087201CF0DAFB0020009001900290034602467249039088201CF0CFFB00200090B2
:40ACC00001900290034603226D4903908D201CF0C4FB002000900190029003460322694903908E201CF0B9FB002000900190029003460322644903908F201CF0AEFB012107
:40AD0000584800781CF0D2FA0121604800781CF0CDFA01215E4800781CF0C8FA1FBD1FB500240CE000205B4901EB041189680870584901EB0411C9680870601CC4B2902C19
:40AD4000F0DB1CF005FA1DF0A3F820F011FC0121022022F0AEFF0020009001900290034601224D49039016201CF077FB002001210090CDE9010103460A46484903901E2094
:40AD80001CF06BFB002000900190029003460122434903906B201CF060FB1CF084FAFF2831D00121084622F084FF0121042022F080FF0121082022F07CFF0121102022F008
:40ADC00078FF0121202022F074FF0121402022F070FF0121802022F06CFF0121080222F068FF1CF060FA0A2862D2DFE800F06105060708095B5C5D5E00BF00BF00BF00BF99
:40AE0000FFF7A6FC55E055E01D07002051070020290700202A0700202B0700202C0700202D0700204E0700204F070020500700202E0700207107002072070020310700207A
:40AE40003207002033070020340700203507002038070020390700203A07002024070020230700203E0700203B0700203C0700203D070020540700205307002040070020C9
:40AE800043070020440700204507002041070020420700207078040813070020180700203707002000BF00BF00BFFEF7CBF900E000BF00BF1FBD10B50120FE4908701EF0D2
:40AEC00088FDFC494860012022F0A4FD1CE0612022F042FD78B145F25550F74908600120486040F6B83088604CF6CC4008600220F049087008E0EF4948681EF092FD642840
:40AF000002D90320EB490870EA4800780128DED010BD10B50020E74908704FF4FA701EF031FDFA201EF06FFDFFF7C5FFFFF7F7FE1CF07AF9C8B1E14800781CF0B9FD40B916
:40AF40000121DF4800781CF0B1F90020DD4908700BE0DD4800781CF0ABFD18B10220D949087002E00120D74908701BF0CFFBEDF7A9F900221146D548DFF854C300DF002062
:40AF800010BD10B572B66FF0040000F059FA6FF0010000F055FA4FF0FF3000F051FA042000F04EFA052000F04BFA062000F048FA072000F045FA082000F042FA092000F018
:40AFC0003FFA0A2000F03CFA0B2000F039FA0C2000F036FA0D2000F033FA0E2000F030FA0F2000F02DFA102000F02AFA112000F027FA122000F024FA132000F021FA14201E
:40B0000000F01EFA152000F01BFA162000F018FA172000F015FA182000F012FA192000F00FFA1A2000F00CFA1B2000F009FA1C2000F006FA1D2000F003FA1E2000F000FA1E
:40B040001F2000F0FDF9202000F0FAF9212000F0F7F9222000F0F4F9232000F0F1F9242000F0EEF9252000F0EBF9262000F0E8F9272000F0E5F9282000F0E2F9292000F07F
:40B08000DFF92A2000F0DCF92B2000F0D9F92C2000F0D6F92D2000F0D3F92E2000F0D0F92F2000F0CDF9302000F0CAF9312000F0C7F9322000F0C4F9332000F0C1F9342028
:40B0C00000F0BEF9352000F0BBF9362000F0B8F9372000F0B5F9382000F0B2F9392000F0AFF93A2000F0ACF93B2000F0A9F93C2000F0A6F93D2000F0A3F93E2000F0A0F949
:40B100003F2000F09DF9402000F09AF9412000F097F9422000F094F9432000F091F9442000F08EF9452000F08BF9462000F088F9472000F085F9482000F082F9492000F01E
:40B140007FF94A2000F07CF94B2000F079F94C2000F076F94D2000F073F94E2000F070F94F2000F06DF9502000F06AF9512000F067F96FF0040000F06CF96FF0010000F00F
:40B1800068F94FF0FF3000F064F9042000F061F9052000F05EF9062000F05BF9072000F058F9082000F055F9092000F052F90A2000F04FF90B2000F04CF90C2000F049F9DD
:40B1C0000D2000F046F90E2000F043F90F2000F040F9102000F03DF9112000F03AF9122000F037F9132000F034F9142000F031F9152000F02EF9162000F02BF9172000F0EA
:40B2000028F9182000F025F9192000F022F91A2000F01FF91B2000F01CF91C2000F019F91D2000F016F91E2000F013F91F2000F010F9202000F00DF9212000F00AF9222049
:40B2400000F007F9232000F004F9242000F001F9252000F0FEF8262000F0FBF8272000F0F8F8282000F0F5F8292000F0F2F82A2000F0EFF82B2000F0ECF82C2000F0E9F860
:40B280002D2000F0E6F82E2000F0E3F82F2000F0E0F8302000F0DDF8312000F0DAF8322000F0D7F8332000F0D4F8342000F0D1F835200FE0E4030020003000401E070020EE
:40B2C0003A070020E00300204B070020AF4B02089D2B040800F0BDF8362000F0BAF8372000F0B7F8382000F0B4F8392000F0B1F83A2000F0AEF83B2000F0ABF83C2000F0FD
:40B30000A8F83D2000F0A5F83E2000F0A2F83F2000F09FF8402000F09CF8412000F099F8422000F096F8432000F093F8442000F090F8452000F08DF8462000F08AF847203C
:40B3400000F087F8482000F084F8492000F081F84A2000F07EF84B2000F07BF84C2000F078F84D2000F075F84E2000F072F84F2000F06FF8502000F06CF8512000F069F870
:40B3800062B610BD38B5044660680090009D206880F3088800BFA84738BD00BFBFF34F8F3048006800F4E0602F490843001D2D490860BFF34F8F00BF00BFFEE710B5002154
:40B3C0002A4800781BF072FF0021294800781BF06DFF0021274800781BF068FF01DF10BD01B500BF04226946234800688C3000F04BF818B921480099C0F87C1400BF08BD94
:40B4000001B500BF042269461B480068903000F03BF818B919480099C0F8801400BF08BD01B500BF0422694613480068943000F02BF818B911480099C0F8841400BF08BDFE
:40B4400000F01F02012191400D4A430942F82310704700F01F02012191400A4A430942F8231070470CED00E00000FA05720700207007002071070020F40300201821002029
:40B4800080E100E080E200E070B504460D461646324629462046EDF7BEFC70BD2DE9F34F82B0844600BF00210A460B460E460F46002001908046009063E09CF80000A0F1E6
:40B4C0003004E5179CF800002E2838D1B8F1000F0CD1FA494FF00009A2FB010A03FB01A102FB0919861949EB07071FE0B8F1010F0CD1F3494FF00009A2FB010A03FB01A160
:40B5000002FB0919861949EB07070FE0B8F1020F0CD14FF47A714FF00009A2FB010A03FB01A102FB0919861949EB070708F1010000F0FF0800200090002213461BE09CF81C
:40B540000000C0B1009810B922462B460FE0009801280CDB0A214FF0000B9146A9FB010E03FB01E102FB0B19021949EB05030098401CC0B200900CF1010C0198401CC0B2CB
:40B58000019003990198884297DBB6185F413046394604B0BDE8F08F2DE9F04F83468946924600BF00BF51465846FFF777FF05460E4651464846FFF771FF07468846781B92
:40B5C00078EB060001DA012407E0E81B76EB080002DA4FF0FF3400E000242046BDE8F08F70B586B00546B7A2B9A102A823F0A8FC1022294602A8FFF7CFFF00283EDD002681
:40B60000002001900090012435E0062C0CD2DFE804F00B0C09070503AE4E08E0AE4E06E0AE4E04E0AE4E02E000BFAE4E00BF00BF9120019021200090AB4890F830000A28E8
:40B6400017D1042201A906F13000FFF71DFF0422694606F12C00FFF717FFA34890F82404A04206D19DF804009F4908639DF80000C862601CC4B2052CC7DD00BF06B070BD6D
:40B6800070B586B0054699A291A102A823F058FC1022294602A8FFF77FFF00282DDD002600200190012425E0062C0CD2DFE804F00B0C09070503874E08E0874E06E0874E2D
:40B6C00004E0874E02E000BF864E00BF00BFFF200190012201A906F2FF10FFF7D5FE824890F82404A04203D19DF80400F0F7C7FA601CC4B2052CD7DD00BF06B070BD70B542
:40B7000086B005467CA272A102A823F019FC1022294602A8FFF740FF00283FDD0026002001909FED780A8DED000A012433E0062C0CD2DFE804F00B0C09070503654E08E08B
:40B74000654E06E0654E04E0654E02E000BF654E00BF00BF002001909FED6A0A8DED000A012201A906F14300FFF78EFE0422694606F5DC70FFF788FE5B4890F82404A04289
:40B7800007D19DF80400F8F7ADFB9DED000AF8F7BAFB601CC4B2052CC9DD00BF06B070BD70B586B0054658A249A102A823F0C8FB1022294602A8FFF7EFFE00282DDD00264E
:40B7C00064200190012425E0062C0CD2DFE804F00B0C090705033F4E08E03F4E06E03F4E04E03F4E02E000BF3E4E00BF00BF64200190012201A906F56970FFF745FE3A480E
:40B8000090F82404A04203D19DF8040004F00EFD601CC4B2052CD7DD00BF06B070BDF0B585B005463BA22AA101A823F089FB1022294601A8FFF7B0FE00283CDD2A4890F85B
:40B840002464012434E0062C0CD2DFE804F00B0C090705031F4F08E01F4F06E01F4F04E01F4F02E000BF1F4F00BF00BF40F6C41000900222694607F56070FFF705FEB442EE
:40B8800004D1BDF800001849A1F880034FF47A5000900222694607F28230FFF7F5FDB44204D1BDF800001049A1F88203601CC4B2052CC8DD00BF05B0F0BD000000CA9A3BFF
:40B8C00040420F0032312E322E302E313000000025730000581B00687017006888130068A00F0068B80B00681821002032312E322E302E360000000032312E322E302E35FE
:40B900000000000035FA8E3C32312E312E302E3900000000322E342E302E3533000000002DE9F04105460E4617463A4631462846EDF7E7FA044604B103DF2046BDE8F08135
:40B94000F0B585B00546F7A2AFF27C0101A823F0F7FA1022294601A8FFF71EFE00282FDDF34890F82474012427E0062C0CD2DFE804F00B0C09070503EE4E08E0EE4E06E0E7
:40B98000EE4E04E0EE4E02E000BFEE4E00BF00BF042206F5C6716846FFF7C2FF0422694606F56270FFF770FDBC4204D19DED000ADF4880EDE20A601CC4B2052CD5DD00BF93
:40B9C00005B0F0BDF0B585B00546DFA2AFF2001101A823F0B5FA1022294601A8FFF7DCFD00282BDDD24890F82464012423E0062C0CD2DFE804F00B0C09070503CD4F08E089
:40BA0000CD4F06E0CD4F04E0CD4F02E000BFCD4F00BF00BF002000900122694607F19700FFF732FDB44204D19DF80000C04981F89700601CC4B2052CD9DD00BF05B0F0BD04
:40BA40002DE9F04186B00546C2A2AFF27C1102A823F076FA1022294602A8FFF79DFD002836DD002001900026B14890F8247400242BE0062C13D2DFE804F0130F0C090603F8
:40BA8000DFF8B0820FE0DFF8B0820CE0DFF8AC8209E0DFF8AC8206E0DFF8A88203E000BFDFF8BC8200BF00BF042201A908F1B400FFF7EAFCBC4206D19D490198C1F8B40070
:40BAC0000846C0F89860601CC4B2052CD1DD00BF06B0BDE8F081F0B587B00646A1A2AFF2102103A823F02CFA1022314603A8FFF753FD002857DD8E4890F8247400244FE08C
:40BB0000062C0ED2DFE804F00E0B09070503894D0AE0894D08E0894D06E0894D04E0894D02E000BF8E4D00BF00BF042205F1300101A8FFF7F5FE13208DF809000198FDF716
:40BB4000C9F918B90198FDF7EFF918B190208DF808000AE00198FDF7DFF918B113208DF8080002E0FF208DF8080001220DF1090105F1B300FFF788FC012202A905F1B2008D
:40BB8000FFF782FCBC4209D19DF80910684880F8B3109DF80800664981F8B200601CC4B2052CADDD00BF07B0F0BDF0B585B005466FA2AFF2E42101A823F0C2F91022294665
:40BBC00001A8FFF7E9FC00282DDD594890F8246401200090002423E0062C0ED2DFE804F00E0B09070503534F0AE0534F08E0534F06E0534F04E0534F02E000BF584F00BF3B
:40BC000000BF0122694607F14B00FFF73DFCB44204D19DF80000464981F84B00601CC4B2052CD9DD00BF05B0F0BDF0B587B0054651A2AFF2643103A823F082F9102229462A
:40BC400003A8FFF7A9FC002839DD394890F82474002431E0062C0ED2DFE804F00E0B09070503344E0AE0344E08E0344E06E0344E04E0344E02E000BF394E00BF00BF01227D
:40BC800006F1280102A8FFF74BFE9DF80800042810D0B2EE040A8DED010A042201A906F5FC70FFF7F1FBBC4204D19DED010A204880ED7E0A601CC4B2052CCBDD00BF07B080
:40BCC000F0BDF0B585B006462DA2AFF2FC3101A823F036F91022314601A8FFF75DFC00287EDD072729A2AFF2184101A823F028F91022314601A8FFF74FFC002800DD09272D
:40BD000000200090002468E0062C49D2DFE804F0494644070503074D45E0074D43E0074D41E00000322E342E302E34340000000018210020581B00687017006888130068EA
:40BD4000A00F0068B80B0068322E332E302E333000000000322E322E302E343600000000D0070068322E322E302E313800000000322E322E302E3200322E322E302E310012
:40BD8000322E312E302E373300000000322E312E302E353400000000F64D04E0F64D02E000BFF64D00BF00BF042205F130016846FFF7B6FD009838440090009814280BD3B0
:40BDC0000422694605F13000FFF75EFBEB48854202D1EB4900980863641C062C94D300E000E000BF05B0F0BD2DE9F3410D46E449ADEB010408460719DF482618AAB23946E6
:40BE00003046FFF741FBDE480719DA482618AAB239463046FFF738FBD9480719D9482618AAB239463046FFF72FFBD5480719D6482618AAB239463046FFF726FBD0480719F0
:40BE4000D2482618AAB239463046FFF71DFBBDE8FC812DE9FE4F81468A46174698460020009000262D2200233846414622F0DDFF05462D2200233846414622F0D6FF9346F7
:40BE800015B9BBF1000F35D0D5B1002416E0C4EB041000EB400048440290C4EB041000EB4000504401902D22DDE90110FFF7ECFA0646009931430091601CC4B2AC42E6D3B0
:40BEC000BBF1000F18D0C5EB051000EB400048440290C5EB051000EB4000504401901FFA8BF2DDE90110FFF7CFFA064600993143009101E0402000900098BDE8FE8F01B515
:40BF000000BF01226946A24800682D30FFF7BCFA20B99DF800109A4880F81D1400BF08BD2DE9FE4F81468A46174698460020009000262D2200233846414622F076FF054634
:40BF40002D2200233846414622F06FFF934615B9BBF1000F35D0D5B1002416E0C4EB041000EB400048440290C4EB041000EB4000504401902D22DDE90110FFF7D1FC06466F
:40BF8000009931430091601CC4B2AC42E6D3BBF1000F18D0C5EB051000EB400048440290C5EB051000EB4000504401901FFA8BF2DDE90110FFF7B4FC064600993143009187
:40BFC00001E0402000900098BDE8FE8F3EB5002002900A200190002000904FF47C71684823F035F9B0216B4823F031F94FF458716848B03023F02BF9012201A96448006800
:40C000009830FFF741FA012261480168983102A8FFF786FC9DF80800401CC0B20190012201A95B4800689830FFF72EFA012258480168983102A8FFF773FC9DF808009DF8F7
:40C040000410884207D05448007840F080005249087001248CE001224D4801682E316846FFF75EFC9DF8000044284CD0FF224FF47C71434823F0C1F84FF47C720023404983
:40C080003E48FFF7E6FE4FF47C7200233C493A48FFF7DFFE4FF47C72002339493548FFF7D8FE4FF47C72002335493648FFF7D1FE4FF47C72002332493348FFF7CAFE4FF473
:40C0C0007C7200232E493148FFF7C3FE4FF47C712B4823F0BCF8B02200232E494FF0D040FFF7B7FE4FF4587200232A49B0312B48FFF7AFFE44200090012269462448006884
:40C100002E30FFF7C1F9B02200234FF0D0412148FFF706FF4FF45872002320491D48B030FFF7FEFE01221A4801682D3119482D30FFF7F6FB124890F81D04672810D00124F0
:40C140006720FFF7DCFE4FF47C710D4823F07FF84FF47C7200230A490848FFF77AFE07E002244FF47C72002304490548FFF7D8FE20463EBDA00F0068B80B0068D00700684B
:40C18000182100208813006870170068581B0068F403002008250020ED030020F401006810B5FC48ECF7E6FD0446204610BD70B58CB000240020089009900A900B9004909D
:40C1C0000590069007900090019002900390F2490870F249087001200870FFF7E1FFFFF7F5FEEF490870EF4AAFF61C1108A822F0A7FE04A81BF044FEEBA104A823F04EF8CD
:40C2000008B1012000E00020054645B1E8A01BF023FEE5A01BF020FEE9A01BF003FE04A81BF012FE102204A908A8FFF7B5F90446DB480078012806D10020D849087008A8A4
:40C240001BF0F0FDCFE0002CFCD0002006F090F8002006F0E0F808A81BF0E4FD002C39DA0020FFF74CFEFF224FF47C71D64822F0C4FF4FF47C720023D349D448FFF7E9FDAC
:40C280004FF47C720023D049D148FFF7E2FD4FF47C720023CC49CF48FFF7DBFD4FF47C720023C949CC48FFF7D4FD4FF47C720023C549CA48FFF7CDFD4FF47C720023C24901
:40C2C000C748FFF7C6FD4FF47C71BF4822F0BFFF03DF88E0C3A2AFF60821684622F030FE102204A96846FFF757F9002838DD0020FFF705FEFF224FF47C71B34822F07DFF01
:40C300004FF47C720023B049B048FFF7A2FD4FF47C720023AC49AE48FFF79BFD4FF47C720023A949AB48FFF794FD4FF47C720023A549A948FFF78DFD4FF47C720023A249A4
:40C34000A648FFF786FD4FF47C7200239E49A448FFF77FFD4FF47C719B4822F078FF03DFA3A2AFF69421684622F0EAFD102204A96846FFF711F9002811DD012008F05DF9E7
:40C3800001219148B130FFF72FFD1AF04DFF30B10320EFF74DFE01219848FFF725FD04A8FFF78FFC04A8FFF740FC04A8FFF7FDFB04A8FFF790FB04A8FFF742FB04A8FFF787
:40C3C00001FB04A8FFF7BCFA04A8FFF728FA04A8FFF7E6F904A8FFF792F904A8FFF750F904A8FFF7FDF80020FCF754FBFCF7EFFE0646FCF7EFFD694800780CB070BD6748C7
:40C400000078704701B500BF012269467C4800683430FFF739F820B99DF800106A4880F8241400BF7748C16B0220DFF8DCC100DF08BD2DE9FE4F0746884615461E464FF08F
:40C44000000AD346714890F84200C006C10A6F4890F8410041EA00206C4991F8401040EA010908F0FBF810B907F018FCD8B1D5B1CEB14D4502D1012E00D1B2464D4502D1E9
:40C48000022E00D1B2464D4502D1032E00D1B2464D4502D1042E00D1B2464D4573D1052E71D1B2466FE0002D6DD1494C042204F1340102A8FFF734FA012204F1B10101A8A1
:40C4C000FFF72EFA0298874205D19DF80400404501D14FF0010A3F4C042204F1340102A8FFF71EFA012204F1B10101A8FFF718FA0298874205D19DF80400404501D14FF035
:40C50000020A354C042204F1340102A8FFF708FA012204F1B10101A8FFF702FA0298874205D19DF80400404501D14FF0030A2B4C042204F1340102A8FFF7F2F9012204F138
:40C54000B10101A8FFF7ECF90298874205D19DF80400404501D14FF0040A214C042204F1340102A8FFF7DCF9012204F1B10101A8FFF7D6F90298874205D19DF8040040454E
:40C5800001D14FF0050ABAF1000F62D0BAF1060F4FD23DE000380040ED030020EE030020EC0300209CBE0008322E302E310000003030303030303030303030300000000038
:40C5C000322E302E302E310018210020D0070068B80B0068A00F00688813006870170068581B0068322E302E302E363500000000322E312E302E333900000000CB2200202A
:40C60000F4030020604200208923040818D10020DFE80AF00F100C090603DFF80CB40CE0DFF808B409E0DFF808B406E0DFF804B403E000BFDFF800B400BF00BF04220BF58A
:40C64000EC716846FFF76CF90098401C08B94FF0000A5046BDE8FE8F38B5F74C042204F5EC716846FFF75CF940F2FD110098884201D0012038BDEF4C042204F5EC716846FB
:40C68000FFF74EF940F2FD110098884201D00220F0E7E74C042204F5EC716846FFF740F940F2FD110098884201D00320E2E7DF4C042204F5EC716846FFF732F940F2FD1130
:40C6C0000098884201D00420D4E7D74C042204F5EC716846FFF724F940F2FD110098884201D00520C6E70020C4E710B54FF47C71D24822F0ACFD4FF47C720023CF49D0486A
:40C70000FFF7A7FB10BD10B54FF47C71CB4822F09EFD4FF47C720023C849C948FFF799FB4FF47C720023C549C348FFF792FB4FF47C720023C149BF48FFF78BFB4FF47C72DD
:40C740000023BE49BA48FFF784FB4FF47C720023BA49B648FFF77DFB4FF47C720023B749B148FFF776FB4FF47C71B44822F06FFD10BD2DE9F0410446884615461F463CB916
:40C78000AF482E183A4641463046FEF77DFE30E0012C07D1A8482E183A4641463046FEF773FE26E0022C07D1A2482E183A4641463046FEF769FE1CE0032C07D19C482E18DF
:40C7C0003A4641463046FEF75FFE12E0042C07D196482E183A4641463046FEF755FE08E0052C06D190482E183A4641463046FEF74BFEBDE8F0812DE9F04104460F46154667
:40C8000098463CB98E482E18424631463846FFF787F830E0012C07D187482E18424631463846FFF77DF826E0022C07D181482E18424631463846FFF773F81CE0032C07D109
:40C840007B482E18424631463846FFF769F812E0042C07D175482E18424631463846FFF75FF808E0052C06D16F482E18424631463846FFF755F8BDE8F08110B56F4890F84D
:40C880002444062C2CD2DFE804F02C030B131B234FF47C72002369496748FFF7DAFA21E04FF47C72002365496248FFF7D2FA19E04FF47C72002361495D48FFF7CAFA11E065
:40C8C0004FF47C7200235D495848FFF7C2FA09E04FF47C72002359495348FFF7BAFA01E000BF00BF00BF10BD2DE9F04105460E461746984643463A4631462846FFF799FD42
:40C900000446062C5ED2DFE804F05E031527394B4FF47C72002348494848FFF701FB4FF47C72002345494648FFF793FA0120FFF769FD54E04FF47C7200233E493F48FFF70C
:40C94000EFFA4FF47C7200233C493D48FFF781FA0220FFF757FD42E04FF47C72002334493648FFF7DDFA4FF47C72002333493448FFF76FFA0320FFF745FD30E04FF47C720E
:40C9800000232A492D48FFF7CBFA4FF47C7200232A492B48FFF75DFA0420FFF733FD1EE04FF47C72002320492448FFF7B9FA4FF47C72002321492248FFF74BFA0520FFF792
:40C9C00021FD0CE000BFFFF790FE0020FFF71AFD00201C494860272014F05CFB00BF00BF04B103DFBDE8F0814FF40050704710B5124890F8240406283ED2DFE800F03E0374
:40CA00000C252D350C4C04220C493C3104F13C00FEF73AFD32E0074C042208493C3104F13C00FEF731FD29E0581B00687017006888130068A00F0068B80B006818210020B8
:40CA4000D0070068503200200F4C04220F4904F13C00FEF719FD11E00D4C04220B4904F13C00FEF711FD09E00A4C0422074904F13C00FEF709FD01E000BF00BF00BF10BDFC
:40CA80000548052170470000881300685421002070170068581B0068A59E5C1F10B51CF098FFFE49086009F0BFFDFC4880ED010A10BD10B5FA4890F84A00022824D1F8489F
:40CAC00090F8BD0102281FD1F64890ED020ADFEDF60AB4EEE00AF1EE10FA0ADBFAF70CFFC4B223467D22ED490C3101200DF046FA2EE0FAF701FFC4B223467D22E7490C31B4
:40CB000000200DF03BFA23E0E648D0ED010AE448B0F8BE0100EE100AB8EE400AF4EEC00AF1EE10FA0ADBFAF7E7FEC4B22346FA22DA490C3101200DF021FA09E0FAF7DCFE87
:40CB4000C4B22346FA22D5490C3100200DF016FA10BD10B52DED048B1AF07EFB002867D0FFF7A7FFEDF744FD18B10020CB49087261E0CA48007A60B9C84890F82000002817
:40CB800059D10120C54908721CF023FFC349086051E0C248007A01280CD1C049C86947F230511CF01CFFA0B30220BC490872FFF775FF40E0B948007A02283CD109F034FDD0
:40CBC000B648D0ED010A30EEC00A10EE104A204627F0C0F841EC190BB0EE490AF0EE690A23F092FCB0EE408AF0EE608A9FEDAF0B53EC102B51EC180B26F0B4FE0ED2A748DF
:40CC000090F82000012805D10020A44948720120087210E00120A14948720CE09F4908684FF4FA611CF0DBFE28B1FFF737FF02E000209A494872BDEC048B10BD994981F86B
:40CC400090007047974981F838007047F0EE400A9FED980A20EE800A704770B52DED0A8B82B004468E4890F8BD010F287ED2DFE800F07D365EFC37FBFAF97D7D087DF8F736
:40CC8000F600EDF7B0FC10EE105A284627F062F841EC1A0BB0EE4A0AF0EE6A0A23F034FCB0EE409AF0EE609A51EC190B26F016FAA0619FED810A84ED1C0A94ED060A84ED46
:40CCC000010AEDF7DAFC18B10020FFF7BBFF02E00420FFF7B7FF0420FFF7B0FF6AE200BF764800781AF0E4FE20B19FED750A84ED060A03E09FED700A84ED060A7148007836
:40CD00001AF0D6FE20B19FED6E0A84ED1C0A03E09FED690A84ED1C0A0420FFF793FF0420FFF78CFF94ED060A84ED010AEEE3634800781AF081FC00EE100AF8EE400A9FED93
:40CD4000621A9FED620A10EE810A84ED0C0AE16821611CF03EFEE060D4E90310091A6161D4ED0C0AB0EE600A0A2100E0BFE304F118000AF006FC94ED060ADFED550AB4EE34
:40CD8000E00AF1EE10FA03D20020FFF75BFF0FE094ED060AF0EE040AB4EEE00AF1EE10FA03DD0120FFF74EFF02E00420FFF74AFF0420FFF743FF94ED0C0AB5EEC00AF1EEB2
:40CDC00010FA02D29FED3C8A01E094ED068A94ED0F0A84ED100A84ED0F8A94ED050AB8EE400ADFED370A80EE201A11EE105A284626F0B0FF41EC1A0B94ED0F0AD4ED100A4A
:40CE000030EE600A10EE101A084626F0A3FF41EC1C0BB0EE4C0AF0EE6C0A23F075FBB0EE40BAF0EE60BA53EC1A2B51EC1B0B26F043FA41EC190B26F051F960639FED1E0A2B
:40CE400084ED1C0AB0EE480AFFF700FF84ED010AD4ED0D0AB0EE600AFFF7F8FE06E0D9E2A9E1E6E2FBE112E103E069E084ED020A4CE3124800781AF0DFFB00EE100AB8EEF0
:40CE8000400ADFED110A20EE200ADFED120A80EE201A84ED0C1AD4ED0C0A1DE018290020182100203C29002000C0DA44000000401857B63FC0A9064600000000520700201F
:40CEC00000007A44560700203333533A9A99193FCDCCCCBE0CAC233FB0EE600A0A2104F118000AF04EFB94ED060ADFEDFE0AB4EEE00AF1EE10FA03D20020FFF7A3FE0FE064
:40CF000094ED060ADFEDF80AB4EEE00AF1EE10FA03DD0120FFF796FE02E00420FFF792FE0420FFF78BFE1FED1C0A84ED1C0AD4ED060AB0EE600AFFF789FE84ED010AE5E201
:40CF4000EA4800781AF078FB00EE100AF8EE400A1FED231A1FED230A10EE810A84ED0C0AD4ED0C0AB0EE600A0A2104F118000AF008FB94ED060A5FED2A0AB4EEE00AF1EE30
:40CF800010FA03D20020FFF75DFE0FE094ED060AF0EE040AB4EEE00AF1EE10FA03DD0120FFF750FE02E00420FFF74CFE94ED0C0AB5EEC00AF1EE10FA02D21FED418A01E03C
:40CFC00094ED068ACA4800781AF036FB00EE100AF8EE400A1FED441A1FED440A10EE810A84ED220AD4ED220AB0EE600A0A2104F170000AF0C6FA94ED1C0A5FED4B0AB4EE10
:40D00000E00AF1EE10FA03D20020FFF717FE0FE094ED1C0AF0EE040AB4EEE00AF1EE10FA03DD0120FFF70AFE02E00420FFF706FE94ED220AB5EEC00AF1EE10FA02D25FED04
:40D04000628A01E0D4ED1C8AB0EE480AFFF7FEFDB0EE401AB0EE680AFFF7F8FD31EE400A10EE105A284626F075FE41EC1A0BB0EE4A0AF0EE6A0A23F047FAB0EE409AF0EEA0
:40D08000609A51EC190B26F029F860603EE2974800781AF0D1FA00EE100AB8EE400A5FED760A20EE200A5FED750A80EE201A84ED0C1AD4ED0C0AB0EE600A0A2104F11800B5
:40D0C0000AF05FFA94ED060ADFED860AB4EEE00AF1EE10FA03D20020FFF7B4FD0FE094ED060ADFED810AB4EEE00AF1EE10FA03DD0120FFF7A7FD02E00420FFF7A3FD7C4898
:40D1000000781AF099FA00EE100AB8EE400A5FED920A20EE200A5FED910A80EE201A84ED221AD4ED220AB0EE600A0A2104F170000AF027FA94ED1C0ADFED6A0AB4EEE00A73
:40D14000F1EE10FA03D20020FFF778FD0FE094ED1C0ADFED650AB4EEE00AF1EE10FA03DD0120FFF76BFD02E00420FFF767FD94ED060AD4ED1C0A30EE600A10EE101A0846EB
:40D1800026F0E8FD41EC1B0BB0EE4B0AF0EE6B0A23F0BAF9B0EE40AAF0EE60AA51EC1A0B25F09CFF09EE100AB0EE490AFFF74EFD84ED010AAAE16421E0681CF010FCE8B3C9
:40D1C0001CF007FCE06094ED0F0A84ED100A494800781EF0A4FB00EE100AB8EEC00A84ED0F0A94ED0F0AD4ED100A30EE600A10EE101A084626F0AEFD41EC1A0BB0EE4A0A8B
:40D20000F0EE6A0A23F080F9B0EE409AF0EE609A51EC190B25F062FF2063D4ED0C0A9FED361A80EE810AF2EE040A80EE201A84ED0C1AD4ED0C0AB0EE600A00E00EE00321BC
:40D2400004F118000AF09DF994ED060A84ED010A0420FFF7F7FC0420FFF7F0FC56E16421E0681CF0BCFB00287DD01CF0B2FBE06094ED0F0A84ED100A1C4800781EF04FFB63
:40D2800000EE100AB8EEC00A84ED0F0A94ED0F0AD4ED100A30EE600A10EE101A084626F059FD41EC1A0BB0EE4A0AF0EE6A0A23F02BF9B0EE409AF0EE609A51EC190B25F0FA
:40D2C0000DFF206394ED0C0ADFED0B0A80EE201A84ED0C1A94ED250A84ED260A074800780EE00000CDCCCC3C33339F40520700205507002054070020CDCCCC3D560700206D
:40D300001EF00DFB00EE100AB8EEC00A84ED250A94ED250AD4ED260A30EE600A10EE101A084626F017FD41EC1A0BB0EE4A0AF0EE6A0A23F0E9F8B0EE409AF0EE609A51ECDF
:40D34000190B25F0CBFE8821085194ED220A5FED160A80EE201A84ED221AD4ED0C0AB0EE600A032100E054E004F118000AF009F9D4ED220AB0EE600A032104F170000AF0A3
:40D3800000F994ED060AD4ED1C0AB4EEE00AF1EE10FA04DD94ED060A84ED010A03E094ED1C0A84ED010AEDF768F918B10020FFF749FC13E094ED1C0AD4ED060A30EE600A37
:40D3C000F3EE090AB4EEE00AF1EE10FA03DD0220FFF738FC02E00420FFF734FCEDF75AF918B10020FFF72AFC13E094ED060AD4ED1C0A30EE600AF3EE090AB4EEE00AF1EEDE
:40D4000010FA03DD0220FFF719FC02E00420FFF715FC7BE09FEDFB0A84ED0C0A9FEDF90A84ED010A0420FFF70DFC0420FFF706FC6CE0FA21E0681CF0D2FAE8B36A4601A98F
:40D44000F14800781EF0BEFB05461CF0C2FAE06094ED0F0A84ED100A9DED000A84ED0F0A94ED0F0AD4ED100A30EE600A84ED0C0A94ED0C0AF5EE000A80EE201A11EE106A75
:40D48000304626F067FC41EC1A0BB0EE4A0AF0EE6A0A23F039F8B0EE409AF0EE609A51EC190B25F01BFE2063D4ED0C0AB0EE600A022104F1180000E018E00AF062F894ED85
:40D4C000060A84ED010A012D06D19DED010AB5EEC00AF1EE10FA03D10020FFF7B3FB02E00420FFF7AFFB0420FFF7A8FB0EE09FEDC50A84ED0C0A9FEDC30A84ED010A0020F0
:40D50000FFF7A0FB0020FFF799FB00BF00BF02B0BDEC0A8B70BD10B519F0B1FED0B1FAF7EBF9C4B22346FA22B84900200CF026FD9FEDB40AB64880ED060A9FEDB20A80ED8D
:40D54000060A042180F8381080F890100020B14948722EE0AE48FFF780FBAF48B0F8BE0118B90220A949087521E0A948D0ED010AA948B0F8BE0100EE100AB8EE400AF4EEA9
:40D58000C00AF1EE10FA09DBFAF7B6F9C4B22346FA229E4901200CF0F1FC08E0FAF7ACF9C4B22346FA22994900200CF0E7FCFFF7D0FA10BD97494872704731B50024BDF851
:40D5C0000000C82803DDC8200090022406E0BDF80000012802DA01200090032400BF022269468E48006800F5DF70FDF74DFF20B9BDF800008849A1F8BE0100BF204638BD20
:40D6000031B50024BDF80000642803DD64200090022406E0BDF80000012802DA01200090032400BF022269467C48006800F5DF70FDF72AFF20B9BDF800007749A1F8BE0148
:40D6400000BF204638BD31B50024BDF80000B0F5FA7F04DD4FF4FA700090022406E0BDF80000012802DA01200090032400BF022269466A48006800F5DF70FDF705FF20B936
:40D68000BDF800006449A1F8BE0100BF204638BD31B50024BDF80000322803DD32200090022406E0BDF80000012802DA01200090032400BF022269465848006800F5DF703F
:40D6C000FDF7E2FE20B9BDF800005349A1F8BE0100BF204638BD31B50024BDF80000C82803DDC8200090022406E0BDF80000012802DA01200090032400BF022269464748F4
:40D70000006800F5DF70FDF7BFFE20B9BDF800004149A1F8BE0100BF204638BD31B50024BDF8000040F26351884203DD08460090022406E0BDF80000012802DA012000905E
:40D74000032400BF022269463448006800F5DF70FDF79AFE20B9BDF800002F49A1F8BE0100BF204638BD31B50024BDF8000045F2CC01884203DD08460090022406E0BDF8B8
:40D780000000012802DA01200090032400BF022269462248006800F5DF70FDF775FE20B9BDF800001C49A1F8BE0100BF204638BD10B52DED028BB0EE408A0024164890F83A
:40D7C000BD010E2853D2DFE800F0072B08122C091336522D4052493700BF00BFBCEEC80A10EE101A88B2FFF7BEFF044648E000BFBCEEC80A10EE101A88B2FFF78FFF044612
:40D800003EE000000000000052070020F82900203C2900201829002018210020F003002000BF00BFBCEEC80A10EE101A88B2FFF752FF044624E000BFBCEEC80A10EE101A6A
:40D8400088B2FFF725FF04461AE0BCEEC80A10EE101A88B2FFF7F7FE044611E0BCEEC80A10EE101A88B2FFF7CBFE044608E0BCEEC80A10EE101A88B2FFF79FFE044600BFC3
:40D8800000BF4120EFF766FE0020FFF793FE2046BDEC028B10BD10B52DED020B00BF04226946F748006800F5E670FDF7EDFD20B99DED000AF34880ED730A00BFF248016DA5
:40D8C0000120DFF8C8C300DF1CBD10B52DED020B00BF04226946EA48006800F5E470FDF7D3FD20B99DED000AE64880ED720A00BFE548016D0120DFF894C300DF1CBD10B51C
:40D900002DED020B00BF04226946DD48006800F5E270FDF7B9FD20B99DED000AD94880ED710A00BFD848016D0120DFF860C300DF1CBD10B52DED020B00BF04226946D04880
:40D94000006800F5E070FDF79FFD20B99DED000ACC4880ED700A00BFCB48016D0120DFF82CC300DF1CBD10B5C64890F83000912809D0C44890F83000922804D0C14890F823
:40D980003000712818D1BF4890F8BD010A2813D19FEDBF0AFFF70CFF9FEDBE0AFFF7C9FF9FEDBD0AFFF7ABFF9FEDBC0AFFF78DFF9FEDBB0AFFF76FFFB24890F83000702824
:40D9C00004D0B04890F83000932819D1AD4890F8BD010A2814D19FEDB30AFFF7E9FE9FEDB20AFFF7A6FF9FEDB10AFFF788FF9FEDB00AFFF76AFF9FEDAF0AFFF74CFF18E0BC
:40DA0000A04890F8BD010A2813D19FEDA60AFFF7CFFE9FEDA00AFFF78CFF9FED9F0AFFF76EFF9FEDA50AFFF750FFBBEE040AFFF732FF944890F8BD01012804D1B7EE000A27
:40DA4000FFF7B6FE53E08F4890F8BD01022804D19FED9A0AFFF7ACFE49E08A4890F8BD01032804D1B3EE040AFFF7A2FE3FE0854890F8BD01042804D11FED9E0AFFF798FEE4
:40DA800035E0804890F8BD01052804D19FED8C0AFFF78EFE2BE07B4890F8BD01062804D19FED880AFFF784FE21E0764890F8BD01072804D0734890F8BD010D2804D1B1EE3E
:40DAC000040AFFF775FE12E06E4890F8BD01092804D19FED7C0AFFF76BFE08E0694890F8BD010C2803D1B2EE040AFFF761FE10BD10B5644890F8BD010A2817D1614890F891
:40DB00003000912809D05F4890F83000922804D05C4890F83000712803D1FA20FFF793FD03E04FF49670FFF78EFD00E000BF00BF10BD00B589B019F08FFB002879D051486A
:40DB400090F8BD010E2875D2DFE800F074072A2B4E7576C274FDFCFBFAF9002000900190029003460246584903900846007819F074FC00200090019002900346024653492E
:40DB800003900846007819F068FC01214E4800781AF011F801214D4800781AF00CF899E100BF002000900190029003460322464903900846007819F050FC00200090019027
:40DBC000029003460322414903900846007819F044FC03213C48007819F0EDFF03213B48007819F0E8FF75E101200021009101910B460A46CDE9021033490846007819F066
:40DC00002CFC01200021009101910B460A46CDE902102E490846007819F01FFC01212A48007819F0C8FF01212848007819F0C3FF50E150E129E100BF0020009001900290DE
:40DC400003460322204903900846007819F005FC0020009001900290034603221B4903900846007819F0F9FB00211748007819F0A2FF00211548007819F09DFF2AE1000027
:40DC8000F003002018210020604200208923040800007A43C6DCB53DB8AF833E52B8444114AE4740000096436744293EE5F25F3E52B862416666E6C133331B410000164393
:40DCC0000080BB440000C8425207002055070020002000900190029003460222F84903900846007819F0B9FB002000900190029003460322F34903900846007819F0ADFB88
:40DD0000002000900190029003460222EE4903900846007819F0A1FB0221E948007819F04AFF0221E848007819F045FF002000900190034614220121029004A804E092E0C2
:40DD400072E01EE0A3E0A1E01DF008FC04A8DFEDDF0A9FEDDF0A02230022DE490090D84800781DF0E3FA04A8DFEDD80A9FEDD80A02230322D8490090D34800781DF0D6FAB5
:40DD8000A8E0002000900190029003460222CC4903900846007819F060FB002000900190029003460322C74903900846007819F054FB002000900190029003460222C2497C
:40DDC00003900846007819F048FB0621BC48007819F0F1FE0621BC48007819F0ECFE002000900190034614220121029004A81DF0B5FB04A8DFEDB50A9FEDB50A02230022A7
:40DE0000B4490090AE4800781DF090FA04A8DFEDAF0A9FEDAF0A02230322AF490090AA4800781DF083FA55E0002000900190029003460222A24903900846007819F00DFB4A
:40DE400001219F48007819F0B6FEA448DFED9F0A9FEDA30A052300229E490090984800781DF064FA36E0002000900190029003460322944903900846007819F0EEFA0021A7
:40DE80009048007819F097FE24E000BF00BF002000900190029003460322894903900846007819F0DAFA002000900190029003460322844903900846007819F0CEFA01214F
:40DEC0007F48007819F077FE01217E48007819F072FE00BF00BF834890F8BD01824908700020FFF767FB00208049087209B000BD7F49097D012900D100E00021084670471A
:40DF00007B48407D70477A48007D08B9012070470020FCE7774909880143764A11807047F7EE000AB0EE600A7C2202706D4A92F8BD210E2A22D2DFE802F007120809130AE0
:40DF40000B1721141B211E1800BF00BF00BF00BF01224270DFED680AB0EE600A0FE000BF00BF022242700AE000BF0422427006E00522427003E00622427000E000BF00BF23
:40DF8000594AD2ED060A60EE800AFCEEE00A10EE902A91B281700A0AC270534AD2ED1C0A60EE800AFCEEE00A10EE902A91B201710A0A42714B4AB2F8BE1181710A0AC27168
:40DFC0007047494890ED010A704701B500BF012269464A48006800F2BD10FDF755FA20B99DF800003F4981F8BD0100BFFFF7BBFC012003F07DF81E20EFF7ACFA08BD01B5F0
:40E0000000BF022269463D48006800F5E870FDF73BFA20B9BDF800003249A1F8D00100BF08BD00202F4991F8BD110E291AD2DFE801F01A0D0A070E0B0810131B151917113D
:40E0400000BF012011E000BF01200EE000BF01200BE000BF012008E0012006E0012004E0012002E000BF00BF00BF00BF704700201C4991F8BD110E291DD2DFE801F01D0FC6
:40E080000B07100C0812151E171C1A1300BF40F2635013E000BF45F2CC000FE000BFC8200CE000BF322009E0C82007E04FF4FA7004E0642002E000BF00BF00BF00BF704737
:40E0C0005207002055070020560700200000000000504347000400400000014030DC002000247449182100203C29002018290020F8290020FC030020C0A90646F0030020DB
:40E100000020C84991F8381009B9142012E0C54991F83810012901D116200BE0C14991F8901009B9152005E0BE4991F89010012900D11720704770B50424BB4880780A2857
:40E1400076D2DFE800F0051376C5C5C5C5BFC1C30020B5490870C8808860FFF750FFB2488078B149487001208870B2E0FFF7C8FFAD4908700846007810B10720887056E05A
:40E18000A948806820B91BF024FCA74988604EE0A54988684FF47A711BF021FC002846D0FFF70FFFBCEEC00A10EE100A85B22846FFF725FF9D48B0F8AC0068B19B48B0F8DE
:40E1C000AC009A49B1F8D011884205DD9748B0F8AC009549C88021E09448B0F8D001002803DC01209049C88018E0904890F8BD01032804D08D4890F8BD01062805D18B485B
:40E20000B0F8D00100F5FA7006E08848B0F8D0018000032190FBF1F08349C8800220824988701BF0D6FB804988600020087350E04EE0FFF7C6FE7C48C08800EE900AF8EE14
:40E24000600AB4EEE00AF1EE10FA05DB7648007B401C7549087302E0002073490873FFF74FFF714908700846007810B10720887027E06D48007B04280DDB6B48C08800EE88
:40E28000900AF8EE600AB0EE600AFFF791FA09206549887015E06449886841F288311BF09EFB70B16048C08800EE900AF8EE600AB0EE600AFFF77CFA07205B4988701820A2
:40E2C000087006E0012404E0022402E0032400E000BF00BF5448007818B153490878F8F7CDFB204670BD5048807870474E480078704700204C498870C870704701B500BFCA
:40E30000022269464A480068AC30FDF7BDF820B9BDF800004549A1F8AC0000BF08BD10B52DED028B414890F8BD0103280ED03F4890F8BD01062809D03C4890F8BD0102289A
:40E3400004D03A4890F8BD0105280CD114F0FAF910B1012806D102E0B7EE008A02E09FED358A00BF01E0B7EE008AB0EE480ABDEC028B10BDB7EE000AF0EE400A2B4890F86D
:40E38000BD010E2818D2DFE800F007100809110A0B1317121417151600BF00BF00BF00BF1FEDAB0AF0EE400A07E000BF00BF00BF00BF00BF00BF00E000BF00BF194890ED66
:40E3C000060A20EE200A7047B7EE000AF0EE400A164890F8BD010E2818D2DFE800F007100809110A0B1317121417151600BF00BF00BF00BF1FEDC00AF0EE400A07E000BF4C
:40E4000000BF00BF00BF00BF00BF00E000BF00BF044890ED1C0A20EE200A70470648407A704700003C290020102A002018210020F0030020D7A3DC4018290020B5EEC00A77
